:020000040800F2
:10000000F0FF0220A9540508F1540508D1C80108E1
:10001000F1540508F1540508F154050800000000EA
:10002000000000000000000000000000F15405087E
:10003000F154050800000000F1540508459E010830
:10004000F1540508F1540508F1540508F154050868
:10005000F1540508F15405087DB2000885B2000886
:100060008DB2000895B200089DB20008F154050851
:10007000F1540508F1540508F1540508F154050838
:10008000F1540508F1540508F1540508F154050828
:10009000F1540508F1540508F1540508A5B200080B
:1000A000F1540508F1540508F154050829D9000850
:1000B00039D9000849D9000859D90008A9A700086A
:1000C0009DA70008F1A70008E5A70008F15405085E
:1000D000F15405080D970108DD970108AD98010856
:1000E000ADB20008F1540508F1540508F1540508B3
:1000F000F1540508F1540508F1540508F1540508B8
:10010000F1540508F154050869D90008F1540508AF
:100110007D9901084D9A0108F1540508F15405082C
:1001200065AF000879AF00088DAF0008A1AF0008E7
:10013000B5AF0008F1540508F1540508F15405085D
:10014000F1540508F1540508F15405082DD40008B0
:10015000C9AF0008DDAF0008000000001D9B0108CA
:1001600039A800082DA800080000000000000000C9
:10017000F1540508F1540508F15405080000000089
:1001800000000000F1540508ED9B0108BD9C01082A
:10019000F15405080000000000000000000000000D
:1001A000000000000000000000000000F1540508FD
:1001B000F154050800000000F1540508000000009B
:1001C000000000000000000000000000000000002F
:1001D0000000000000000000F1540508F15405087B
:1001E000F154050841D30008F1540508F1540508FD
:1001F000F1AF000805B0000819B000082DB00008E4
:0C02000041B0000855B0000869B00008CB
:1080000030B5EAB18E464FEA014C034600F1C00597
:10801000002419689A6841EA0C0142EA0E029A604B
:10802000C3E900140C33AB42F3D1D0F8C030C0F830
:10803000C44043EA0E03C0F8C030C0F8C84030BDA9
:108040004FEA014E8C46E0E710B40C4C2368002B3D
:1080500011DD002004F1040C0146DCF8743003F15A
:10806000C00259600C339342FBD123680130834234
:108070000CF1AC0CF1DC5DF8044B7047E01600200D
:1080800070B5474C04EB401393F8D02202B970BD91
:108090004C2202FB004294F8145694F815E692F82C
:1080A000B66383F8B66275454FF000034FEA401C93
:1080B00082F8B6330CD00EEB4E0304EBC30393F8F7
:1080C0001826561E012E4FEA4E035BD9032A53D0C1
:1080D00004EB0C00A0F8B412EFF31182902383F3A9
:1080E000128890F8B632B0F8B41243EA4103002186
:1080F000D2B29BB280F8B61282F311881A0994F8B2
:10810000781682EA13225A40D1B1D0F8CC42D0F886
:10811000B812646FD2431B019BB202F00F02012020
:108120008840134304F1C0015A0013F4004F93B286
:1081300002D16268024362600C348C42F4D170BD9B
:10814000D0F8CC12D0F8B8024C6F1B0100F110012E
:108150009BB202F00F0201208840134304F1C001DA
:108160005A0013F4004F93B202D162680243626076
:108170000C34A142F4D170BD0EF1010202F00302F1
:10818000AA42A5D0734404EBC303184490F8251603
:1081900000299DD004EB0C03012283F8B62297E757
:1081A000E0160020704700BF704700BF024B03EB92
:1081B000401090F8D1027047E01600204368826CAE
:1081C00010B49A61EFF31182502383F3128841684F
:1081D000C46B0B6823EA0403446C2343D2B20B60E4
:1081E00082F31188D0E907418268036912681C6034
:1081F0005960D0E909419C60D960B0F85C10D16247
:1082000000235DF8044B0376704700BF026890F8C6
:1082100010C01168022303FA0CF3194200D1704711
:1082200010B4074C41684FF0000C84F879C6086818
:108230006CF3000008605DF8044B5360704700BFAA
:10824000E0160020704700BF0B4890F8B01689B1C7
:1082500001EB4101002310B4490000F5D7601C4632
:1082600050F82320063302B114608B42F8D15DF838
:10827000044B7047704700BFE01600200B4890F891
:10828000B01689B101EB4101002310B4490000F59B
:10829000D7601C4650F82320063302B1146099427F
:1082A000F8D15DF8044B7047704700BFE01600201E
:1082B00001207047034B00EB400003EBC00090F837
:1082C000C9067047E01600201F4890F8B036CBB3BF
:1082D00000222DE9F04100F5D7631C4F50262C25D4
:1082E000144607E053F8181B0C6090F8B0160132E2
:1082F000914225DD197C0029F4D059684FEA912E6E
:10830000AEF5801EBEF1530F4FF0FE0C98BF17F86C
:108310000EC0EFF3118E86F31288D1F8248005FB8E
:108320000C0C08F10108CCF8A087D1F8148048F0B3
:1083300001085FFA8EFCC1F814808CF31188D1E734
:10834000BDE8F081704700BFE0160020006C050812
:1083500007EE900AB8EE670A704700BFBCEEC00A8D
:1083600010EE103A98B2704708B51D200FF09CFF30
:1083700008B183794BB11E200FF096FF08B18379C5
:1083800003B108BD5523C38008BD5523C380F2E760
:10839000704700BF704700BF704700BF704700BF05
:1083A00001207047094A0A4BD2F8BC29D3F8900241
:1083B000526AD3F8941292F85330012B08BFB2F8E6
:1083C0005030A0EB010008BFC0187047E016002035
:1083D000D8270020012380F85130704710B4EFF304
:1083E0001181802383F312880C4AC9B2D2F89832E3
:1083F000D2F89C42D2F89802D2F89C2281F31188DC
:10840000904203F1FF33A3EB04038CBF0020012053
:1084100003EBC0205DF8044B704700BFD827002055
:108420004A4B4B4A1B6893424CD015D9494A934258
:1084300051D027D9484A934256D002F1B77202F57B
:10844000585293427DD1454BD3F8A4200B2161F3C0
:108450000F32C3F8A4207047414A93424DD020D92F
:10846000404A934252D002F1B77202F558529342F9
:108470006AD13A4BD3F8A420052161F30F32C3F837
:10848000A4207047384A934249D0384A93425AD17F
:10849000324BD3F8A420062161F30F32C3F8A42095
:1084A0007047334A934243D002F1B77202F55852F3
:1084B000934247D1294BD3F8A4206FF30F32C3F86E
:1084C000A4207047254BD3F8A420042161F30F3278
:1084D000C3F8A4207047214BD3F8A420092161F3ED
:1084E0000F32C3F8A42070471C4BD3F8A4200821F6
:1084F00061F30F32C3F8A4207047184BD3F8A420BF
:10850000032161F30F32C3F8A4207047134BD3F853
:10851000A420022161F30F32C3F8A42070470F4B4F
:10852000D3F8A420072161F30F32C3F8A4207047C9
:108530000A4BD3F8A420012161F30F32C3F8A42021
:108540007047704770477047704700BF00000020B9
:10855000007A030A001C4E0E0052BC0F0038024085
:1085600000D8B805000E270700B0710B00E6DF0C3D
:10857000006CDC02074BD0F894105B68D0F8A020A8
:108580005B1A9A42B8BFC0F8A030012380F8CC3003
:1085900000207047001000E003689A69D10508D5F3
:1085A0004FF4807213218177DA611A6822F0800219
:1085B0001A609A69920508D54FF4007213218177E9
:1085C000DA611A6822F080021A609A69510508D5AA
:1085D0004FF4806213218177DA611A6822F08002F9
:1085E0001A609A69120508D54FF400621321817749
:1085F000DA611A6822F080021A609A69D10408D5FB
:108600004FF4805213218177DA611A6822F08002D8
:108610001A609A69920408D54FF4005213218177A9
:10862000DA611A6822F080021A607047184BD3F89A
:10863000A012D3F8A4228A1A322A15D8D3F8B82265
:108640008A4200D37047D3F8A822E2B1106892881A
:1086500010B44469224218BF120432315DF8044B51
:108660008261C3F8B8127047D3F8A8223AB193F8E0
:10867000B40291881268C00748BF090491610022C2
:10868000C3F8B82270473231C3F8B812704700BF40
:10869000D8270020064AD2F8A8323BB192F8B4128B
:1086A0009A881B68C90748BF12049A610020704766
:1086B000D82700204FF40070034B1060D3F8C83265
:1086C0000B600020704700BFD827002000207047B3
:1086D0000120704701207047002070470123437735
:1086E00000207047D0E90B2108B583690B448361F2
:1086F0000AB108469047002008BD00BF436A1B68C6
:108700001B6A5B685B78024613F0010008BF507774
:10871000704700BF70B5224A224C234B94B00546E7
:10872000CDE90042214A0992A4F108020A922A7F67
:108730000493201D0023CDE905039A42CDE90E33B1
:108740000B931093139314BF0520042011936B6AAD
:108750000C9002200122029018688DF80C200E4621
:1087600007928DF820208DF834208DF848204BF0AA
:10877000BDFA2B7F93B1330E04F8073C063C320C54
:10878000330A22706370A670686A69460FF0E8F8D1
:108790006B6A18684BF0AAFA14B070BD073CEEE79C
:1087A000D02A00200C000020FD860008DD8600088D
:1087B00010B5044694B05022064968464EF058F968
:1087C000606A69460FF0CCF8636A18684BF08EFA5D
:1087D00014B010BD546C0508C2628161704700BFBF
:1087E0002DE9F0410446406A00681E460F46904657
:1087F0004BF07CFA237F002B37D0254DA069052351
:10880000EB64030E6B7505F116039870020C000AF9
:1088100058701A703B68AB650020D8F800302B66A2
:10882000012E2363286727D0022E1CD1D8F80420FC
:10883000A866796885F86400E966134415496A6793
:108840000120236385F87800E967134B617F606A34
:1088500003F11402002914BF194611460FF080F8E5
:10886000E36A83B1206BBDE8F081094DA069042360
:10887000EB6405F11503C8E7064B85F86460C5E9AC
:108880001A306867E1E7636A18684BF02FFAE9E786
:1088900000000020E58600081C000020704700BF93
:1088A00000B583B081610192049A0093C2620123F2
:1088B0006A4601A9FFF794FF03B05DF804FB00BF0F
:1088C000043070470D4B93F80023D3F8FC12024498
:1088D000D2B283F8002393F8002308441206C3F8A9
:1088E000FC0205D593F8002382F0800283F8002370
:1088F000034B012283F89420704700BFD827002043
:10890000000000202DE9F047144FD7F80453ED0A7A
:108910001ED00026B04607F54F79D7F80833104827
:10892000D3F828A0C7F83483AC19641010234A4642
:10893000E102D0470F280BDD0A4B03F1100C53F86E
:10894000041B013107D16345F9D12546B542E4DC6A
:10895000E802BDE8F087661CF8E700BFD8270020D2
:10896000E02A0020142B0020012141F20102002303
:1089700041F2011C017202804FF60B71FF22A0F838
:1089800004C043818381C38101828274704700BF28
:10899000164BFF224FF0FF3CF0B5C270027102721D
:1089A0004272427382738274C27403F11207664684
:1089B000172516244FF0150E002202EB82028118B3
:1089C000BB4200F802E04C708D70CE7081F804C09C
:1089D0000BD093F9062093F807E01C7A5D7A93F99F
:1089E0000A6093F90BC00633E7E7F0BDA46C0508F5
:1089F0004FF0000C01210222032380F805C0817191
:108A0000C2710372704700BF4FF4F07140F22E4CF8
:108A100001804FF47A71A0F81EC041844FF4FA6CC3
:108A20004FF4F5610122A0F820C0818440F2262C89
:108A300042F22011A0F81CC0418142F2267C0E2196
:108A40008271427440F201220723A0F808C080F826
:108A500026104FF0000C40F20341828240F2056282
:108A60008370A0F812C0C18202838376704700BF72
:108A70008388C3F30B039342A8BF134670B51A460D
:108A80001D460C46064680684DF0F2FF621994427E
:108A9000B569074B08D0074814F8011B00FB03F326
:108AA000A24283EA0103F7D12B60012070BD00BF11
:108AB000C59D1C81930100010023037043708370E6
:108AC000C37070470023037043708370C370704796
:108AD00000220123027042708270C27003714371E0
:108AE0008371C371704700BFFF23037043708370AD
:108AF000C3707047002306214FF47A72C0E9012346
:108B000001700373704700BF10B50023411CFF22A2
:108B100000F8132001F8132001330B2BF8D10C4B74
:108B20004FF0FF3103F1180400228C4605E013F9E1
:108B300002CC13F9011C13F8032C00F812C000EB4F
:108B4000420E03339C428EF80110F0D110BD00BFDD
:108B5000BF6C05084FF0260C2721022280F800C0C8
:108B6000C1704FF0200C0321427180F806C0C27121
:108B70004FF0210C0172827204212C22012380F813
:108B800009C0C1724FF0000C02731221FF22437022
:108B900083700371437380F80EC0C1730374427411
:108BA000704700BF03230370704700BF0A4491421F
:108BB00019D000B501F1FF3C02F1FF3E41F2210165
:108BC0001CF8012F082380EA022010F4004F81EAEC
:108BD00040020ABF400090B280B2013BF5D1E645A9
:108BE000EED15DF804FB7047704700BFD0ED007A0E
:108BF000D0ED016A30EE677AE6EE877AB0EE670A6A
:108C0000C0ED007A704700BFD0ED017AD0ED026A66
:108C100030EE677A90ED000AE6EE877A37EEC07A9A
:108C2000C0ED017AA6EE870A80ED000A704700BF0A
:108C300090ED017AD0ED036AD0ED027A30EE470A6A
:108C4000A6EE807A90ED000A80ED017A37EE676A31
:108C5000E6EE867A37EEC07AC0ED027AA6EE870A93
:108C600080ED000A704700BFDFED277AB4EEE70A17
:108C7000F1EE10FA0CDDDFED256A9FED257AF0EEBE
:108C8000407AF4EEC77AF1EE10FA30EE660AF6DCBE
:108C9000DFED207AB4EEE70AF1EE10FA0CD5DFED45
:108CA0001B6A9FED1D7AF0EE407AF4EEC77AF1EE82
:108CB00010FA30EE260AF6D4DFED187AB4EEE70AA1
:108CC000F1EE10FA14DDDFED107A37EEC00A60EE37
:108CD000006A9FED136A9FED137ADFED137AA6EE1B
:108CE000867A20EE266AE6EE877AA6EE270A704795
:108CF000DFED0E7AB4EEE70AF1EE10FA44BFDFEDD5
:108D0000057A37EEC00AE2E7DB0F4940DB0FC940C6
:108D1000E4CB1641DB0F49C0E4CB16C1DB0FC93FE2
:108D200092E741B99730083C15A82ABEDB0FC9BFAE
:108D3000D0ED056AD0ED017A90ED007A90ED066AEB
:108D4000D0ED025A90ED035A80ED050A66EEA77A3F
:108D5000C0ED066AE7EE007A90ED077AE5EE867AD6
:108D600090ED086AD0ED045A80ED087AE5EE477A76
:108D7000E5EEC67AB0EE670AC0ED077A704700BF2D
:108D8000D0ED057A90ED006A90ED067AD0ED035AA9
:108D9000E6EE007A90ED016AF0EE406AA6EE267AE1
:108DA000B0EE670AD0ED047A90ED026A67EEC07A01
:108DB000A5EEC07AE6EE267A80ED057AC0ED067A59
:108DC000704700BF2DE9F047089F3C460E4614F857
:108DD000011B002B054614BF4FF030094FF020094E
:108DE00041B3002A2CDD234600E0B2B113F8010B99
:108DF0009046013A0028F8D1A8F102086AB1C246AB
:108E000049462846B0475346002B0AF1FF3AF7DCA3
:108E1000397828EAE872013249B1D71B2846B047B1
:108E2000E01914F8011B0029F8D1BDE8F0871046BD
:108E3000BDE8F087002A02F1FF38E0DC0846F4E7DD
:108E40000022EAE703685A1C02601970704700BFED
:108E5000024BD3F84C0303681B681847D82700203F
:108E6000884210B54FF001043ED301FB04F4B0FB7F
:108E7000F4FC8C45F9D2CCB122BB08E0A14203F846
:108E800001EBB4FBF1F211D8B0FBF2FC1446BCF1DB
:108E9000090F0CF1570E0CF1300204FB1C00EDDC45
:108EA000A14203F8012BB4FBF1F2EDD900221A70B4
:108EB00010BDA14203F801EBB4FBF1F2F6D8B0FB10
:108EC000F2FC1446BCF1090F0CF1370E0CF1300224
:108ED00004FB1C00EDDCA14203F8012BB4FBF1F212
:108EE000EDD900221A7010BD8446002AEAD1CEE7DF
:108EF000002870B503DA2D2301F8013B4042092810
:108F000086464FF0010307DD03EB83035B00B0FBF4
:108F1000F3F2092AF8D8EBB1104CBEFBF3FCA4FB2A
:108F20000320C008BCF1090F0CF130060CF1570505
:108F3000024607D8092B01F8016B03FB1CEE09D987
:108F40000346EAE7092B01F8015B03FB1CEE01D99C
:108F50001346E2E700230B7070BD00BFCDCCCCCC34
:108F6000F8B5164D6B78BE2B26D1022229464FF656
:108F7000FF70FFF71BFE124FAC1C22884AB1A618E7
:108F8000BE4219D2052A17D92146FFF70FFE3446F3
:108F9000F3E721460222FFF709FE0222A118FFF79C
:108FA00005FE0634074B641BA3F8504341F60F53EC
:108FB000C31A58425841F8BD0020FCE700400008A1
:108FC00000800008D827002010B5084C084843F05E
:108FD000CDFD4022002104F555704DF0ACFD4FF061
:108FE000FF33C4F89433C4F8973310BDD82700205A
:108FF0000E004400114B002130B50160818003F167
:109000000C054FF448748E460A4602EB420200EB10
:10901000420C00F812E08CF80110DA788CF802208B
:10902000AB42ACF8044007D093F9062093F807E070
:10903000197A5C890633E8E730BD00BFD46C0508B7
:10904000092900D001B9704701394B0003F008022B
:10905000930001F00301A3EB9203C1EB0111C3EBF9
:109060000313C1EB011100229B0089000260818083
:1090700043807047F8B5164D1648174F00214FF43E
:109080000F724DF058FD05F644364FF0804105F65D
:1090900028343A46002301E054F8332091420BD0A3
:1090A00001330F2BF8D100201C3548F0E5FEB54206
:1090B0000CD055F81C1CECE7084A02EBC3031C3526
:1090C00093F8300C48F0D8FEB542F2D1F8BD00BF9D
:1090D000046D0508581E002000000140006C0508C2
:1090E00030B4436919690A686FF300020A609A682C
:1090F000B3F80CC01468E26822EA0C02E26004686B
:1091000090F810C02068082202FA0CF202403AD10E
:10911000224890F87856022000FA0CF06060002D8A
:109120002FD0187E01282FD0D3F8A0100131C3F81A
:10913000A010EFF31180502181F312885C68DD6B81
:10914000216821EA05011D6C2943C0B2216080F32A
:10915000118898681969DC6A00680C601C6B4C60A7
:109160005C6B8C609C6BCC604262B3F87C20C2620A
:109170000A68012422430A601C76C2689B89134353
:10918000C36030BC7047FEE7D3F8A4000130C3F8D9
:10919000A4000B6862F300030B60F2E7E016002006
:1091A0001A4A0368934210B504460AD0184A9342FB
:1091B00013D0184A93421CD01A6842F001021A6078
:1091C00010BD154843F0D2FC14492368D1F820287B
:1091D00022F40012C1F82028EEE7114843F0C6FC43
:1091E0000E492368D1F8202822F48002C1F82028F3
:1091F000E2E70C4843F0BAFC08492368D1F820287C
:1092000022F40002C1F82028D6E700BF0054004035
:1092100000580040005C0040150020000030024073
:1092200016002000170020003D2202230270437028
:10923000704700BF4FF4007141F20142002340F239
:109240001F4C0180428040F68C210122A0F806C00C
:10925000038143818181C281704700BF2DE9F041C4
:109260001A4D10F00DFE2968002907464FF0000640
:109270004FF0AC0817DD00231C4608FB03520133F6
:1092800092F8A1208B4244EA0204F6D110F0F8FDD6
:10929000C01B2643B0F5FA6FF6B206DC2CB1296884
:1092A00000292646E7DC10F0EBFD26B1084B93F8C9
:1092B0009B23542A02D03046BDE8F081B3F8A023A6
:1092C0000132A3F8A0233046BDE8F081E01600206B
:1092D000D8270020C94B93F878360BB90120704786
:1092E0002DE9F04FC64FC749D7F8A022C64BA1FBC6
:1092F00002125209A3FB023B4FEADB0B0BEB8B0B79
:1093000085B0A2EB4B0B5FFA8BF3039307F28C63F0
:109310000193BA4B07F56B7A03F52D7900230AEB1D
:109320008B0B1D46D7F89C37AB4240F31A81D9F816
:109330001830D9F80460D3E9258410F0A1FD4FEA74
:10934000860E0EF1085E0EEB481E97F89B83029086
:1093500004F1806197F894073939B8F1540F0EEB96
:1093600081110EEB801301D1A7F8A203994240F2BC
:109370006B811A68002A00F05F811A6C002A00F0E5
:109380007181D3F88020002A00F06E81D3F8C020CC
:1093900003F58073002AE9D1A3EB0E0E99424FEA40
:1093A000AE1E40F25181A4EB0E0145294FF000049E
:1093B00028BF452103EB81119C46204626460DE03F
:1093C0001A6C002A40F0D480D3F88020002A40F0A4
:1093D000FA80D3F8C02003F580732AB9994206D9E0
:1093E0001A68002AECD04033994200F2C580112E51
:1093F000344640F22D81D6F1150200F129818349CE
:10940000029ED1F898309E45D7F8983738BFC1F8FA
:1094100098E0F11A002919DB03F5F42303F59073A2
:109420009E4288BF029B794988BF0533C7F89837A9
:10943000764BD3F89830052B86BF053BDBB2002373
:1094400087F894374FF0FF33C1F8983042B100FAF3
:1094500002F2C4F11404012000FA04F444EA020008
:109460006B4BC0F3C43203EB8202D2F8A44C00F081
:109470001F0203EB8202D2F8A41CC0F3441203EBD8
:109480008202C0F3842003EB8000D2F8A43C41EABE
:10949000043141EA0311D0F8A43C41EA032181EAF6
:1094A000112383EA131303F00F030F2B40F0B48052
:1094B000B1F5803F80F0B080B8F1540F4FEA111140
:1094C00004D1B7F89C330133A7F89C33D7F894360E
:1094D000B1F5606F03F10103C7F8943600F0D58051
:1094E000019B99819AF858300398834214D0DBF895
:1094F0000820DAF800309B1ACAF80030DBF8302078
:10950000DAF804309B1ACAF804300023CBF808308C
:10951000CBF830308AF85800DAF800300133CAF856
:109520000030DBF808300133CBF808304FF6FF731A
:10953000994209D1DAF804300133CAF80430DBF873
:1095400030300133CBF83030019B01351433082D16
:109550000AF15C0A0BF15C0B019309F120097FF41D
:10956000E1AE0123012087F8903705B0BDE8F08F08
:10957000803399427FF63BAFA3EB0C029211541C4F
:10958000244A82FB04C2A2EBE472012AB8BF012282
:10959000904001241644013A04FA02F210431C469A
:1095A000226892B1226C002A60D0D4F88020002A70
:1095B0005ED0D4F8C02004F580743AB1A142EFD84F
:1095C0009C4623460AE7C0330EE74034A142F7D950
:1095D000E31A9B115A1C0F4B83FB02C3A3EBE273EC
:1095E000012BB8BF012398401E440122013B02FA1F
:1095F00003F3184323469C462346EFE6E01600207B
:10960000D82700201F85EB51CDCCCCCC000000200A
:10961000006C050856555555B8F1540F2AD0D7F8A7
:1096200094360133C7F89436D7F890360133C7F82B
:1096300090364FF6FF7155E74033A3EB0E0E99427B
:109640004FEAAE1E3FF6AFAE10B1013887F894076F
:10965000B8F1540F7FF478AFB7F89E330133A7F811
:109660009E3371E7803397E6C03395E68034ADE7EB
:10967000C034ABE7B7F89C330133A7F89C33D7F875
:1096800094360133C7F89436CEE7084A92F8153677
:1096900003EB430302EBC3032B4493F825360D2B56
:1096A0007FF41EAF019A802393771BE7E01600201A
:1096B00010B504464CF040FC81B22046BDE8104095
:1096C000FEF7DEBC38B50B4D00EB400005F5D76367
:1096D00003EBC00393ED027AD3ED037AE7EE007A51
:1096E000C4002C44B0EE670A4CF026FCD4F8B8361F
:1096F000186038BDE0160020F8B51F4E96F8142605
:1097000096F815369A4231D13568002D12DD0024C5
:1097100096F878661948274606B3037E012B20D0B9
:1097200002691368013443F00103AC4200F1AC005C
:109730001360F1D110F0A4FB114BD3F8A047002C1B
:109740000BDD03F2A47303EBC40419689A88C8689C
:1097500008330243A342CA60F7D1F8BDFEF72EFDDD
:10976000DEE780F89C70FEF729FDD9E748F054F950
:109770000028C9D1F8BD00BFE0160020E416002083
:10978000D827002038B51A4B93F8142693F81536CD
:109790009A4228D1174D95F8C4371BB34FF0000CEF
:1097A00005F5F9626146136859621868083261F379
:1097B000C710186032F8040CD862186840F08000B6
:1097C0001860186861F341001860DC6832F8020C18
:1097D00095F8C4E70CF1010C2043E645D86022F867
:1097E000021CE0DC38BD48F017F90028D2D138BDA2
:1097F000E0160020D82700200C4AF8B513685569F8
:109800002B4003EA000555617DB1094F0126B5FAE9
:1098100085F4C4F11F0407EB840306FA04F4D3F8BB
:10982000540303689847A543F1D1F8BD003C0140BB
:10983000D82700200269C3682DE9F04712EA03091E
:109840002AD005460E464FF000474FF00008B9FAFF
:1098500089F327FA03F2D2431B3B2A6109EA020982
:10986000042B16D8DFE803F0332A221A0300B36A68
:10987000002B35D003F1FF3A1FFA8AFAC6F8288088
:10988000746A34B123682046514698476468002CB6
:10989000F8D1B9F1000FDAD1BDE8F0877068A98E70
:1098A00003689847B9F1000FD1D1F5E7B068298F67
:1098B00003689847B9F1000FC9D1EDE7F068E96B8B
:1098C000036889B29847B9F1000FC0D1E4E7306965
:1098D000296C036889B29847B9F1000FB7D1DBE76B
:1098E000E96A1FFA81FACBE730B5124A124CD2F876
:1098F000303883B043F00103C2F830384FF4C0551C
:109900004FF0817369462046CDE9005343F0C4F916
:10991000636A23F470236362636A43F420236362FF
:10992000636A23F470436362636A43F420436362AF
:1099300003B030BD00300240000002402DE9F04786
:1099400004460068237C0268022101FA03F31A42EC
:1099500001D1BDE8F087D4F814A0DFF878829C4AE2
:10996000DFF874925268C9F808284C2707FB0A8769
:10997000D7F8BC23B7F8C0131668D7F8F453F268C9
:1099800022EA0102F2602A686FF300022A6098F866
:10999000782612B94360BDE8F087284643F0F4F812
:1099A000D9F81038012287F8E023002B00F00A8153
:1099B00033686FF3C71333604C2303FB0A834FF004
:1099C000FF3293F8F033F262062B29D8DFE813F068
:1099D000D2002800AA002800820028000700336A6D
:1099E0006FF30C3333624C2303FB0A83326A93F820
:1099F000F11361F34D323262F26993F8F21361F3BD
:109A00000922F26193F8F323F36962F30F33F361F0
:109A1000F3696FF38B23F361336A43F4805333624A
:109A20002A684C2303FB0A834BF6EF7002400020A8
:109A3000A3F8D4032A602968B3F8D4230A432A6020
:109A40002A6893F8DD1361F30D322A602A6893F8CF
:109A5000DB1361F38B222A602A6893F8DA1361F32F
:109A600009222A602A6893F8D91361F3C7122A6081
:109A700093F8D8132A6861F386122A6093F8DC13EE
:109A80002A6861F345122A60B3F8D6136A6861F355
:109A90000F026A60D3F8CC23AA60D3F8D023EA601F
:109AA000D3F8F42316215160116841F001011160CF
:109AB000D3F8BC23B3F8C03312682068D1680B43D5
:109AC000D360434A237C5168C9F80C18022202FA79
:109AD00003F35FE7336A6FF3082333624C2303FB1E
:109AE0000A83316A93F8F12362F349213162316AC2
:109AF000C2F3400262F3CB213162F26993F8F213B0
:109B000061F30102F26193F8F323F36962F307133F
:109B1000F361F3696FF38303F361336A43F4807392
:109B200033627DE7336A6FF3041333624C2303FB24
:109B30000A83316A93F8F12362F345113162316A85
:109B4000C2F3400262F3C7113162B26993F8F213B3
:109B500061F30922B26193F8F323B36962F30F331F
:109B6000B361B3696FF38B23B361336A43F01003BE
:109B7000336255E7336A6FF3000333624C2303FB10
:109B80000A83316A93F8F12362F341013162316A49
:109B9000C2F3400262F3C3013162B26993F8F21377
:109BA00061F30102B26193F8F323B36962F307131F
:109BB000B361B3696FF38303B361336A43F00103A5
:109BC00033622DE710F05CF9C9F81008F0E600BF29
:109BD000001000E0E0160020D827002038B51E4C09
:109BE000D4F8903273B1D4F89422D4F890329A42D7
:109BF00008D0D4F89432E218013392F81408C4F86B
:109C0000943238BD154BD3F8BC390022596AC4F8D8
:109C1000942291F8533003F0FF05ABB1B1F85050E6
:109C200081F853205DB193B2C8182344007983F8BA
:109C30001408B1F85000013293B29842F3D80848A2
:109C40004022043147F0FCFDC4F89052D4F8900251
:109C50000028CED1D5E700BFD8270020E01600208D
:109C60009820002090F850305A1C0344D2B280F85B
:109C7000502083F83C1090F851300BB1132A01D9D1
:109C80004AF0BEBC704700BF002280F851204AF065
:109C9000B7BC00BF38B544F0DFFA214B93F8A141BF
:109CA0002922012C23F8862C23F87E2C01D00120B8
:109CB00038BD1C4DC3F8A451FFF716FE1A4842F0F8
:109CC00055FFFEF7ADFB47F03FFF184A02F5805302
:109CD0004FF0A04083F8784383F88543C2F8B40975
:109CE000816B41F40011816305F1200205F1480107
:109CF0000F4DC3F87C534FF40165A3F87A534FF42A
:109D000081750024A3F8805383F8834349F09CF8BD
:109D1000224621464FF0FF3043F006F8204638BD7A
:109D2000D03800209C00002007003400E0160020FE
:109D3000400040012DE9F0430446406A354D00687B
:109D400095B00E469146984649F0D0FF324B0193AC
:109D5000324B049305F58A730093217F022302930B
:109D600005F58672012300278DF80C3005920697C1
:109D7000002937D08DF834308DF84830CDE9097797
:109D8000330ECDE90E77CDE9107785F80D31052337
:109D9000CDF82C908DF82070CDF83080139705F514
:109DA00087750793330C1E4F2B70330A6B70AE70A0
:109DB000D7F8AC01656A0DF0F5FE637FA8803BBB68
:109DC00005A928460DF0CCFD636A186849F08EFF9E
:109DD000D7F8B0010DF0E6FE636A9880404615B0F2
:109DE000BDE8F0838DF834308DF848300423CDE998
:109DF0000911CDE90E11CDE91011CDF82C908DF897
:109E00002010CDF83080139105F20D150793C9E7A6
:109E10006946D6E700000020783A0020FD86000859
:109E2000D03800202DE9F047089F884615460021CC
:109E3000202204461E464CF07EFE4FB13B68E38173
:109E40001B0C23827B687A89E3821B0C628223834A
:109E500040464AF029FCEB0619D4431EB8B108EB82
:109E6000000701E0013B12D317F801CDBCF12E0F22
:109E7000F8D1C01A421E032AA8BF0322082B03F1FF
:109E8000010AA8BF08239146C2441A4606E00828E2
:109E90000246C246A8BF08224FF000094FF0203307
:109EA00041462360636004F1080720464CF0E0FD62
:109EB000174B23815146BB704A4638464CF0D8FDBB
:109EC000611EE31D11F801CFACF1610EBEF1190F57
:109ED0009CBFACF1200C81F800C08B42F2D1384617
:109EE00004F10B0110F8013BA3F16102192A9CBF98
:109EF000203B00F8013C8842F4D118232373330C33
:109F0000A382E572099B6683E361BDE8F08700BF29
:109F1000202020002DE9F04FDFF88094D9F8A0022E
:109F2000C9F8A40287B0002B00F0D88001F5FE78B4
:109F30001344DFF86CB40393164601F12007C246C0
:109F40001FE0002E62D0D9F8D432B34200F0CA80AC
:109F5000D9F8D032B34200F0FD80D9E9B631B3422E
:109F60004BD8B14200F29781711A204646F0E0F9D1
:109F7000039B01369E4207F500770AF5007A00F050
:109F8000AD80D9F8E052B542A7F12004D9D8751BAD
:109F9000D9F8F08205F00702EB080492D8F83020D7
:109FA0000233934203D3D8F8382093420BD9414669
:109FB0001846059346F08CF9059B8046002800F072
:109FC0008A81C9F8F00298F80420002A40F0328112
:109FD000D8F82850002D00F07781D8F830209B1A4F
:109FE000049A02EBC303D8F80C20204602EB43226C
:109FF0004FF400714346A847BAE7B142B4D92046AE
:10A000004FF4007200214CF096FDB1E74FF400725E
:10A01000314620464CF08FFD802387F89E310C237B
:10A0200087F8A231D9F8D032D34AD9F8C812C4F887
:10A03000C6319342C4F8CA1100F33281CF4AD04CE2
:10A0400082FB03021A44D817C0EB621284FB02544D
:10A05000CC4D85FB03C5C0EB2530C2EB821587F8DC
:10A06000A1015B1B801020F03F0001330343144427
:10A0700087F8A031D317C3EBE4142244BE4B87F812
:10A080009F214A1E9A4200F31781BC4BBC4883FBB8
:10A0900002311144D317C3EB611180FB0140B94C6D
:10A0A00084FB0254C3EB2433C1EB811487F8A53140
:10A0B000121B9B1023F03F0301321343084487F81F
:10A0C000A431CB17C3EBE010014487F8A31155234B
:10A0D00087F8DE31AA2387F8DF3149E7002007B08F
:10A0E000BDE8F08F4FF0FF3384F8EC3184F8ED31A8
:10A0F00084F8EE3184F8EF31D9F8E832C4F8E83169
:10A100005223237063706123A37084F8E7314123E5
:10A110000025E37084F8E631722384F8E43184F892
:10A12000E5314FF4F0722946A7F11C004CF003FD15
:10A130005523C7F8D051C7F8D451C7F8D85184F87F
:10A14000FE316FF0550384F8FC5184F8FD5184F81A
:10A15000FF310DE700214FF4007220464CF0EBFC7C
:10A16000894A03CA47F81D0CEB2007F8200C582039
:10A1700007F81F0C902047F8191C07F81E0C002345
:10A1800002220821F820E372227307F8131CA2733D
:10A19000E37307F8102C07F80B0CD9F8D00284F8F9
:10A1A0002C20D9F8C8226376121A2262D9E9B602A5
:10A1B000121A3F2020764FF0FF30A0763E20207705
:10A1C0000120E3766377A377E37784F82D3084F872
:10A1D0002E3084F82F30626284F8300084F83130F9
:10A1E00087F82610802187F82010292187F822106F
:10A1F000942187F823100E2187F824100D21634A3B
:10A2000087F82510552187F8DE11AA2187F8DF117C
:10A2100003CA5F4BC7F82700C7F82B1003CB13887E
:10A22000A7F82F309378C7F83200C7F8361087F8B0
:10A2300031309DE64FF40072002120464CF07BFC4B
:10A24000049B002B4ED1D8F84030002B00F0AA80A0
:10A25000049AD8F830304F49CDE900222046112227
:10A26000FFF7E0FDD8F840301A6C002A00F0AD800E
:10A27000049A1B6BCDE90022474911223846FFF7AB
:10A28000D1FDD8F8448007F120044FF4E075B8F10F
:10A29000000F3FD16CE6F11A204646F049F867E618
:10A2A000FF2387F89F3187F8A13187F8A031324B1F
:10A2B0004A1E9A427FF7E9AEFF2387F8A33187F859
:10A2C000A53187F8A43102E7294620464FF40072F1
:10A2D0004CF031FC4CE6A7F1240343F804BF9A4547
:10A2E000FBD145E6D8F84030049AD8F84480002BDA
:10A2F0000CBF01230223C3EB02154346002B3FF49E
:10A3000037AE013D9B6CF9D198464FF40075002B98
:10A310003FF42EAE2544203423462035444604968F
:10A3200098460EE05CF81C1B236BCDF800C000269D
:10A330000196FFF777FDA46C08F12008CCB1A84581
:10A3400017D02379A44604F11C0E1122A8F1200095
:10A35000002BE7D162792669236B216842F0210244
:10A36000CDE900E6FFF75EFDA46C08F12008002CA3
:10A37000E5D1049EFCE500BFFF03FB0083200882BB
:10A38000818080809755454158E2050864E20508C0
:10A3900070E2050850E2050854E20508D8270020BD
:10A3A000DEADBEEF049BD9F8CC12CDE900332046D8
:10A3B0000822FFF737FDD8F84480B8F1000F3FF4CA
:10A3C000D7AD3C464FF4F075A4E7049BCDE90033CC
:10A3D00052E700BF38B590F82830012B044604D06E
:10A3E000407F40B10023637738BD406A03681A7B21
:10A3F00092B9637F0BB9012038BD0A4D0A49022387
:10A4000005F5DA720DF0DCFA95F8B53103F00103C9
:10A4100083F001006377E7E71B6A002BE9D0002097
:10A4200038BD00BFD0380020180100202DE9F041D0
:10A430000446154E90F82800637F144F06F5DA782D
:10A44000012805D00BB1002363770120BDE8F0811E
:10A45000606A05682A7B82B9002BF6D00223424647
:10A4600039460DF0ADFA96F8B53103F00103637784
:10A47000002BEAD094F82800E2E72A6A002AE8D103
:10A48000002BE2D0EAE700BFD038002018010020FE
:10A49000F0B511F0010583B00AD190F82860012EC3
:10A4A000044607D0C368B3F1807F01D90123237725
:10A4B00003B0F0BD0A4B476AD3F8AC010DF072FB54
:10A4C000E368B880B3F1807FF2D9B7218DF804102A
:10A4D000267733462A46384601A90DF071FAE7E798
:10A4E000D0380020144B154910B5044618681B7964
:10A4F000206284F82430152204F125004CF06CFB16
:10A500000F4B93F8B6214FF0010E84F83AE012B9E0
:10A5100084F83B2010BD03F5DC7CBCE80F00206014
:10A520006160A260E360BCE80F0084F83BE020615A
:10A530006161A261E36110BD7CE2050884E2050867
:10A54000D038002010B50021382204464CF0F3FA30
:10A550000D490E4A0E482061C4E905120D480E4A05
:10A56000E061012341F61E614FF0090CE18484F89B
:10A5700008C0A37384F82130A26221460748BDE8D1
:10A58000104030F0B7BF00BF1A046C070019750304
:10A590006400DC0543080E001E7D010194E20508FD
:10A5A0002DE9F041584F3B78B12B8AB070D1FEF7BE
:10A5B000D7FC80F00104E4B2544B554DB3F8243D70
:10A5C000544EADF8003004F00104B54262D3002CC3
:10A5D00000F097801022002106A84CF0ACFA4E4BF8
:10A5E0004E494F4A0497DB1B05934E4B484F596029
:10A5F0005A6059645A6401228DF824203422DA60AA
:10A600006946022204A80025089549F0DFFB0222D2
:10A6100069464FF6FF70FEF7C9FA0446B74246D3C3
:10A62000022201A904A80025ADF8045049F0CEFB90
:10A63000022201A92046FEF7B9FA40BAC043ADF89C
:10A640000800022204A802A949F0C0FB079860B1E3
:10A6500006ABC0F10402294618444CF06CFA06A976
:10A6600004A806F0DFFACDE907509DF824300898D9
:10A6700043B12C4B1A6942F080021A611A6D42F004
:10A6800080021A65B0FA80F040090AB0BDE8F08196
:10A69000012491E7A988A868C1F30B0145F05CFB90
:10A6A000AB691B681C35834218BF01248DE7B7F8DE
:10A6B00004808DF80D50C8F30B0808F10603ADF8BF
:10A6C00008303B88C3F30B02ADF80A201B0B0622AF
:10A6D00002A904A88DF80C3049F078FB062202A9E3
:10A6E0002046FEF763FAB9680446424604A849F0DA
:10A6F0006DFBB96820464246FEF758FA1C370446FF
:10A700008CE70120C1E700BF00400008006C05088D
:10A71000B86C0608607406080080000823016745CD
:10A72000AB89EFCD003C0240174A1849D2F8883077
:10A7300030B443F47003C2F888300B6843F001036F
:10A740000B600B689B07FCD58B68104A6FF3010305
:10A750008B60936813F00C0FC3F38101F9D1916002
:10A76000136809480A4D23F0867323F4803313607D
:10A770004FF41F044FF000635560C2F8A010D4607E
:10A7800030BC8360704700BF00ED00E0003802403D
:10A7900002300300704700BF002070470148FDF7FA
:10A7A000FBBE00BFC03A00200C4BD3F80832023B7E
:10A7B000072B11D8DFE803F00D0D0A0A0707040480
:10A7C000074849F0CDBC064849F026BD044849F089
:10A7D000A1BD034849F046BE704700BFD0380020F5
:10A7E000C03A00200148FDF7D7BE00BF143B00204F
:10A7F0000C4BD3F85C32023B072B11D8DFE803F097
:10A800000D0D0A0A07070404074849F0A9BC0648C9
:10A8100049F002BD044849F07DBD034849F022BE1D
:10A82000704700BFD0380020143B00200148FDF7DE
:10A83000B3BE00BF683B00200C4BD3F8B032023BE4
:10A84000072B11D8DFE803F00D0D0A0A07070404EF
:10A85000074849F085BC064849F0DEBC044849F089
:10A8600059BD034849F0FEBD704700BFD0380020F5
:10A87000683B0020F0B40668D6E9041574684A689D
:10A88000A36813F08003FBD1002D00F09080686175
:10A890000F7CD1F800C06968022000FA07F747F082
:10A8A0000C07CCF804702F7C2D68B84040F00C00E9
:10A8B0006860106863F300001060086863F30000CC
:10A8C00008600B68B06943F002030B6013684BF635
:10A8D000EF752B401360176803893B4313601368BF
:10A8E000477C67F30D3313601368C77B67F38B23D3
:10A8F0001360877B136867F309231360477B136832
:10A9000067F3C7131360077B136867F3861313603D
:10A910001368077C67F3451313605368478967F32F
:10A920000F035360F369066840689660D06008685A
:10A93000284008600D6818892843086008685D7C15
:10A9400065F30D300860DD7B086865F38B200860D7
:10A950009D7B086865F3092008605D7B086865F3E6
:10A96000C71008601D7B086865F3861008600868DA
:10A970001D7C65F34510086048685D8965F30F002C
:10A980004860D3E900038860CB600B6843F00103A3
:10A990000B60136843F001031360636843F0010325
:10A9A0006360636843F002036360F0BC7047486112
:10A9B000087C09680223834043F00C034B60136852
:10A9C00065F3000313601168B3694BF6EF70014043
:10A9D000116010681989014311601168587C60F397
:10A9E0000D3111601168D87B60F38B211160116803
:10A9F000987B60F3092111601168587B60F3C711DF
:10AA000011601168187B60F386111160187C116861
:10AA100060F3451111605889516860F30F0151606E
:10AA2000D3E900139160D360136843F0010313600E
:10AA3000136843F002031360636843F0020363602A
:10AA4000F0BC7047F8B505462C6895F83870636817
:10AA5000012284F824201A686FF386121A60A888ED
:10AA60002289824219D0B0F5807F0246A8BF4FF4F8
:10AA70008072022AB8BF02221968002A92FAA2F252
:10AA8000B2FA82F208BF4FF0FF32013A21F03801EA
:10AA900041EAC20292B21A6020812A7BA17A9142D5
:10AAA0000AD01968002A72D06FF341011960196841
:10AAB0006FF300011960A2721A6842F040021A6036
:10AAC000216A8A68002A79D000200646143116448B
:10AAD0008A680130002AF9D1227B62B15FB1012876
:10AAE00072D8072E70D800EB80029200216A0A44C7
:10AAF000127B002A68D0226A92680026002A4FD072
:10AB00000EB1327B22B1AA6812B1116892888A62B2
:10AB1000226A1768226A5168226A926802F1FF3C31
:10AB200092B117B33A4612F8010B17469A6892078A
:10AB3000FCD5D8609A68D207FCD5DA6809B101F86B
:10AB4000012BBCF1010CECD2236A1B7BC3B9236A35
:10AB50001B6963B1236A686C1B69984701280AD096
:10AB6000022804D100232362F8BDFF20DEE7266A15
:10AB7000236A14332362236A9B688BB16368BFE73F
:10AB8000AB68002BE3D01A689B889361DFE741F044
:10AB900002011960196841F001011960A2728BE786
:10ABA000236A1B68002B35D0236A1D68236A596805
:10ABB000236A21620022C3E9002245E7217B0029A4
:10ABC00099D0002F92D196E7206AA3698268016824
:10ABD000B9B159600121597392B25A812B685B69EE
:10ABE00033B14168E369B9B10120596058735A81A2
:10ABF000AB6813B11A689B8893622846BDE8F84099
:10AC000038E659730649FF2681F81A6101F58D71FE
:10AC10005960E1E72362F8BD024858605973E6E7DE
:10AC200000000020F83B002038B5D0F890102B4BE6
:10AC300004465A68D0F8880071B1131A99420BDCA7
:10AC400094F88030C4F88820012B10D0D4F88430D8
:10AC50000133C4F8843038BDD4F89430C4F8882067
:10AC60000344C4F88C3094F88030012BEED1616835
:10AC7000201D04F19805EFF3118C102383F3128843
:10AC800063681B6A0BB3D4F8A0302A461BB1D369A2
:10AC90001432002BFBD10B6A6BB1996839B993421E
:10ACA00009D0196829B15B6899680029F7D0143375
:10ACB000F3E7C3E900055FFA8CFC8CF31188D4F844
:10ACC00084300133C4F8843038BD0D625FFA8CFCE7
:10ACD0008CF31188FFF7B6FEB8E700BF001000E064
:10ACE0002DE9F041826992F88C30012B8AB005463B
:10ACF00049D0023B012B50D892F8FC30D26C2D4C3D
:10AD000063F07F0313708669336DD6F8108003F10A
:10AD1000010E0FCCEC46ACE80F00F36CCDE9003E21
:10AD20000FCCACE80F0094E8030006F110078CE8A4
:10AD30000300EFF31180102383F3128833691B6A39
:10AD4000002B2ED0029B6A461BB1D3691432002B14
:10AD5000FBD1D8F8203073B1996839B993420AD041
:10AD6000196829B15B6899680029F7D01433F3E7B3
:10AD70001F60C3F804D0C0B280F31188AA691169BA
:10AD80000B6A002BFCD1136D5A8852BAEA819A885B
:10AD900052BA2A82DB885BBA6B8201200AB0BDE816
:10ADA000F081C8F820D0C0B280F311883846FFF790
:10ADB00049FEE3E7287905082DE9F04190F88C3049
:10ADC000056D012B8AB004466ED015D8C36C4FF0C8
:10ADD000FF321A605A609A60DA60D0F8903005222B
:10ADE000B3F57A7FC0F8A02079D8032380F88C309F
:10ADF00001200AB0BDE8F081023B012BF8D890F8A1
:10AE0000FD30C26C4F4E63F07F031370036DD0F8BA
:10AE1000108003F1010E00F110070FCEEC46ACE8F4
:10AE20000F00E36CCDE9003E0FCEACE80F0096E8D2
:10AE300003008CE80300EFF31180102383F31288E2
:10AE400023691B6A002B6FD0029B6A461BB1D36932
:10AE50001432002BFBD1D8F8203073B1996839B97E
:10AE600093420AD0196829B15B6899680029F7D024
:10AE70001433F3E71F60C3F804D0C0B280F3118825
:10AE80002269136A002BFCD16B885BBAA4F880306E
:10AE9000AB885BBAA4F88230EB8801205BBAA4F8D7
:10AEA00084300AB0BDE8F08190F8FC2090F8FD30C5
:10AEB0009B1A5B100133DBB205EB430235F813300C
:10AEC0005BBAA0F8803053885BBAA0F882309388D0
:10AED0005BBAA0F8843001200AB0BDE8F0810369B4
:10AEE0001A7B52B35B6943B390F848302BB390F8A8
:10AEF000FC30C26C606563F07F03137090F8FC1047
:10AF000090F8FD30026D1048C4F8B4005B1A0733A6
:10AF10000121C4F8AC30E36C84F8B0100A44C4E9F1
:10AF2000293284F88C1063E7C8F820D0C0B280F3CF
:10AF300011883846FFF786FDA2E7022384F88C309B
:10AF400056E700BF287905087585000810B1036829
:10AF500082889A61704700BF10B1036882889A6244
:10AF6000704700BF0348D0F8283113B100F58E7048
:10AF700018477047000000200348D0F84C3113B147
:10AF800000F5A07018477047000000200348D0F873
:10AF9000703113B100F5B2701847704700000020FF
:10AFA0000348D0F8943113B100F5C47018477047C6
:10AFB000000000200348D0F8B83113B100F5D67076
:10AFC00018477047000000200348D0F8DC3113B167
:10AFD00000F5E87018477047000000200348D0F8DB
:10AFE000003213B100F5FA701847704700000020D6
:10AFF0000348D0F8243213B100F5067018477047A3
:10B00000000000200348D0F8483213B100F50F705B
:10B0100018477047000000200348D0F86C3213B185
:10B0200000F5187018477047000000200348D0F85A
:10B03000903213B100F521701847704700000020CE
:10B040000348D0F8B43213B100F52A70184770479E
:10B05000000000200348D0F8D83213B100F5337057
:10B0600018477047000000200348D0F8FC3213B1A5
:10B0700000F53C70184770470000002010B50138FB
:10B080000B4C0C4B00EBC00004EB8004D4F81C010B
:10B0900098420CBF3620382046F0EEFED4F81C2132
:10B0A000D2F8003143F00103C2F8003110BD00BFF7
:10B0B0000000002000640240F8B50138124C00EB9B
:10B0C000C00004EB80041E461048D4F81C318342B3
:10B0D0000CBF3620382015460F4646F0CDFED4F87A
:10B0E0001C01D0F8003143F00103C0F8003194F99D
:10B0F0002D01C4F82871C5F30112A909C4F8306103
:10B10000BDE8F84041F010BE00000020006402409D
:10B11000D3B20D2B2AD84FF0000C10B46346144C58
:10B1200004E00133202B1DD014F803CF6045F8D183
:10B1300094F801C08C45F4D10E4902EB420401EBB6
:10B14000840201F545700C4903EB43030B4400EB0B
:10B15000840093F8523D5DF8044BC2F81C3382F82A
:10B160001433704700205DF8044B7047002070478F
:10B170005079050800000020006C050810B40C4C44
:10B18000002304F54B7C01E0152B0CD003EB4302AC
:10B1900001331CF802108142F6D122445DF8044BC1
:10B1A00092F92E0370474FF0FF305DF8044B704763
:10B1B000D038002030B40023114C124D04E001338C
:10B1C0001C2B1AD054F8085FA842F8D125798D427B
:10B1D000F5D10D480D4902EB420400EBC30001EB31
:10B1E000840390F8B52DC3F81C2301F5457101EBDC
:10B1F000840083F8142330BC7047002030BC7047B3
:10B20000B079050800000140006C0508000000202E
:10B21000F0B110B504460F4894F804E0002300F59F
:10B220004B7C01E0152B11D003EB430201331CF8DA
:10B2300002107145F6D10244617992F92E232068FB
:10B24000D3B20D2B02D8BDE81040B3E7002010BDEB
:10B2500000207047D0380020800AA0F580105328C5
:10B2600006D8044B1B5C0C2B02D8034AD0567047FF
:10B2700000207047006C050858E305080120FEF720
:10B28000BBBA00BF0220FEF7B7BA00BF0420FEF72A
:10B29000B3BA00BF0820FEF7AFBA00BF1020FEF718
:10B2A000ABBA00BF4FF47870FEF7A6BA4FF47C40FB
:10B2B000FEF7A2BA30B1036882881B691A4214BF34
:10B2C00001200020704700BF30B50C4683B0054612
:10B2D00018B3036803F13F4303F57E039B0A104A4A
:10B2E000134493F8900E46F0C7FDA9880091C4F36B
:10B2F0000013C4F341128DF8043028688DF805203E
:10B3000004F003036946C4F381048DF806308DF818
:10B31000074041F0C1FC03B030BD4FF0FF33DEE722
:10B32000006C050800B1CFE7704700BF0E4B70B549
:10B33000D3F89C67002E14DD0C4C002503E0B542C9
:10B3400004F120040DD0237F0135002BF7D0E068F5
:10B350000028F4D0217DFFF7B7FFB54204F12004A7
:10B36000F1D1012070BD00BFD82700209419002022
:10B37000F8B502680446007C1368022181400B4244
:10B3800006D1116808238340194218BF5360F8BDE5
:10B3900004238340656951605360EFF311835022A9
:10B3A00082F312882A6C1168C9070BD5DBB283F3CC
:10B3B000118895F86C3013B195F88560EEB122686C
:10B3C000207CDEE7516889B279B9D5E909708742F6
:10B3D0002AD0AE690644D66021D82E69301A80B2D0
:10B3E0005060A962002185F86C10116841F00101DC
:10B3F000DBB2116083F31188DBE795F87A000CF07B
:10B4000053FFAB6EDA68012166F3C302DA6085F898
:10B4100085100028D3D02821FFF756FFCFE7381A30
:10B4200080B25060AF62DDE7012285F86C20BDE795
:10B4300070B50C4682B016460546002847D0036812
:10B4400003F13F4303F57E039B0A224A134493F81A
:10B45000900E46F011FDAB880093C4F34113C4F382
:10B4600000128DF80530694604F0030328688DF852
:10B470000420C4F381048DF806308DF8074041F0B4
:10B480000BFCAB882A68B3FA83F3C3F11F0303F004
:10B490000701890013F0F80F06FA01F60BD1136AC1
:10B4A0000F2000FA01F123EA01011162136A1E4321
:10B4B000166202B070BD536A0F2000FA01F123EA50
:10B4C00001015162536A1E43566202B070BD4FF0D3
:10B4D000FF33BAE7006C050800B1A9E770472DE912
:10B4E000FF47A04C542303FB00430746D3F8D86121
:10B4F000002E00F02B81D3F8E081B8F1000F04D0CA
:10B5000098F80630002B40F02181542303FB0743B9
:10B51000D3F8E4511DB1AB79002B40F017817B1CAF
:10B52000DBB2B8F1000F04D0152288F8062088F8A5
:10B53000073015B11622AA71EB71307E46F09CFCE3
:10B540002946404648F0D6FB542047433C444046F9
:10B5500094F8EA3194F8E821002B14BF3621162123
:10B56000FFF7BAFF94F8EA3194F8E921002B14BFF1
:10B57000362116212846FFF7AFFF7B4807443C22BF
:10B58000002138464BF0D7FAD4F8D8315D68C4F8BA
:10B59000F051684641F07AFADDED037AB4F8EC81B7
:10B5A0009FED727ADFED725AF8EE677AF0EE083AA4
:10B5B000C7EE274A4FF0000E40F2145407EE908A6F
:10B5C0009FED6C7AF8EEE77A64EEA33A87EE274AAD
:10B5D000DFED697AB0EE007AE4EE877AE4EE875A1E
:10B5E00074EE672A37EEA56AB7EE005AB8F5C87F41
:10B5F0000EF1010C07EE90CAD5BF642332234FF43D
:10B60000967078200344B8EEE77A07EE903A27EE7A
:10B61000247AF8EEE76AD8BF4FF4167986EE873AB7
:10B62000CABF4FF4827921464FF4FA7101EB090346
:10B6300073EE456AFCEEE67A17EE902A07EE909AD2
:10B64000B8EEE73A07EE903A23EE043AF8EEE77ADE
:10B65000C3EE276A36EEE53A72EEE66AC3EE077A83
:10B6600077EEC57AFCEEE77A17EE901AC6EE877A87
:10B6700077EEC57AFCEEE77A17EE903A03F102090D
:10B6800009EB010A07EE90AAF8EE677AF0EE466A37
:10B69000E7EE276AB4EEE64AF1EE10FA5BDC5FFAF9
:10B6A00082F9B9F10F0F58D8323807EE900AF8EE48
:10B6B000E77A77EEE37AC7EE876AFCEEE67A17EE72
:10B6C000900A5FFA80F9B9F10F0F46D81FFA81F995
:10B6D000B9F1FF0F41D81FFA83F9B9F1FF0F3CD838
:10B6E0001205264B49EA0E7402F07F6200041443EF
:10B6F00000F47F00044303EA01210C433846FDF7C0
:10B700004FFD2B686FF300032B602C612B6843F413
:10B7100070632B60AB686FF38A23AB60AB686FF329
:10B720000903AB60AB6843F40043AB6000221146F1
:10B7300096F91A0041F0F8FA002296F9190011461C
:10B7400041F0F2FA2B6843F001032B6004B0BDE82E
:10B75000F087E6464AE7013192E7BCF10F0FF8D1D6
:10B760000024CBE7D0380020C03A0020286B6E4E72
:10B7700000001643002474490000704200FFFF00DF
:10B780002DE9F843B04D05EB0017D7F86C33002BCB
:10B7900000F0C5800446060197F8760346F06CFB7E
:10B7A00097F8763303F01F025B090121013B01FA90
:10B7B00002F2042B0BD8DFE813F0DC000500E200F6
:10B7C000E800EE00A14B596921EA02025A61AB1967
:10B7D000013493F870030CF067FDE4B2804610B1B9
:10B7E00012238371C471AB1993F871030CF05CFDE3
:10B7F000814610B11323C4718371AB1993F872039E
:10B800000CF052FD074610B11423C4718371AC19BA
:10B81000404694F873232621FFF75EFE94F87423C4
:10B8200048462621FFF758FE94F87523384606212E
:10B83000FFF752FED4F86C33854A934200F0C9807A
:10B84000844A934200F0AD80834A934200F0E68040
:10B85000824A934200F0ED80AB19814AD3F86C33F1
:10B86000596841F002015960596841F0010159607D
:10B87000D9696FF3CB21D96192F8BC1300295FD14C
:10B88000186861F3CF301860186861F38E30186063
:10B89000186861F38A201860196892F8C34364F34A
:10B8A0004921196092F8BD03196801285BD06FF334
:10B8B00008211960196860F38201196092F8BE13BB
:10B8C00007292ED858686FF34920586058686FF3DD
:10B8D00008205860186861F3C5001860196892F86C
:10B8E000BF4364F3C7111960196892F8C04364F349
:10B8F000CB211960196892F8C14364F341011960C2
:10B90000196892F8C22362F3000119601A690720CE
:10B9100060F30F021A611A6842F040021A60BDE833
:10B92000F8830A296DD058686FF349205860586829
:10B9300040F480705860186861F3C5001860CDE766
:10B94000012951D0022937D00329A5D1196841F422
:10B9500000411960196841F48041196019686FF35A
:10B960008A21196098E7012CA1D141F480711960F6
:10B97000A0E7364B196921EA02021A6127E7334B27
:10B98000996921EA02029A6121E7304B596A21EA5A
:10B9900002025A621BE72D4B196A21EA02021A625F
:10B9A00015E7304841F0E2F82F4AD2F8203823F466
:10B9B0008043C2F820384FE7196841F4004119600C
:10B9C00019686FF38E31196019686FF38A21196055
:10B9D00062E7264841F0CAF8234AD2F8243823F413
:10B9E0008053C2F8243837E719686FF3CF311960F4
:10B9F00019686FF38E311960196841F4806119601C
:10BA00004AE7596841F40071596059686FF3082199
:10BA1000596019686FF3C50119605FE7144841F078
:10BA2000A5F8114AD2F8203823F40043C2F8203890
:10BA300012E7104841F09AF80B4AD2F8243823F460
:10BA40000053C2F8243807E7D038002000380240FD
:10BA50000030014000380040003C0040003401400C
:10BA6000000000200E002000003002400C002400E6
:10BA70000F0020000D0024002DE9F04F8DB0A94BE0
:10BA80000793A94BDFF8C0820024A3F69865A74F5F
:10BA9000DFF894A2BB0AA3F58013532B4FF00006E6
:10BAA0004BD8EB5C0C2B48D818F90390A04B93F8BB
:10BAB000BE33012B40F00781B9F1010F33D14FF0B4
:10BAC000010B1FFA8BF1484610F0B6FD10F042FE54
:10BAD000037813B1542B40F01F810BF1010BBBF124
:10BAE000050FEED1ACB34FF0000C8E4A00210BE0F5
:10BAF000EB5C0C2B0FD818F903304B450ED00131FD
:10BB0000A14202F1AC0221DA906803689B0AA3F516
:10BB10008013532BECD900234B45F0D143799AF88D
:10BB200005009842EBD10136082E45D05AF81C7F0B
:10BB3000BB0AA3F58013532BB3D97D4B93F8BE33C7
:10BB4000013B012BEFD94FF00009B8E7BCF1000F22
:10BB5000E9D1DAF80800774B002205E001320E2A1D
:10BB600003F10C0300F0CA8359688842F6D152B23F
:10BB70009AF805103846FFF71DFB6F4A406800230E
:10BB80005168884203F1010300F09A800E2B02F104
:10BB90002402F5D14FF0FF33684A03EBC30302EBF5
:10BBA000830393F83431002BBDD15F4BC6EBC6063F
:10BBB00003EB8606079B9E60079B0134AC33042C85
:10BBC00007937FF464AFDFF8849109F204434FF0E8
:10BBD000010B98465A4BD3F89C270BF1FF339A423E
:10BBE0006BDDD9F80C50002D00F084832968AE88F5
:10BBF00001F13F41B6FA86F601F57E01C6F11F0656
:10BC0000890A504B1F68002F40F3A480043300249E
:10BC100005E00134BC4203F1AC0300F099801A68DE
:10BC20008A42F6D13F4AC9F80460AC2303FB0424DE
:10BC3000C9F818405FFA8BF315B1EB710323AB71B0
:10BC4000404B616C93F87806E36B720003279740D2
:10BC50003B43E363012303FA02F20A4362640028D0
:10BC600039D0A26C03FA06F63243A2646DB1304BB0
:10BC7000AA8893F814142B68490141F0050101F0DA
:10BC8000E5019A612846FFF71FFB606FB1B2012200
:10BC9000FCF7B6F920460BF1010BFCF78FFA0123F4
:10BCA000BBF1090F89F81C3089F81D3088F8113074
:10BCB00009F1200908F118088CD10DB0BDE8F08F0A
:10BCC000DBB2013B68E7022B7FF4F9AEB9F1080F54
:10BCD0003FF4F5AE27E7A26C06F1100103FA01F17B
:10BCE0000A43A264002D00F08B8003FA06F6104B85
:10BCF000AA8893F814142B68490141F00501120435
:10BD000001F0E5019A612846FFF7DEFA606FB1B2F3
:10BD10000022FCF775F9BDE74FF0010C002C7FF411
:10BD2000E4AE00E7E4160020987A0508000401401C
:10BD3000D0380020140300201C0100200000002047
:10BD4000D8270020E016002058E3050894190020A9
:10BD5000032C58DC8B4AAC2303FB0723D86800284C
:10BD600000F0C1825422596083F8AC200131854A29
:10BD700083F8AD107B1C1360834B99F8102093F867
:10BD8000D53308928168814C00229C4605E001323F
:10BD90000E2A04F10C0400F0B18263689942F6D1D6
:10BDA00041790068CDF81CC052B2FFF703FA754B19
:10BDB000DFF800A2D0E90141AC2202FB0732079B69
:10BDC000C2E90541514600224868844202F101025D
:10BDD0001ED00E2A01F12401F6D16D4B93F81021EB
:10BDE000002A00F0288268486A496B4A6B4BC0F809
:10BDF000FC13C0F8F423C0F804340DB0BDE8F08F94
:10BE000003FA06F682E7604A032382F8D433EAE7AE
:10BE1000D2B25F49013A02EBC20201EB8202AC24CA
:10BE2000584992F83401099007FB04F401EB040C23
:10BE30000146BCF8AC000029D5D1A2F8340162104B
:10BE400002EBA402C2EBC21202EB8232920102EBBD
:10BE5000A4025349520002EBA40202EB420E0C442E
:10BE600050498C200EEB0E1E00FB02F201EB8E0EF1
:10BE700001F54C7101EB42020A922A68CCF80820C5
:10BE80000A9ACCF898203322DCF80C10CCF87C20ED
:10BE90003F4ACCF89C00062B086812680791CCF842
:10BEA00078E000F0F581072BDFF80CC13E4B3F49ED
:10BEB00008BF19463E4B08BF6346B2FBF1F101F1E2
:10BEC000FF3C3049B2FBF3F3AC2202FB0712013B0B
:10BED0009BB2A2F86030A2F880C0C36200238362E4
:10BEE000426942F001024261026863F30922026082
:10BEF000026863F306120260036843F08003036084
:10BF0000036843F080030360079B597901394900B6
:10BF1000C9B207290BD8DFE811F0B8010A00B50152
:10BF20000A00B2010A00AF0108000A234367036850
:10BF30006FF3000303600022012303930193049233
:10BF400002920092062247F06FFB01231A46079BDC
:10BF5000597918680139914001F0FE0140F02AFF3B
:10BF6000079A53791268013B5B00DBB2072B29D893
:10BF7000DFE813F07D012800780128007301280014
:10BF80006E012400E0160020D038002014030020A9
:10BF900000000020FD6A0108F96A0108056B01082C
:10BFA000E4160020E83C00201055220044950800CB
:10BFB000D0DD06001C01002040771B00136F43F00A
:10BFC00008031367079B1879002840F077811368EE
:10BFD00043F001031360B04AAC2303FB0723596904
:10BFE0000023DAF80420914203F1010300F01E81DE
:10BFF0000E2B0AF1240AF4D14FF0FF3AA74A0AEBBC
:10C00000CA0302EB8303A64AD3F81C0107939042AC
:10C010000CBF3620382045F02FFF079B9E4AD3F8EF
:10C020001C11A048AC2303FB0723D1F8002142F0E8
:10C030000102C1F80021DA684FEACA030793537975
:10C04000D2F800C0944A013BDBB2032B9BBF964958
:10C0500001EB43030021B3F8781FAC2303FB072354
:10C060004FF0000E1982734606E0944500F04081BF
:10C070000133042B00F0458150F83320002AF4D11D
:10C080008A4A9E461346D2F8A0270132C3F8A02759
:10C0900003EBCE024FEACE03C2F8A4C703440998CB
:10C0A0009A8811439980902281492346FFF704F82A
:10C0B000079B7A4A7849534402EB8303AC2202FB84
:10C0C0000717D3F83C31B9691A6861F306021A60A0
:10C0D0007B691A6842F002021A604FF4407C4FF408
:10C0E000807A1022A4F870C0A4F86CA0A4F868208C
:10C0F000B7F87CE0A4F86AE0B968022201F1180000
:10C1000084F86E20206609901031B86F84F86F2093
:10C1100007911968606621F4804121F0100109043B
:10C12000090C1960196841F010011960196841F48F
:10C1300040511960196862F38B211960196862F324
:10C14000092119601A6842F080021A601A686FF3B8
:10C1500086121A601A686FF345121A605A686EF3F5
:10C160000F025A60099A9A60D8601A68E2615A68A8
:10C1700022629A6862620021DA68A262A4F88CA046
:10C18000A4F890C0A4F88810079AB7F89C00C4F8E7
:10C190008020012284F88E20A4F88A00D7F898C065
:10C1A00084F88F201F68C4F884C027F4804727F0E4
:10C1B00010073F043F0C1F601F681F601F6847F493
:10C1C00040571F601F6862F38B271F601F6862F370
:10C1D00009271F601A6842F080021A601A6861F32A
:10C1E00086121A601A6861F345121A605A6860F381
:10C1F0000F025A60079A9A60C3F80CC01A68E2628C
:10C200005A6822639A686263DA68A2631A6842F025
:10C2100002021A60089B89F81030C9F80460C9F856
:10C220000C50C9F818405FFA8BF306E5DBB20993AE
:10C2300003F1FF3AE2E61849AC2202FB071292F83A
:10C24000AD1092F8AC2083F8102183F81111CAE5E3
:10C25000D36943F40063D361B4E6D36943F00803C0
:10C26000D361AFE6936943F400639361AAE69369EF
:10C2700043F008039361A5E60A23036457E60A2303
:10C28000C36354E60A23836351E60A2343634EE6FD
:10C290000849094B11E600BFE0160020000000200D
:10C2A000006402407C2F0020006C0508D827002085
:10C2B000E1900008882A1100A0BB0D000B920BF042
:10C2C000F3FF0B9A0A9048B1079B0A21DA79FFF72E
:10C2D000AFF80A9B5422DA80079B1A68536C43F428
:10C2E0000043536473E6084A022382F8D4337AE5A4
:10C2F000DB00D3E64FF0FF36314682E400235B6873
:10C30000FFDE00239B88FFDED0380020F8B590F8D0
:10C310007A301C09013C072C0FD81A4E06EB440258
:10C320000546B2F8800F03F00F0340FA03F2D2077C
:10C3300003D595F88570012F01D00120F8BD07FACB
:10C3400003F3013B1840344448F0DAFE94F8902F90
:10C350000D49104451F8302001EBC00110698B8861
:10C360001840EBD0002395F87B2085F885300846EF
:10C370000A21FFF75DF8AA6ED36843F00803D36083
:10C380003846F8BD006C0508EC370020094AD2F8A1
:10C39000A83BD2F8AC2B002140F22A4058605162F1
:10C3A000116841F0010111601A6842F001021A603F
:10C3B000704700BFD0380020002800F0AB812DE985
:10C3C000F04F002287B02F21064610F019FA0546DB
:10C3D000E0B1654FD0F80090C7F8AC9BFEF718FFAE
:10C3E000804698B14068C7F8A80B78B15F4C00232D
:10C3F00022465168884202F1240203F101030FD062
:10C400000E2BF6D15A4B93F8100118B1002007B04B
:10C41000BDE8F08F2F2283F8102183F81101F6E791
:10C42000DBB2DFF84CA1013B03EBC3030AEB830350
:10C4300093F834B1BBF1000FE8D130462F26A3F8B2
:10C4400034610BF031FF0346C7F8B40B20B1DE8036
:10C45000EA790A21FEF7ECFF464A4749002301E04A
:10C4600051F83320914500F05F8101330F2BF7D154
:10C47000002045F001FDD7F8AC0B404A03686FF38C
:10C4800000030360DAF800309342C0F0458103F105
:10C49000B7723B4902F55852A1FB0221890D0139BF
:10C4A00089B24A1C0139B3FBF2F3364A364E1B0AF5
:10C4B000A2FB03231A09A6FB026252081B09A7F874
:10C4C000B22B013B5200C362A7F8B02B81624369D3
:10C4D00043F00103436103686FF3092303600368BA
:10C4E0006FF306130360AA7912F0020600F01781B9
:10C4F00002F00106002213464FF0010C6979013960
:10C500004900C9B207290DD8DFE811F041010C003C
:10C510003C010C0037010C00320108004FF0000E06
:10C52000C0F874E0CDE90126002203930092CDF813
:10C5300010C0062247F078F8D7F8AC0B036843F038
:10C54000800303606B79013BDBB25A00D1B207294B
:10C5500020D8DFE811F008011F0003011F00FE00D2
:10C560001F00F9001B0000BFD03800201C01002074
:10C5700000000020000001402C780508006CDC025F
:10C58000819F5E16598B4F01ABAAAAAA066F46F08F
:10C5900008060667032B9CBF844BD218C36894BF60
:10C5A000B2F8782F00221343C360AB799B0748BFD2
:10C5B00001314FF0010248BFC9B240F0FBFBD7F890
:10C5C000A80B224600235168884202F1240200F0A1
:10C5D000B78001330E2BF6D14FF0FF3606EBC606BF
:10C5E0000AEB8606724BD6F81C0198420CBF362027
:10C5F000382045F041FCD6F81C11D1F8003143F049
:10C600000103C1F80031D7F8A86B22460023516816
:10C610008E4202F1240203F1010300F08E800E2B02
:10C62000F5D16449584600236022FEF745FD336882
:10C630006FF300033360304640F0A6FA6B79D7F809
:10C64000AC5B012B00F0A880022B00F0A880032B2C
:10C6500000F0A880042B16BF05EB830305F1400111
:10C6600003F13001D7F8A83B1A684BF6EF7002408F
:10C670001A601A6842F010021A601A68012060F30A
:10C680000D321A601A68022060F38B221A601A6851
:10C6900060F309221A601A6842F080021A601A6870
:10C6A0006FF386121A601A686FF345121A605A689F
:10C6B00040F22A4060F30F025A603F4A9960DA6004
:10C6C000002261688B4204F1240402F1010231D09E
:10C6D0000E2AF6D14FF0FF3202EBC2020AEB820AB9
:10C6E000D8F80800DAF83C21116860F306011160FF
:10C6F0001A6842F002021A601A68012002431A60A6
:10C700006B6C43F400436B642B6803432B6007B0EE
:10C71000BDE8F08F002070474FF0FF31C5E602F012
:10C720000102B4460123E9E6204A02EBC30393F871
:10C73000300C9EE6D2B2013ACEE75FFA83FB70E797
:10C740005E1CF6B2013E49E7C66946F40066C66162
:10C7500020E7C66946F00806C6611BE7866946F40D
:10C760000066866116E7866946F00806866111E76D
:10C770004FF0000EC0F840E0D4E64FF0000EC0F8D5
:10C780003CE0CFE64FF0000EC0F838E0CAE64FF0CC
:10C79000000EC0F834E0C5E605F1340162E705F1AA
:10C7A00038015FE705F13C015CE700BF006C05085C
:10C7B000006402400D820008B4D4002030B40B4A5B
:10C7C0000B4B82B0CA25532402EB800000225D622D
:10C7D0005C62019201905D625C620198FF220160DF
:10C7E0005A625A6202B030BC704700BF5028004005
:10C7F00000280040F0B5013B0E469DB2644B346802
:10C800001B68B3FBF2F2013AE562A262636987B08A
:10C8100043F00103BDF830109DF8342063612368B4
:10C820006FF30923236023686FF306132360757980
:10C83000B37907460AB183F0010313F0020010D068
:10C84000002203F001004FF0010C1346013D6D0082
:10C85000EDB2072D0AD8DFE805F01D094A09800965
:10C860005C6E03F0010284460123EFE7CDE901206D
:10C87000002200922946CDF810C0039306222046DC
:10C88000023D46F0D1FE052D14D8DFE805F03D133A
:10C8900073134F6161630021CDE902030192CDF86A
:10C8A00010C000910622204646F0BEFEA36943F068
:10C8B0000803A3613268536C43F400435364136864
:10C8C00043F0010313607379012B58D0022B59D028
:10C8D000032B5AD0042B16BF02EB830302F1400353
:10C8E00030330021C7E90032196007B0F0BDA16301
:10C8F00001920022CDE902030092CDF810C0062279
:10C900000221204646F090FEA36943F40063A36130
:10C91000D0E721640192002200920622CDE90203B1
:10C92000CDF810C01146204646F07EFEE36943F480
:10C930000063E361BEE7616701920022CDE9020373
:10C940000092CDF810C006220721204646F06CFE6A
:10C95000236F43F008032367ACE7E16301920022F1
:10C96000CDE902030092CDF810C006220421204632
:10C9700046F05AFEE36943F00803E3619AE702F1E7
:10C980003403AEE702F13803ABE702F13C03A8E75A
:10C99000000000202DE9F04FD0F80890046C99F8C1
:10C9A00005A099F80680D9F80060054687B02046B2
:10C9B0000AF1FF3B40F0E8F85FFA8BF35F000022DA
:10C9C000FFB208F0020885F82C20072F0DD8DFE809
:10C9D00017F0D2000C00DB000C00E4000C00ED00AE
:10C9E0000800326F6FF3C3023267B8F1000F15D140
:10C9F000AAF10203022B05D84FEA4A08A8F102085F
:10CA00005FFA88F800224146304640F0D3F9BBF186
:10CA1000030F11D8DFE80BF096918C0C022B00F27B
:10CA200084804FEA4A0808F1FF385FFA88F8E9E79E
:10CA3000F3696FF30923F36195F83B30049395F89C
:10CA40003A30039395F83930029395F838300193D2
:10CA500095F83730009395F8363095F835203946FB
:10CA6000304646F0E1FD99F805309A1E022A50D969
:10CA70000023736341460122304640F09BF9072FA3
:10CA800009D8DFE807F073086E0869086404336F9B
:10CA900043F00803336723684BF6EF7110220B4015
:10CAA0002A842360236813432360236895F8292090
:10CAB00062F30D332360236895F8272062F38B23FC
:10CAC0002360236895F8262062F3092323602368F6
:10CAD00095F8252062F3C7132360236895F8242076
:10CAE00062F386132360236895F8282062F34513C8
:10CAF000236063686A8C62F30F036360D5E90623E1
:10CB0000A260E360236843F00203236007B0BDE83E
:10CB1000F08F5B00023BDBB2042B53D0062B4ED0D0
:10CB2000022BA7D10023B363A4E74FF0000869E705
:10CB3000F3696FF30103F3617EE7B3696FF30923D0
:10CB4000B36179E7B3696FF30103B36174E7F36924
:10CB500043F40063F3619EE7F36943F00803F36174
:10CB600099E7B36943F40063B36194E7B36943F0B1
:10CB70000803B3618FE7B2696FF3C302B261B8F122
:10CB8000000F3FF435AF49E7B2696FF3CB22B261D2
:10CB9000B8F1000F3FF42CAF40E7F2696FF3C30226
:10CBA000F261B8F1000F3FF423AF37E7F2696FF39A
:10CBB000CB22F261B8F1000F3FF41AAF2EE7002349
:10CBC000336457E70023F36354E700BF2DE9F04FC8
:10CBD000B44B93F8784685B024B90124204605B0BB
:10CBE000BDE8F08FB04ED6F8A0520DF049F9AF4B2A
:10CBF00093F8EC3B002B00F04D81AD4BAD4FA3FB08
:10CC000005235B09A7FB0327FF0807EB8707A3EBB7
:10CC10004707D6F81038C31A0093A24B03F56D7B73
:10CC2000FBB206F56B78019306F28C6308EB87077D
:10CC30005D4600269946CDF80CB011E02846FFF776
:10CC4000A9FE9A4B93F8EC4B0136A64208F15C081A
:10CC500007F15C0709F1140905F14C0580F2C18068
:10CC6000009A002A03DB2B6B934200F3FD808D4B6F
:10CC70004C2202FB063393F8E033002BDED0AB6886
:10CC8000A9891A682B6C5B681FFA83FED368CEF102
:10CC9000160E23EA0103BEF1070FD360CED9824AF4
:10CCA000D2F894360133C2F89436AB6C02939C46AA
:10CCB000002201215CF8044B92468B461BE0DCF815
:10CCC0000000BAF1140FA0EB04031DDC13F10804FB
:10CCD00048BF03F1170423110AEB241A0446581E17
:10CCE000013102FA03F38E450BFA00F242EA030225
:10CCF0000CF1040C08D37145E1D3CAF11503DCF83B
:10CD000000404FF0150AEAE7BAF1150F5ED16A4804
:10CD1000C2F38423C2F3441100EB830300EB8101CF
:10CD2000D3F8983FD1F8981F1B0243EA011302F091
:10CD30001F0100EB8101C2F3C43200EB8202D1F883
:10CD4000981FD2F8982F0B4343EA023383EA132249
:10CD500082EA121202F00F020F2A37D1C3F30F1327
:10CD60004FF6FF72934231D0B3F5606F00F08180CF
:10CD7000A9F80C3098F858200198824210D0B96870
:10CD8000D8F80020521AC8F80020396BD8F80420CF
:10CD9000521AC8F804200022BA603A6388F8580092
:10CDA000D8F800200132C8F80020BA680132BA6011
:10CDB0004FF6FF7293427FF441AFD8F8043001334D
:10CDC000C8F804303B6B01333B6337E7364AD2F88F
:10CDD00090360133C2F89036002E3CD04FF6FF73E8
:10CDE000C8E73149DDF80CB00122002381F8902713
:10CDF000C1F81038002C3FF4F0AE04EBC40304EB90
:10CE000043040BEB840403250CE0022E03F1FF33F3
:10CE10001FD9002101220BF14C0B3FF0CBFF5C45E9
:10CE20003FF4DBAEDBF808301868426865F30612A1
:10CE300042609BF810105B7911F0020103F1FF369C
:10CE4000A3F102024FEA4303DFD1022AA3F1020356
:10CE5000E0D8D9B2DEE702F5E7600299582249F03E
:10CE600007FE4FF6FF7385E70024204605B0BDE8B6
:10CE7000F08F0C4991F8152602EB420201EBC20239
:10CE8000324492F825260D2A7FF472AF802289F869
:10CE90001E206FE70449012281F89027C1F810385D
:10CEA0009CE600BFE0160020D8270020D0380020E4
:10CEB0001F85EB51CDCCCCCC006C0508F0B50446F9
:10CEC00085B0A56EEB686FF34D33EB60684666790D
:10CED000A7683FF0DBFD934B9D4206F0020605D0AC
:10CEE00003F580639D4201D0039B00E0029B03EBAE
:10CEF00083035A008C4BB2FBF7F2A3FB0213DB084F
:10CF000003EB8301A2EB4102042A88BF0133AA6824
:10CF10009BB263F30F02AA60EB686FF31C73EB60C4
:10CF2000EB686FF30C33EB602B6966F30D332B6109
:10CF30006679A26E7107C6F3800300F18880D1681C
:10CF400063F34921D160D16863F38A21D1605369C9
:10CF50006FF30823536153696FF3492353612179B8
:10CF600011F0010740F0C48011F0020540F0BB80D1
:10CF70006E4B03F1200053F8041F8C4254D09842AA
:10CF8000F9D116F008035DD0536943F008035361EB
:10CF9000D36843F40053D360002F3DD0E06B0028EA
:10CFA00000F0AB806569666EA7893FF0EDFDE36B2D
:10CFB0001A684BF6EF710A401A601A681A601A680C
:10CFC000012161F30D321A601A686FF38B221A6027
:10CFD0001A686FF309221A601A6842F080021A6018
:10CFE0001A686FF386121A601A6842F020021A60FB
:10CFF0005A6867F30F025A609E60DD601A680A4340
:10D000001A60A16E4A6942F040024A615B68217968
:10D010009BB2E36501F0020515BBA26ED36843F431
:10D020000053D36005B0F0BD002CAAD094F8843032
:10D03000002BA6D0A16E0B6943F400430B6116F0E0
:10D040000803A1D1516963F3C3015161A0E7D3681B
:10D050006FF34923D360D36843F48063D36076E7EA
:10D06000206C002855D0266EA569278A3FF08CFDDC
:10D07000236C1A684BF6EF710A401A601A6842F086
:10D0800010021A601A68012161F30D321A601A68E1
:10D090006FF38B221A601A686FF309221A601A68FC
:10D0A00042F080021A601A686FF386121A601A68DA
:10D0B0006FF345121A605A6867F30F025A609E6058
:10D0C000DD601968A26E41F002010020196058600D
:10D0D000536943F0800302F10C0153610B6843F084
:10D0E00040030B609AE7D36843F00803D3603FE73F
:10D0F000D36843F00403D36036E76FF02003136076
:10D10000D36843F02003D360D36843F01003D360A7
:10D1100082E7A26ED36843F0800302F10C01D36072
:10D12000DCE700BF00100140CDCCCCCCC0440020D7
:10D130002DE9F843434C04EB8004D4F8F44B002C65
:10D140003DD0656FA1601F463F4B23606B68A366AF
:10D15000AB6B63616B6BA361EB8FE360AB8F2361A0
:10D160003A4B23670646204690460CF019F995F88D
:10D170002C0000285DD194F87A000BF095F802227B
:10D18000390794F8789084F885201BD588B317F078
:10D19000510F0CBF0122002217F0410F14BF402194
:10D1A000202141EA021101360B22C671827194F8E6
:10D1B0007B2041F00601FEF73BF9E36B6BB32046A1
:10D1C000BDE8F88318F0020F13D090B10B228271E2
:10D1D00017F0410706F10102C2712DD1A36EDA6882
:10D1E000012167F3C302DA6084F885102821FEF775
:10D1F0006BF818F0010FE0D048460BF055F8002806
:10D20000DBD00C220136C671827194F879200A2194
:10D21000FEF70EF9E36B002BD1D195F8301095F99C
:10D220002E00C1F3011289093FF07EFD2046BDE8C2
:10D23000F88344F021FE9EE794F87B200A21FEF754
:10D24000F7F8D6E7D0380020187C05080DC3000891
:10D250002DE9F047884600294AD04618DFF8989013
:10D26000DFF898A0451E013E8024EFF3118184F37E
:10D270001288D9F89832D9F89C02D9F89822D9F8AE
:10D280009CC2C9B281F31188624512E001200EF000
:10D2900003FFEFF3118184F31288D9F89832D9F89B
:10D2A0009C02D9F89822D9F89C72C9B281F31188EE
:10D2B000BA428CBF002201221B1A03EBC223012BAE
:10D2C000E4D0EFF3118284F31288D9F89C3215F878
:10D2D000011F5344D2B283F8141CD9F89C32013395
:10D2E000C3F30A03C9F89C3282F31188B542BCD15A
:10D2F0004046BDE8F08700BFD8270020D038002086
:10D30000F8B50D4B93F89C3C032B00D0F8BD0B4EA9
:10D310000D46D6F8A072144609E0FFF799FFD6F83B
:10D32000A032DB1B322BA4EB00040544EED8002C0A
:10D3300021462846F1DCF8BDE0160020D827002061
:10D34000344BD3F8BC39596A91F85230012B56D17D
:10D3500070B5314C314AD4F81C0360BBD2F8980246
:10D36000D2F89C32984221D0D2F89802D2F89C325E
:10D37000984249D8D2F89C32D2F898021B1AD2F8B7
:10D38000982291F8520088B1B3F5007F28BF4FF47E
:10D3900000731D46002381F85230214921480A4478
:10D3A000ABB281213FF084FEC4F81C531E4B6FF0DA
:10D3B00001021A6170BDD2F8985200F03F03284470
:10D3C000C2F89802D2F89802B0F5006F04BF0020AE
:10D3D000C2F898020020C4F81C03002BBED1D2F87A
:10D3E000982291F852000028E4D00D4881F852307C
:10D3F0000244BDE870400B4881213FF059BE0A4B02
:10D400006FF001021A617047D2F89832C3F50063D9
:10D41000B5E700BFE0160020C8490020D82700204B
:10D42000E444002098200020004C014043F034BB2D
:10D43000344B292270B523F8862C23F87E2CFCF778
:10D4400053FA314A314ED2F83438314C43F080032C
:10D45000C2F83438FAF7E4FF44F076FB40F0FCFE03
:10D460004FF0A0402B49826B01F5805342F400122B
:10D470008263C3F87C634FF401660122A3F87A63E8
:10D480004FF481760025C1F8B40983F8782383F836
:10D49000852304F57B7104F57172A3F8806383F82A
:10D4A000835345F0D1FC23681B4A1C4C1C4EA2FB45
:10D4B00003239B09013B0422E262A3626369194AC8
:10D4C00043F001036361236865F309232360236844
:10D4D000C6F8202365F306132360236843F0800316
:10D4E0002360E36843F00103E36069202A460221D8
:10D4F0003FF01AFC236843F00103236006F54870EF
:10D5000070BD00BFD0380020003002404000400114
:10D5100000000020E0160020D34D6210004C0140B6
:10D52000C8490020487C0508BFF34F8F0549064BCA
:10D53000CA6802F4E0621343CB60BFF34F8F00BFB1
:10D54000FDE700BF00ED00E00400FA0508B500218A
:10D550000320FFF733F972B6FFF7E6FF08B5184C62
:10D56000D4F8742394F87A034AB11168938809694E
:10D570000B40F8B9003B18BF0123002BF4D1142055
:10D580000EF08AFD00BFD4F8743363B11A689B882B
:10D59000116994F87A230B4042B9003B18BF01236C
:10D5A0000BB1FFF7D3FFFBF741F8EBE7B3FA83F3D7
:10D5B0005B09F5E7B3FA83F35B09002BD4D1DEE70F
:10D5C000C849002008B572B6FFF7AEFFF0B5AC4B06
:10D5D000B3F5C07F85B000F08D8100F21381B3F503
:10D5E000807F00F03481B3F5A07F40F006810324F2
:10D5F000A44B1B8A03F00703A34240F07D81A2489D
:10D600003FF0B4FAA149A24B0A68A24842F48072E2
:10D610000A60FF24CA2153225C6259625A62D0F820
:10D620007438DB0000F1F9809B4A994B9B4FCA2567
:10D6300053240020FF215D625C62029002925D62D1
:10D640005C62029E0432BA42306059625962F2D181
:10D6500093490020FFF7B2F8924B00210391039306
:10D66000039B1B680093009B012B00F0E68086481B
:10D670003FF07CFA854A8C4B1069012161F302006E
:10D6800010611A6E61F301021A663FF0D5F98749FD
:10D69000804A0B6843F480330B60D2F800389F0354
:10D6A00007D44FF44053D2F800188E0301D4013B45
:10D6B000F9D1D2F800389D03EFD57C49754A0B6843
:10D6C00043F001030B60D2F800389C07FBD5774B81
:10D6D00070495A6842F480025A605A68482464F3D8
:10D6E0008E125A605A68012060F303025A605A6829
:10D6F00060F312425A601A6842F080721A60D1F8E0
:10D7000000389801FBD5694B9A686FF307129A604D
:10D710009A68042161F34F329A609A6861F38C220F
:10D720009A60D3F8A42042F03002C3F8A4209A688B
:10D73000022060F301029A609A68C2F38102022A11
:10D74000FAD1D3F8A4206FF30512C3F8A420D3F8BC
:10D75000A4200B2161F30F32C3F8A420D3F8A0203A
:10D760006FF34D32C3F8A0209A6812F00C0FC2F389
:10D77000810100F0B18002296BD04D4C4D4B2360EC
:10D780004A4A4D49906823684C4DC0F30310014448
:10D7900011F8801CCB402360EB684FF6FF010B4073
:10D7A00043F0052343F47A03EB603A49444B506F4E
:10D7B000AB60D1F83438434823F00043C1F8343823
:10D7C000536F43F0807353673FF0D0F90CF00EFBBA
:10D7D00023683D4AA2FB03239B09013BB3F1807FF1
:10D7E00009D24FF0E022F02053610021072385F891
:10D7F00023009161136105B0F0BD802B14BF052497
:10D800000624F5E6B3F5E07F05D0B3F5007F14BF3D
:10D8100005240024ECE60124EAE62C4B00220192C8
:10D820000193019A03F11973126803F59E3303F211
:10D83000E1139A427FF4F8AE0EE70320FEF7BEFF35
:10D84000234B1A6882F308885B689847FEE7042434
:10D85000CEE65A685A6859685868154C154DC2F397
:10D860008813C0F302401B4A125C01F00F0105FB54
:10D8700003F312FB01F2B3FBF2F3236080E700BF76
:10D88000C000000000C0FF1F1C00400000700040EE
:10D890000028004000300240542800406C2800401E
:10D8A000316665425C280040003C0240003802407E
:10D8B0000000002000127A00F87C050800ED00E06E
:10D8C000000000081F003000D34D621050280040B7
:10D8D0000000FF1F50E30508D3F8A0200D4C5204B0
:10D8E0007FF54CAFD3F8A030DB047FF547AF0A4B90
:10D8F000236045E702247BE6084B0949094A596041
:10D900005A6059645A6445F023FF204645F0FEFEF4
:10D91000FFF758FE00000020006CDC02003C0240D3
:10D9200023016745AB89EFCD01490248FBF782BF70
:10D93000581E00200000014002494FF08040FBF7D4
:10D9400079BF00BF841E002001490248FBF772BF67
:10D95000B01E00200004004001490248FBF76ABFE6
:10D96000DC1E00200008004001490248FBF762BFAE
:10D97000081F0020000C0040F8B5CB7813B9002533
:10D980002846F8BD00F110070C460646897838464F
:10D990000AF038F905460028F1D0E0780AF084FC56
:10D9A000B06123780133DBB210B1C37122238371DC
:10D9B0000521FDF7B7FCB069FDF7C8FA0C4AD2F8AB
:10D9C000A032632BFBD90B480AF0ECF8B082384642
:10D9D0003CF01EFC074620B9E0780AF0C5FC3D4645
:10D9E000CEE7306986F8887046F0DCF9C8E700BFFA
:10D9F000D827002040420F00264A92F8C4377BB354
:10DA0000D2F8C817884235D0012B29D0D2F8D017C8
:10DA1000814233D0022B23D0D2F8D81788422FD09E
:10DA2000032B1DD0D2F8E01788422BD0042B17D03F
:10DA3000D2F8E817884227D0052B11D0D2F8F0177A
:10DA4000884223D0062B0BD0D2F8F81788421FD07B
:10DA5000072B05D0D2F80018814208BF07230AD04F
:10DA600002EBC30103F1010CC1F8C80782F8C4C777
:10DA7000184670470023DBB2184670470123FAE7C7
:10DA80000223F8E70323F6E70423F4E70523F2E78C
:10DA90000623F0E7D827002038B5384B4C2202FB8C
:10DAA000003292F8C32302B938BD93F814C693F834
:10DAB000152694450ED002EB420403EBC40494F8FF
:10DAC00018E60EF1FF35012D4FEA420446D9BEF1AA
:10DAD000030F3ED04FF04C0C0CFB003CACF8B413E1
:10DAE000EFF31181902282F31288BCF8B4439CF8C2
:10DAF000B62342EA44020024C9B292B28CF8B6437B
:10DB000081F31188110A93F8784681EA1211514085
:10DB100004B1C9434C2404FB00341201184BD4F85F
:10DB2000FC03D3F87C3301F00F0192B20A430121C8
:10DB30009847D4F8F813B4F8C0C3CA88D4F8F433BB
:10DB400042EA0C02CA8058601A6842F001021A6068
:10DB500038BD551C05F003056545BBD0224403EBD9
:10DB6000C202024492F825160029B3D04C2202FBCF
:10DB70000032012482F8B643ACE700BFE016002073
:10DB8000C849002030B4037F083300EB43035B88AF
:10DB9000047F9BB214B98469022C51D0FF2B3AD870
:10DBA0000382037F012B16D08369032B26D0836960
:10DBB000022B23D0038A0468244D6068DBB242EA5A
:10DBC000034242EA010300EA0502134343F00073F3
:10DBD000636030BC70478369022BE5D1038A046817
:10DBE0001A4D6068DBB242EA034242EA010300EAEE
:10DBF00005010B4343F080736360EAE704680A435E
:10DC0000018A636811480340C9B2134343EA0143E0
:10DC1000636030BC7047FF230382B0F810C0056812
:10DC20005FFA8CF06C6842EA0042084842EA01035D
:10DC300004EA00010B4343F080736B6030BC704713
:10DC4000448A838A23449BB2A8E700BF009800FC63
:10DC5000032108B505460846FEF7B0FD72B6104B25
:10DC6000D3E9E02352EA03010AD10024214604202B
:10DC7000FEF7A4FD21460520FEF7A0FDFFF754FCAA
:10DC80000848D0F8A04229B24EF6602000FB01F10E
:10DC9000A41843F100030C1943EBE171E7E700BF5F
:10DCA000C8490020D82700200548D0F8083323B100
:10DCB000DB6A13B100F5427018470248704700BF95
:10DCC000D8270020887C050838B5184CD4F888334C
:10DCD0001B8843B9164D002384F8943385F800332C
:10DCE000C5F8FC3238BDD4F88C23002AF2DD012AB5
:10DCF00009D0D4F8903359880D4DA4F89613012318
:10DD000084F89833E7E7D4F890138A884988013279
:10DD1000521A9A42F0D1064DD5F8083300221B69F9
:10DD2000C5F8342305F542709847D4E7C849002068
:10DD3000D82700200748D0F804331BB1064B93F8CE
:10DD400098330BB100207047D0F8083300F54270CB
:10DD50005B681847D8270020C849002030B4154A0E
:10DD6000154D92F8003305F567742344036095F868
:10DD70009433446092F80003834292F8000312D86F
:10DD8000834204D3002030BCC1E90000704792F800
:10DD90000023002BC2F180020CBF0120022030BC06
:10DDA000C1E9002370471B1A0022012030BCC1E9E1
:10DDB00000327047D8270020C84900200E4B0F4A78
:10DDC00093F8001392F8940393F80023904293F889
:10DDD00000230CD8904238BF93F80023D3F8FC32CC
:10DDE0003ABFC2F180028018002018447047D3F86F
:10DDF000FC32801A18447047D8270020C8490020F8
:10DE000030B51C4C1C4D94F8003394F8001385B0C9
:10DE100005F567721344029395F8943303928B428D
:10DE20001DD894F80023934211D294F80013019363
:10DE3000C1F180010091D3B9012208B93F2906D967
:10DE40000023694602A846F039F995F8943394F80E
:10DE50000003C01AB0FA80F0400905B030BD94F854
:10DE600000130022591A019200910122E5E719449A
:10DE70000222E2E7D8270020C84900202DE9F0431C
:10DE8000164685B0002936D0441E254D254F04EB9B
:10DE900001084FF0000901E0A0452CD095F894034B
:10DEA00014F8013F411C2844C9B280F89C330B068A
:10DEB00048BF002097F8003385F894134ABF014605
:10DEC000084685F894938B4297F800338ABFC3F1D4
:10DED0008003C01AC0183F28DED997F800338B4260
:10DEE000DAD0114B93F89430002BD5D00020FFF7F7
:10DEF00087FFA045D2D1694602A8FFF72FFF20B1C6
:10DF0000DDE9003213443F2B02D805B0BDE8F083B1
:10DF10000246334602A846F0D1F805B0BDE8F083CA
:10DF2000C8490020D82700200000002030B585B067
:10DF3000694602A8FFF712FF58B9094C04F542756B
:10DF4000D4F8083328465B6898470028F8D005B015
:10DF500030BD0246012302A846F0B0F8EDE700BF4D
:10DF6000D827002070B5124E1546D6F804330A465D
:10DF7000411999420F4988BF1D1A91F8941396F8D8
:10DF80000033994282B0044603D00192FFF7CEFFDE
:10DF9000019AD6F8081308480023C6F834332B46F4
:10DFA0008D6A2146AC4602B0BDE87040604700BFB4
:10DFB000D8270020C8490020E02A00208C461346BC
:10DFC000014662461846CDE738B52448244C002364
:10DFD000C4F8043302461178022902F106022CD05B
:10DFE0000133062BF7D11F4DD4F808330022C5F8B2
:10DFF0009023F3B1DA6AE2B11B489047D5F8903329
:10E00000C5F88803A3B19A885B88D21A436802FBDB
:10E010000333C4F80433FAF775FC95F8942394F8A5
:10E0200000339A42054601D0FFF780FFC4F8FC5246
:10E0300038BD0E4BC5F8883338BD0A4DD4F80823D7
:10E0400003EB430300EB4303C5F8903312B1D26AEC
:10E05000002AD1D10548C5F88803D4E7E44D002053
:10E06000D8270020C8490020E02A0020887C050825
:10E0700010B50A4CD4F808335B6A13B104F542704A
:10E080009847074AD4F8FC32D2F888235288013BDB
:10E09000134452421340C4F8FC3210BDD82700206C
:10E0A000C8490020084B09498B4202460AD218464B
:10E0B00002E01C30884205D20388C3F30B039A4266
:10E0C000F7D1704700207047B86C060860740608E6
:10E0D00070B585880B460446C5F30B052A4600211A
:10E0E000184648F028FD6169084A9142034602D368
:10E0F000074A914205D319B1BDE870401846084758
:10E1000070BD2A46BDE8704048F0B2BC6074060895
:10E110006C76060838B5064C064DAC4206D2A168AE
:10E1200020461C34FFF7D4FFAC42F8D338BD00BF03
:10E13000B86C0608607406084840082310F0800F89
:10E1400082EA40010ABF4000C8B2C0B2013BF5D12B
:10E15000704700BF30B505688D4219D901F1FF3E07
:10E160006C1E00231EF801CF082183EA0C0313F074
:10E17000800F82EA430C0ABF5B005FFA8CF3DBB2CC
:10E180000139F4D17445EDD16A1C02602B7030BDA9
:10E1900000236A1C02602B7030BD00BF07EE901A8E
:10E1A000B8EE677ADFED7C7A27EE000A60EE277A18
:10E1B000BDEEE77A17EE103A2033402B00F2DB80F9
:10E1C0009FED767AB4EEC70AF1EE10FAB0EE677AF8
:10E1D0000CDDDFED735A9FED736AF0EE476AF4EEE3
:10E1E000C66AF1EE10FA37EE657AF6DCDFED6E6A9C
:10E1F000B4EEE67AF1EE10FA0CD5DFED695A9FED38
:10E200006B6AF0EE476AF4EEC66AF1EE10FA37EE8A
:10E21000257AF6D4DFED666AB4EEE67AF1EE10FA0E
:10E2200000F39D80DFED636AB4EEE67AF1EE10FA5A
:10E2300044BFDFED5D6A36EEC77A27EE075ADFEDA1
:10E240005E5A9FED5E6ADFED5E6ADFED5E4AA5EE27
:10E25000256A27EE054AE5EE066AF7EE005AA4EEB7
:10E26000267AF0EE656AE7EE646AE7EE245A86EEF7
:10E27000A54A9FED4F7A77EE877ABDEEE77A17EEE3
:10E28000103A2033402B6FD89FED4F7AB4EEC70A77
:10E29000F1EE10FA0CDD9FED426ADFED426AB0EE5E
:10E2A000677AB4EEE67AF1EE10FA77EEC67AF6DC2B
:10E2B0009FED3D7AF4EEC77AF1EE10FA0CD59FEDA2
:10E2C000386ADFED3A6AB0EE677AB4EEE67AF1EEDC
:10E2D00010FA77EE867AF6D49FED357AF4EEC77AA7
:10E2E000F1EE10FA4CDD9FED397A77EE677A67EE42
:10E2F000A74A9FED317A9FED315ADFED316AA4EEE6
:10E30000875A67EEA43AE4EE856AB7EE006AE3EE58
:10E31000A67AB6EE007A36EE676AB8EE005A67EE75
:10E32000857A26EE077AB7EE005AC5EE256A0023F5
:10E33000836143610362C36180ED044A26EE877AFC
:10E3400026EE866A66EEA77A80ED095A80ED007A9D
:10E3500080ED016A80ED027AC0ED037A7047DFED4F
:10E360001B6A36EEC77A68E7DFED197AB6EE007AF7
:10E37000B7EE006AD7E7B7EE004AF0EE445A78E706
:10E380009FED0C7AF4EEC77AF1EE10FA44BF9FEDE0
:10E39000067A77EE677AAAE727D4D2360024F448C3
:10E3A000DB0FC940E4CB1641DB0F49C0E4CB16C1FB
:10E3B000DB0FC93FDB0FC9BF92E741B99730083C7B
:10E3C00015A82ABEF304353F00247448DB0F4940EA
:10E3D000000000009FED2E7A70EE077AFDEEE76AEE
:10E3E00016EE903A2033402B4FD8B4EEC70AF1EE28
:10E3F00010FA0CDD9FED276ADFED276AB0EE677A31
:10E40000B4EEE67AF1EE10FA77EEC67AF6DC9FED1E
:10E41000237AF4EEC77AF1EE10FA0CD59FED1D6A5F
:10E42000DFED1F6AB0EE677AB4EEE67AF1EE10FA2D
:10E4300077EE867AF6D49FED167AF4EEC77AF1EE8F
:10E4400010FA1DDC9FED177AF4EEC77AF1EE10FAA0
:10E4500044BF9FED127A77EE677A27EEA76ADFED69
:10E46000125ADFED126A9FED127AE6EE256A67EE28
:10E47000865AA6EE267AE5EE877AB0EE670A7047EE
:10E480009FED0C7A77EE677AE7E79FED0B0A70470E
:10E49000DB0FC93FDB0FC940E4CB1641DB0F49C09E
:10E4A000E4CB16C1DB0FC9BF92E741B99730083CF6
:10E4B00015A82ABEDB0F494000000000F0EEC07A2C
:10E4C000B0EEE07AB4EEE77AF1EE10FAB4BFB0EE57
:10E4D000676AB0EE476AB5EE406AF1EE10FA46D0D0
:10E4E000B4EEE77AF1EE10FA8CBFF0EE675AF0EE78
:10E4F000475AC5EE866ADFED1F2ADFED1F3ADFEDD2
:10E500001F4A9FED1F5A9FED1F3A9FED1F4ADFEDF7
:10E510001F5AE6EEE23AA6EE834AE6EEA34AB7EECB
:10E52000006AA6EEA45AA6EE846AE6EE855AC5EE07
:10E53000866AB4EEE77AF1EE10FA48BFDFED147A9E
:10E54000F5EEC00A48BF77EEE66AF1EE10FA48BF72
:10E55000DFED107AB5EEC00A48BF77EEE66AF1EE5D
:10E5600010FA48BFF1EE666AB0EE660A7047DFED5A
:10E57000076ADEE739094E3DE3B59E3E88FA163E4E
:10E5800045FE7F3F99FB243F69A2163EA7DFA834D2
:10E59000DB0FC93FDB0F494090ED005A9FED4C0A5D
:10E5A00035EE000A08B5FDEEC07A17EE903A20333A
:10E5B000402B7BD8FAF758FBF0EE403AFDEEC57AD7
:10E5C00017EE903A2033402B7FD8B0EE450AFAF789
:10E5D0004BFBB0EE405AD0ED014A9FED3D0A34EEC0
:10E5E000800AFDEEC07A17EE903A2033402B69D8AE
:10E5F000FAF73AFBF0EE405AFDEEE47A17EE903A65
:10E600002033402B5BD8B0EE640AFAF72DFBF0EE16
:10E61000404A90ED023A9FED2E0A33EE000AFDEEDD
:10E62000C07A17EE903A2033402B45D8FAF71CFBFE
:10E63000B0EE404AFDEEC37A17EE903A2033402BFD
:10E6400037D8B0EE430AFAF70FFBF0EE407A24EE2B
:10E65000233A27EEA36A24EE057A67EE856AB0EEC8
:10E66000462AF0EE432AA7EE242AE6EEE42AA6EE96
:10E67000247AE3EE646A24EE254A65EEE77A25EE15
:10E68000655A65EEA35A81ED004AC1ED017AC1EDEC
:10E69000024A81ED032AC1ED042A81ED055AC1ED3C
:10E6A000066A81ED077AC1ED085A08BDDFED093A27
:10E6B00084E7DFED087ACAE79FED064ABAE7DFEDA7
:10E6C000054AA6E7DFED035A96E79FED025A82E777
:10E6D000DB0FC93F000000002DE9F04389B0541C56
:10E6E00003941478002C00F0078100250746884623
:10E6F0001E46A94609E021463846C047039A01351F
:10E70000531C03931478002C3DD0252CF3D1931C7B
:10E71000CDE903395078302800F09480A0F130031F
:10E72000DBB2092B4FF0000440F297806C2838D000
:10E73000782822D857282AD9A0F15803202B1CD892
:10E74000DFE803F0B41B1B1B1B1B1B1B1B1B1B95B8
:10E750009D1B1B1B1B1B1B1B1B1BAF1B1B1B1B11FD
:10E760001BA71B1BB40056F8043B049A009300231C
:10E7700041463846FAF726FB0544039A531C039397
:10E780001478002CC1D1284609B0BDE8F0830028D8
:10E79000F9D02528F1D125213846C0470135039A03
:10E7A000AEE7039B5A1C039219787829A8D85729F9
:10E7B00058D9A1F15803202BA2D801A050F823F07A
:10E7C000C5E8000801E7000801E7000801E70008C4
:10E7D00001E7000801E7000801E7000801E7000879
:10E7E00001E7000801E7000801E700086FE80008FA
:10E7F000DDE8000801E7000801E7000801E700087C
:10E8000001E7000801E7000801E7000801E7000848
:10E8100001E7000801E70008A5E8000801E7000893
:10E8200001E7000801E7000801E7000867E70008C2
:10E8300001E70008E9E8000801E7000801E700082F
:10E84000C5E80008D31C03939078A0F13003DBB235
:10E85000092B4FF001043FF669AF04AA03A941F068
:10E8600011FD63E700298ED0252994D048E756F89A
:10E87000041B3846C9B2C0470135039A40E756F831
:10E88000040B05A9FAF734FB05AB0093049A234661
:10E890006EE756F8040B05AB00220A21FAF7E0FAFE
:10E8A000F2E7039A56F8043B1D6029E7A0F15802ED
:10E8B000B2FA82F256F8040B520905AB1021FAF7AE
:10E8C000CFFAE1E7A1F15802B2FA82F256F8040B4E
:10E8D000520905AB1021FAF7C3FAD5E756F8040B35
:10E8E00005A9FAF705FBCFE756F8040B05AB0022A4
:10E8F0000A21FAF7B5FAC7E7254644E70EB400B592
:10E9000084B005AB019053F8042B0649039301A88A
:10E91000FFF7E2FE019B00221A7004B05DF804EBE1
:10E9200003B07047458E00082DE9F043DFF8E8900A
:10E93000374F93B0FFF7C8F9FFF746FB99F800335C
:10E9400097F894239A4201D0FFF7F0FAD9F804839C
:10E950000025C9F8FC52B8F1000F11D02D4E6C46BD
:10E960002A4631462046FFF7C9FF204645F09CFE67
:10E970002035014601222046FFF780FAA845EFD84E
:10E9800099F8003397F894239A4201D0FFF7CEFA12
:10E99000D7F888339B7B012B33D099F8003397F855
:10E9A00094239A4201D0FFF7C1FA0027C9F8FC72FC
:10E9B000B8F1000F28D0DFF85C903D466C462A463F
:10E9C000494609A8FFF79AFF21220021204648F076
:10E9D000B2F8202221462846FFF7C4FA2022064634
:10E9E00009A92046154448F0E3F808B9202E00D0C4
:10E9F0000137A845E3D8B7FA87F0400913B0BDE85E
:10EA0000F083FFF735FBC8E7012013B0BDE8F083C2
:10EA1000C8490020A0E20508D82700202DE9F043CE
:10EA2000002483B00646048021463046013434F089
:10EA3000CBF8082CF8D10023DFF8688086F8EA309C
:10EA4000C6F8EC30C6F8F030C6F8F430C6F8F83046
:10EA50001F46FC3699463A46414601A8FFF74EFF4D
:10EA60003546032401AA12F8013B6BB1013C05F8BD
:10EA7000013BF8D10137082F85F8009006F1040614
:10EA8000E9D103B0BDE8F083284622462021254481
:10EA9000013748F050F8082F85F8009006F1040679
:10EAA000D9D1EEE7C0E2050803685A1C026019706C
:10EAB0000368090A5A1C02601970704702681146FF
:10EAC000531C036011F802CB0160D31C5178036022
:10EAD00093781B0443EA0123111D0160D07843EAB7
:10EAE0000C0343EA00607047A0F13003092B07D9FB
:10EAF00020F02000413819288CBF002001207047E9
:10EB000001207047303809288CBF00200120704751
:10EB1000413819288CBF002001207047613819281E
:10EB20008CBF002001207047202805D00938042818
:10EB30008CBF00200120704701207047A0F14103E5
:10EB4000192B98BF20307047A0F16103192B98BF93
:10EB50002038704710B500F100440246013C04E043
:10EB6000B3EB0E0015D1A24214D012F8013BA3F171
:10EB70004100192811F8010BA0F1410C98BF203376
:10EB8000BCF1190F00F1200EEAD91B1A04D100289C
:10EB9000E9D110BD002010BD184610BD02B310B55C
:10EBA0008446841804E0B3EB0E0014D1A44513D0BE
:10EBB0001CF8013B11F8010BA3F14102192AA0F145
:10EBC000410298BF2033192A00F1200EEBD91B1AFD
:10EBD00004D10028EAD110BD002010BD184610BD98
:10EBE0001046704770B5044608460D4645F05CFD7A
:10EBF000064602E014F8013F43B12046324629465A
:10EC0000FFF7CCFF0028F5D1204670BD1C462046FA
:10EC100070BD00BF2DE9F041044686469EF800C055
:10EC2000BCF1200F7046ACF109050EF1010EF5D0D4
:10EC3000042DF3D9BCF12B0F5BD0BCF12D0F3BD1D0
:10EC4000102A4FF0010600F1010E58D19EF800C0C5
:10EC5000BCF1300F5FD04FF010086FF070450F27F8
:10EC600042460EF1010E00200DE0ACF1300C5FFACF
:10EC70008CFC94450FDA854274462DD32AD008FBCC
:10EC800000C01EF801CBBCF1390FEED94CF0200CBE
:10EC9000BCF1600F0BD801B10C600EB323B1B0F121
:10ECA000004F28BF4FF000404042BDE8F081ACF17A
:10ECB000570C5FFA8CFCDCE7102A864649D04FF0EF
:10ECC000FF35B5FBF2F502FB05F7FF43FFB29046B7
:10ECD0000026C6E76745D2D21E404FF0FF30D0E78E
:10ECE000002BE2D06FF00043984228BF1846BDE8E1
:10ECF000F081102A4FF0000600F1010EA6D04FF06F
:10ED0000FF35B5FBF2F502FB05F7FF4390F801C0B4
:10ED1000FFB29046A5E79EF801C0ACF1410019286A
:10ED20000EF10104624601D80CF12002782A4FF05E
:10ED3000100805D0A6466FF070450F27424690E7B1
:10ED40009EF802C06FF070450EF1020E0F2742468A
:10ED500087E700267AE700BF2DE9F04F41F694627D
:10ED60008DB00021BD4847F0E6FEBD4A002309935F
:10ED700009920999043209680A930A920A9A10685A
:10ED800051EA000240F05881B64B03934C22002117
:10ED9000B24847F0D0FE4C220021B04847F0CBFEED
:10EDA000039BAE49D3F84434AF4A0A600124C1E959
:10EDB00007334B620C7144F0F1FAFFF705F90021BB
:10EDC000084609F001FBF9F79DFDB0F1000B40F397
:10EDD0000481A64BA64D0193A04BA64E002402949D
:10EDE00003F14C092746A24605F5886804E00AF5B8
:10EDF000006AD34540F3AA80019AD2F8A032C2F843
:10EE0000A432F9F713FC202241465046FFF7AAF836
:10EE100099491222404647F0CBFE0028E7D1BA4577
:10EE200022D00299954BCDF8149001EB410203EBEF
:10EE300082004A1C924902920490FFF75FFDDDE9CF
:10EE40000403D9F81C2043F84C0BC9E908228D4A69
:10EE5000C9F80C70C9F82820AAEB07070122C9E9F4
:10EE60000477C9F808209946039BD3F84434C9F8BD
:10EE70001C3057461222A918335D91F8401499426C
:10EE800002F101020BD00024202AF4D12037BB4527
:10EE90004146384650DBFFF765F80022EBE70134C6
:10EEA000152CF1D1D01978492022FFF75BF80BA976
:10EEB00000230A227448CDF82C80FFF7ABFE0490A3
:10EEC0000B98002301300A220B90FFF7A3FE079056
:10EED0000B98002301300A220B90FFF79BFE06904F
:10EEE0000B98002301300A220B90FFF793FE059048
:10EEF0000B98002301300A220B90FFF78BFE074688
:10EF00000B980023013019460A220B90FFF782FE6E
:10EF1000049989B1DDE9063243EA4212059B7F017B
:10EF200047EAC323A1F2BC7143EA600342EA4122EB
:10EF300043EA0243C9F81C30029B642B00F0EE80C8
:10EF400057460AF5006AD3453FF756AF029A642A3E
:10EF500000F0E480BA4500F0E580484C4849494E4D
:10EF60000C2303FB0244531C1A462046AAEB070558
:10EF70000293FFF7C3FCD9F81C30C9F80040C9E977
:10EF80000375C9E908330123C9F81450C9F828608A
:10EF9000C9F80830029B5D1C4C22304F02FB05F57E
:10EFA0007B190021184647F0C6FD4C22002147F08E
:10EFB000C2FD039A3549D2F844247951029C426239
:10EFC000C0E904BBC0E907220122023486628260E4
:10EFD0004FEA4B03B3F1805F1EDA4C221F4D02FB58
:10EFE00004F42B191846002147F0A5FD4C220021FE
:10EFF00047F0A1FD0399CBF10062D1F84414034618
:10F00000520023482851C3E90422C3E90711022210
:10F010005A71012259629A60104A95682DB9137984
:10F020001BB11368002B40F08B80002108460DB007
:10F03000BDE8F04F09F0C8B94FF47A7218180023F0
:10F0400045F0F6FF134B40F26D11A3FB00231B0CA0
:10F05000022440F2B2720D4627E000BF20B6002025
:10F060006028004000000020A8650608D82700207E
:10F07000C8490020ECE20508C8E20508284E002037
:10F08000DCE20508BDDF0008084E002004E30508A7
:10F0900014E3050807452EC2013212F00304A3EB66
:10F0A00001030CBF4FF4B77129469942F4DD794949
:10F0B000002C3FD003910399D1F814148B4272DBDA
:10F0C000754D01245B1A55F8041F994204F101049F
:10F0D000F8DD013343EA4413A2F2BC7243EA42234F
:10F0E0006E4A039DB0FBF2F102FB11024FF4616026
:10F0F0003C24B2FBF0F100FB11221C20C5F81804DF
:10F10000B2FBF4F004FB1022521042EA401242EA31
:10F11000C12242EA0343C5F8443437E66423604E13
:10F12000029337E7029B01245D1C002B3FF450AF94
:10F130005B4E31E70C4603911D21C4F81814BAE761
:10F14000C2E911551564D56329462E46D46C02F1E7
:10F150004C0354B39C681E64481E8442C3E9116684
:10F16000DE6312D0481C844216D08C427FF45DAF1F
:10F17000084600283FF459AF116CCC6B0134CC63C6
:10F180001964936401461A46E0E700293FF44DAF45
:10F19000884253F80C2CECD1117900293FF445AF8B
:10F1A00053641A64EEE7012493E73E49022226469F
:10F1B00013E0CB6B0A635B011DBF03F6FF7702F11F
:10F1C000FF3303EB17331346C1E90466C1E90D337E
:10F1D00051F84C0F5A1C0135C8B10B79002BE8D1FE
:10F1E0000F690A63002F47D14F691046531E4863C9
:10F1F000002F4AD007F6FF7703EB1733201A8B63F3
:10F20000C41851F84C0F5A1C01350028E5D1264985
:10F210002648C1F8F4523E220D46013BC1F8D022E7
:10F22000019140223F21C5E9B512C5E9B934990FD2
:10F230009A00C5F8CC0253B340F2FF10121841F106
:10F240000001520A42EAC15202F1400101980A4407
:10F2500002EBC303C0F8E022DA0DC0F8C422114A61
:10F26000C0F8EC22C0F8F0225A02C0F8DC12C0F854
:10F27000C832C0F8C022D8E607F6FF77531E03EB6A
:10F2800017304F694863002FB4D11346B6E7012207
:10F29000DAE700BF000000201404002080510100C4
:10F2A000BDDF000820B60020D827002020E3050895
:10F2B00001230A220021ADE42DE9F04117461E4644
:10F2C00005464FF47A7200233846314645F0B0FEC9
:10F2D0004449454A014482FB0143C8170B44C0EB33
:10F2E000631382FB03021A44D817404CC0EB62122E
:10F2F00084FB02044FEAE27C3D48CCEBA40C80FB8B
:10F300000C404FEAEC74C4EBE010C3EB0314A1EB28
:10F310008401A971C2EB0211A3EB81036B710CEBA9
:10F320004C03A2EBC30240F2B55303FB10CCBCF577
:10F33000896F2A714FEA800045DA40F2DA239C4552
:10F3400048DCBCF5B77FB4BF00220122294B02EB99
:10F35000420103EBC1034FEA420833F8463C91B245
:10F36000254C08EB020E04EBCE0416344FF00B0EC6
:10F3700001E034F8023D634520DDBEF1010EF8D115
:10F380001C4B424403EBC2024FF0010E32F85C3CCE
:10F3900085F802E000F5FA600CF1010C0844ACEBD2
:10F3A000030C288085F803C04FF47A720023384696
:10F3B000314645F03DFE2A81BDE8F0810EF1010E97
:10F3C0005FFA8EFEE4E7032140F296530A464FF0BF
:10F3D0000608C5E7022140F229430A464FF0040817
:10F3E000BEE700BF80BC92C789888888ABAAAA2ADA
:10F3F00073B06D16F87C05089C7C050808B50D4BAC
:10F40000D3E9E02352EA030C09D1002340F20112B0
:10F4100042808380837103800381184608BD0649BA
:10F42000D1F8A0128A1843F10003FFF745FF01202D
:10F4300008BD00BFC8490020D827002090422DE910
:10F44000F0410B46044615460AD2B0FBF5F6134AC6
:10F4500005FB16441846135D00F8013BBDE8F0813A
:10F46000B0FBF2F69642B6FBF2F706D20B4A05FB6A
:10F470001767D15D03F8011BEAE7BA42B7FBF2F860
:10F4800007D9064A05FB187812F8081003F8011B83
:10F49000EDE74046FFF7D2FF0346F2E728E3050811
:10F4A000B5EEC00ADFED347AF1EE10FACCBF30EEE3
:10F4B000270A30EE670ADFED317A20EE270A70B5B1
:10F4C000FDEEC07A86B017EE904A054684EAE470F5
:10F4D000002303A9A0EBE470CDE9003302933FF0D1
:10F4E000B1FA002CACBF20232D2303A88DF80030E7
:10F4F00045F0DAF801286E4628D0022832D00328D9
:10F500001CD003A9304647F01EFB304645F0CCF82E
:10F510000338C4B222463146284647F0A9FA0023F0
:10F520002B55284645F0C0F82E232B5401303119B5
:10F53000284447F024FB284606B070BD302303A9B9
:10F5400030468DF8013047F0FEFADEE743F2300234
:10F55000302303A93046ADF801208DF8033047F081
:10F56000F2FAD2E743F2300303A93046ADF8013096
:10F5700047F0E9FAC9E700BF6F12033A00007A4486
:10F580000378202B024600F10100F9D0092BF7D0B7
:10F590002D2B28D02B2B03BF5378B7EE000A024641
:10F5A000B7EE000AA3F13001C8B209289FED567AE0
:10F5B00010D8F2EE046A07EE901AF8EEE77A12F825
:10F5C000013FE7EE267AA3F13001C8B20928B0EE78
:10F5D000677AF0D92E2B5ED003F0DF03452B07D0DE
:10F5E00020EE070A70475378BFEE000A0246D9E7BB
:10F5F00010B451782D2978D02B296AD0A1F130038D
:10F60000092B02F101026BD80024002303EB8303D2
:10F6100001EB430312F8011FA1F130000928A3F107
:10F620003003F3D9B3F59A7F1A4628BF4FF49A7284
:10F63000072B66D9DFED356A1346F7EE007A083BF3
:10F64000072B67EEA67AFAD802F00702DAB1F2EEDB
:10F65000046A012A67EEA67A15D0022A67EEA67A16
:10F6600011D0032A67EEA67A0DD0042A67EEA67A97
:10F6700009D0053A67EEA67A05D067EEA67A012A88
:10F6800018BF67EEA67A6CB387EE277A5DF8044B55
:10F6900020EE070A70475378A3F13001C8B2092859
:10F6A00002F1010298D8F2EE046AF0EE665A07EE13
:10F6B000901AF8EEE77A12F8013F87EEA66AA3F1F6
:10F6C0003001C8B2092866EEA56A37EE067AEED98F
:10F6D00082E79178A1F13003092B02F1020293D95C
:10F6E000F7EE007A27EE277AD0E79178A1F1300380
:10F6F000092B02F1020288BFF7EE007AC4D8012478
:10F7000083E7F7EE007AA1E70000000020BCBE4CC2
:10F710006D4BB3F81C2CB3F820CCB3F8220CB3F823
:10F72000261CB2F57A7F88BF4FF47A7210B588BF75
:10F73000A3F81C2CB3F81E2CB2F57A7F84BF4FF4CB
:10F740007A72A3F81E2CBCF57A7F88BF4FF47A7CBE
:10F75000B3F8242C88BFA3F820CCB0F57A7F84BFFF
:10F760000020A3F8220CB2F57A7F84BF4FF47A729E
:10F77000A3F8242CB1F57A7F84BF0021A3F8261CBE
:10F7800084459CBF0020A3F8200C914228BF002292
:10F79000B3F8321C28BFA3F8242CB3F8342C9142C0
:10F7A00084BF0022A3F8322CB3F83C2C82B0002A8C
:10F7B0005CD0464C94F8AE33062B97BF44499FED7E
:10F7C000450A01EB830191ED010A94F8B013002979
:10F7D00049D1414B93F8340007EE902A07EE100A06
:10F7E000F8EEE77AF8EEC76A94F8B22386EEA77AC5
:10F7F0000AB130EE000AB4EEC70AF1EE10FA36DDB7
:10F8000067EE807ABCEEE77A8DED017A9DF8041000
:10F8100007EE101AB8EEC77AF4EEC77AF1EE10FAD6
:10F82000C4BF0131C9B200294BD01029A8BF102193
:10F83000C9B281420A4638BF024683F8342093F8A1
:10F840003D20032A17D9002283F83D2093F83C205D
:10F850002249D964032A18D9214A1A65002183F85C
:10F860003C1002B010BD042B19D8DBB91A4B93F829
:10F870003D20032AE7D81949C2EB021201EB4201ED
:10F8800093F83C20D964032AE6D8154902EB82009C
:10F8900002EBC00201EB82021A6502B010BD053B0B
:10F8A000032BE3D9F7EE007A87EE800A46F044FB9B
:10F8B000B4F8AC23084B904228BF1046A4F8AC0320
:10F8C000D5E70121B4E700BFC8490020D0380020A7
:10F8D000F87C05086F120338C05A0020D852002067
:10F8E000505300202DE9F04FA14C83B094F85430D0
:10F8F000A3F11702022A00AF00F2B8829D4B3B60D1
:10F9000094F864A09C4EDFF88CC2DFF88C82DFF89C
:10F910008CE20AF1FF3B5FFA8BFB31460020B146D7
:10F92000C7F804B00D6815F0010600F099820130A7
:10F93000C0B26B08AA0802F0333203F077331344E5
:10F94000EA0802F01132EB1A9B1A03EB131303F0CF
:10F950000F33ACFB03B2D209C2EB02229A1AAB03FB
:10F9600001D5012A1AD0012A40F26F82082A15D83F
:10F970001EB115EA0E0F40F068826E060AD515F426
:10F98000057F07D0BAF10F0F00F05F827B68062B6E
:10F9900040F25B8238EA050300F057824E46764813
:10F9A0000DF000FA0025022084F804510DF03EFA13
:10F9B00094F80831022B00F0EF82002800F04C830D
:10F9C0006E4B94F8D5A103F524794FF47A784FF073
:10F9D000000E4FF0640B5A88B2F57A7FB3F84620D8
:10F9E00088BFA3F80280B2F57A7F9A8888BFA3F80F
:10F9F0004680B2F57A7FDA8888BFA3F804809988B8
:10FA0000B2F57A7F84BF0022A3F806E09142B3F8F2
:10FA10005A10B3F85C2098BFA3F804E0914293F821
:10FA20006B2088BFA3F85AE0013A632A93F86C2050
:10FA300088BF83F86BB00132D2B2092A88BF83F83D
:10FA40006CE003F166001946002291F80AC010F834
:10FA5000015B0132AC4538BF00F801EC032A01F12B
:10FA60000601F2D1BAF1010F18BF83F885E0A43383
:10FA70009945B0D1424B93F8AE33042B00F0C782C6
:10FA80004BB93F4AB2F8AC33B3F5F07F84BF4FF4C3
:10FA9000F073A2F8AC33FFF73BFE3A4894F8EF114D
:10FAA000F9F7CEFA94F8FD110E30F9F7C9FAB4F867
:10FAB0000A22B4F808321343B4F80C2213431BB2E1
:10FAC00013B10123A4F80E32D4F8C4312E4A1A40DF
:10FAD000002A00F0D682D90700F142825A0440F190
:10FAE000D6812A49D4F8C8210B400A40C4F8C43151
:10FAF000C4F8C82113F4004200F01682002284F8F2
:10FB00006B2084F87B20D90440F1188294F81B32D2
:10FB10001F4D022B04BF012384F81B3205F1780826
:10FB20002B4602E0063343450CD01A78072AF9D158
:10FB30009978DA78914202D35A79002AF2D00720D4
:10FB400020F04AFF00234FF4806084F804310DF068
:10FB50006DF9002800F07382DFF83490CB469BF8F3
:10FB6000051041B39BF8000018B32B461BE000BF03
:10FB7000C05A0020F87C0508545B00205053002038
:10FB8000D0380020B05C002009600002F6DFFFFDE5
:10FB9000E05C00208180808040000200BC02020006
:10FBA0000633434507D01A788A42F9D15A79002A98
:10FBB000F6D020F011FF0BF1060BC345CFD1C04B9F
:10FBC00093F8AE53082D00F0D98194F8D531BD4992
:10FBD000D4F8C821A3F10103B3FA83F35B0984F8D5
:10FBE000983294F8D631A3F10103B3FA83F35B0999
:10FBF00084F89C3291F8193C032B84BF002381F8D0
:10FC0000193CB149D4F8C431C2F3C0300B400A40AA
:10FC100094F84A1084F89A02C4E97132002900F07D
:10FC2000DF81B4F8B032002B40F0E481D4F8B43274
:10FC300013F07F4F1CBF0023C4F8B432D4F8BC3299
:10FC400023F4007323F002031BB140F20223C4F833
:10FC5000BC3294F8B83294F8C0A2013B042B88BFA0
:10FC60000123A5F1050588BF84F8B832032D40F2C1
:10FC70005081BAF1000F1BD000237B60DFF864B223
:10FC8000CBF1000504E005EB0B03534580F0038145
:10FC90001BF8010B0028F6D00CF096FC0028F2D0DF
:10FCA00083799B07EFD57A680123002A40F0F8801A
:10FCB000834B93F8B2331BB1814A002382F8B233ED
:10FCC000B4F8223413F00C0F03D1C3F30313022B47
:10FCD00003D94FF42063A4F82234B4F8243413F089
:10FCE0000C0F03D1C3F30313022B03D940F60123F6
:10FCF000A4F8243494F89D3494F891249A4294F80A
:10FD0000903405D9002284F8912453B1A4F89424A6
:10FD100094F89C249A4204D2002384F89034A4F8E6
:10FD2000943494F8863594F892246849D7F800A062
:10FD30009A4284BF002384F8923401F1780B11F8C1
:10FD4000013C03EB43035344032593F800E193F88C
:10FD500001C193F802010B461A787245A8BF72469A
:10FD600003F8012B5A796245A8BF62465A719A7806
:10FD70008242A8BF0246013D9A70EDD11E318B45EB
:10FD8000DDD1D4F88C20002A00F02481002001214C
:10FD900099F80030282B08D199F80130043301FA82
:10FDA00003F313421CBF9A43012009F10609C14520
:10FDB000EED108B1C4F88C20DFF82C9109F10808C5
:10FDC0004B4613F8012B072A00F290809845F8D192
:10FDD000EB4688B06B46FF211846202246F0ABFE6A
:10FDE0004946034611F8012B53F82200013040F038
:10FDF0008480884543F82220F4D1B4F8CE21B4F8A9
:10FE0000CC319A42DD4602D3314BC4F8CC31FF23CA
:10FE1000304984F8B83596F90430142B04D0326890
:10FE200031EA020200F0F0802B4B0C36B342F2D1E3
:10FE3000234B93F8A131022B03D1214A002382F8EE
:10FE4000A1310C37BD46BDE8F08F234B0C318B42FE
:10FE50007FF468AD013802284E467FF6A3AD9EE5DB
:10FE600091F90430142B7FF464AD97E51B4A3A6096
:10FE700002EBC30393F82020002A3FF441AD5B6AF4
:10FE8000002B7FF43DAD172384F8543038E51D076F
:10FE90006FD5134926E67A680023002A3FF408AF9D
:10FEA000074991F8BD23002A7FF40AAF91F8B123E6
:10FEB000012A3FF4FDAE002B7FF4FAAE00E700BF4D
:10FEC000D0380020C84900209EDFCDFDDB52002045
:10FED000AE014A0101000200C05B0020F87C050869
:10FEE000FE9FFFFD843C00208F3C0020EB4688B045
:10FEF0002022FF21684646F01EFE09F8015B01350D
:10FF0000082D3FF47AAF09F8015B0135082DF4D1D3
:10FF100073E7614B002283F8B023BAF1000F00F0C1
:10FF2000A48001237B60A9E694F86B1000293FF4BC
:10FF3000EAADD90484F87B203FF5E8AD1A067FF5D9
:10FF4000E5AD94F85410182906D8544B01228A4084
:10FF50001340002B7FF4DAAD514D05F17808F1E53F
:10FF60005049D4F8C8210B400A40C4F8C431C4F841
:10FF7000C82198047FF5BEAD4B49B3E51A4693F806
:10FF8000B233002B3FF421AE92F8BD33012B04BFF6
:10FF9000022382F8BD3318E600283FF411AD434B2D
:10FFA00094F8551190F904C04FF0FF0E03F16C0066
:10FFB00093F90820624504D1013983F808E0C9B2F9
:10FFC00001250C338342F3D1002D3FF4F9AC84F8C2
:10FFD0005511F5E4282020F0FFFCD4F88C20D5E65C
:10FFE00033490B430A43C4E97132B4F8B032002BF1
:10FFF0003FF41CAE94F8AC020CF0E6FA00287FF453
:020000040801F1
:1000000015AEA4F8B00211E684F8B83510E7D4F8BC
:10001000C431214A23F48053C4F8C431D4F8C83120
:1000200023F48053C4F8C831B2F8CE33B3F57A7FE5
:10003000BFF431AD4FF47A73A2F8CE332BE5D4F888
:10004000C43123F00063C4F8C431D4F8C83123F0BC
:100050000063C4F8C8317FE5D4E9712322F080023F
:1000600023F08003C4E97123AAE41A4693F8BD3350
:10007000002B7FF425AE92F8B133012B7FF420AE34
:1000800016E6D4F8C82143F0080342F00802C4F889
:10009000C431C4F8C8211EE5D03800200041000159
:1000A000E05C0020F79FFFFDF6BFFFFD185C00201D
:1000B000000605002DE9F04F794F7A4BD7F8C82597
:1000C00002F2DC52C7F8C825774A934283B080F029
:1000D000E48003F11C059B46744B754E4FF0010AFA
:1000E00003F10208714B5A88002A00F0BE8008EB29
:1000F0000203B34280F0B980444608E01A881C46E7
:100100001344002A00F0B180B34280F0AE80052A8B
:1001100040F2AB8035F81C2C6188C2F30B0291428F
:10012000ECD162799207E9D1238855F8141C94F830
:10013000049001935846FDF7CBFF35F81C2CB9EB22
:10014000123F00F09A804FF0000A35F8181C55F85D
:10015000140CC1F30B013FF0FFFD55F8043C18608F
:10016000514B0BF11C0B9B4505F11C05BAD3D7F87D
:10017000C431C7F8C831FFF7B5FB97F83C304D4A9A
:100180004D4C03EB830103EBC10397F83D10A2F143
:100190007800C1EB011100EB410102EB8303C7E9D9
:1001A00013131FF093FE4FF0FF33386DC4F848343B
:1001B0002AF032FC20F064FC404B03F1780102E0AD
:1001C00006338B4263D01A78002AF9D19D78D8780B
:1001D000854202D358790028F2D097F8183284F873
:1001E0004C2403EB830303EB83039B00632BB7F8DF
:1001F0001C223349C7F80C16D8BF6423C7F8C03592
:10020000642303FB02F2632ADCBF1A46C7F8C43535
:100210004FF00003C8BFC7F8C425C7F8C835C7F8F2
:10022000CC35C7F8D035C7F8D435C7F8D835C7F8B6
:10023000DC25A7F8E03587F8E2352BF017FAB7F898
:10024000140697F8161621F091FA35F075FB16F0A2
:100250005FF91C4AD2F8A022C7F8C82501235046EE
:1002600087F8E13503B0BDE8F08F55F8141C584607
:10027000FDF72EFF4FF0000A67E7019BA11D9A1FB3
:100280005846F8F7F5FB00287FF45FAF5BE797F877
:100290004B20003A18BF01229FE74FF0010A66E7A2
:1002A000C05A0020B86C06086074060800400008B8
:1002B000008000085053002000000020E05C002077
:1002C000C85C0020D827002070B5164D164EFFF7E9
:1002D00009FBD5F8C835012403F2DC53C5F8C8354D
:1002E00085F81846FAF75CF928B13378B12B02D1BA
:1002F000F8F736FE18B9032C0FD00134F2E70B4A99
:100300000023D2F8A01285F818360122C5F8C815C6
:1003100085F8E12585F8193670BD40F0CFF940F039
:10032000B3FB00BFC05A002000400008D8270020BF
:1003300010B50B4C012384F8703F84F84A30FFF766
:10034000C3FFFFF7B7FE41F20242FF23A4F8742F68
:1003500084F8763F0E20BDE810400CF0B9BE00BF17
:10036000C05A002070B51B4D01230328064685F8AE
:10037000703F1ED9711CC9B249004029164A28BFD6
:100380004021002302244FF0140ED454023302EB18
:10039000030C99420CF801ECF7D8FF2E08BF02219C
:1003A0002944FF2381F8743FBDE870400E200CF013
:1003B0008FBE06EB8603094885F83C6006EBC30355
:1003C00000EB830028652AF027FB21F0EFFC21F0E9
:1003D000C3FDCFE7C05A0020346A002050530020EC
:1003E000054BD3F8B82F012142F4001283F8B51F52
:1003F000C3F8B82F704700BFC05A0020F0B5067987
:1004000006F0E003402B03D145794FF0FF3406E0BE
:10041000602B4FF00105F8D1447905FA04F400236C
:10042000012006F00706AB4200D1F0BD052E0FD823
:10043000DFE806F00308101D242448B1C85CD75C2F
:1004400078400FE020B1C856D756C71B7842784194
:100450000133E8E70028FBD031F8130032F81370BD
:10046000784080B220420CBF01200020F0E7002835
:10047000EED031F9130032F91370E6E70028E7D027
:1004800051F8230052F82370DAE7F8B50C4E3378B0
:1004900005468BB9F8BD25B12388C3F30B039D42F4
:1004A00004D0D4E90201A28846F0E2FA1C34BC422E
:1004B000F1D300233370EDE7024C034FF7E700BFA1
:1004C0005CE50020B86C060860740608037903F048
:1004D0001803102B1CD004D82BB1082B06D00020F9
:1004E0007047182BFBD1B0F80B007047104BB0F8D9
:1004F0000B0093F90030591C06BF0E4B1B78DBB282
:1005000003EB830203EBC20300EB830080B270476E
:10051000074BB0F80B0093F901305A1C06BF054B8E
:100520005B78DBB2C3EB031300EB4300EEE700BFE5
:1005300068040020FC5A002020B10078B0FA80F056
:10054000400970470120704738B5074C074DAC4251
:1005500003D3074B01221A7038BDD4E90210A288D8
:1005600046F086FA1C34F2E7B86C06086074060898
:100570005CE50020214BB0F5FA6F1A680346A8BF6E
:100580004FF4FA63B3F57A7FB8BF4FF47A73D204AD
:100590001FD540F2DC5290421ED007EE903A40F256
:1005A000DB529042F8EE677A97BFDFED156ADFED18
:1005B000156A9FED157A9FED150A85BF9FED147A98
:1005C0009FED140A77EEE67A77EEE67AA7EE870AD1
:1005D0007047B0F57A7F02D89FED0F0A704707EE9B
:1005E000903ADFED0E6A9FED0E7A9FED0E0AF8EE5F
:1005F000677A77EEE67AA7EE870A7047885C002074
:1006000000007A4400A0BB44D62000C000E0824431
:10061000D6200040000083440000000000407A44DF
:10062000661000400000404207F056B813B568B1AC
:100630004C1E14F8011F21B902B0BDE8104007F0AC
:100640005FB8019007F048F80198F2E702B010BDDA
:1006500073B5104C0192064660680D46A0B10E4974
:10066000FFF7E4FF60683146FFF7E0FF0B49606881
:10067000FFF7DCFF0A49019B60682A46FEF72CF869
:1006800008496068FFF7D2FF237A0BB10123637238
:1006900002B070BD5CE500206BE3050841E9050888
:1006A0002906010878E3050870B50546B0F8090089
:1006B000FDF7F8FC054B1E7804462846FFF706FFB9
:1006C00016B1E368184470BDA368FBE75CE5002041
:1006D00038B505460C46FFF7E7FF2B7903F0E0023B
:1006E000602A03F007032AD1052B0CD8DFE803F0BA
:1006F000030B0F0B1B1B6A7901239340DBB20278BB
:1007000014B11343037038BD22EA0303FAE76A7990
:10071000012393409BB2028814B113430380F2E794
:1007200022EA0303FAE76A79012303FA02F2036873
:1007300014B113430360E6E723EA0203FAE7052B4B
:10074000E1D8DFE803F00303050507070470DAE7E3
:100750000480D8E70460D6E708B5202146F002FA05
:10076000034620B11A78202A00F10100F8D018467B
:1007700008BD70B50D461446FFF7EEFF0646A0B162
:10078000FEF796FD40F634039842A8BF1846B0F530
:10079000617FB8BF4FF46170A0F561731920B3FB9E
:1007A000F0F32B702378013323703046FFF7D4FF2A
:1007B0000646A0B1FEF77CFD40F634039842A8BF80
:1007C0001846B0F5617FB8BF4FF46170A0F5617352
:1007D0001920B3FBF0F36B7023780133237030469C
:1007E00070BD10B50C4628B1C94301F001010138B4
:1007F00007F02CFEE30701D4FCF7E4FE10BD38B58A
:1008000007490546FEF7EEF90649041E284618BFBB
:100810000124FEF7E7F908B144F00204204638BD90
:100820007CE3050879FC0508F7B5114E074630460C
:10083000002300F80A3F0C460E4B0F49002F08BF5B
:100840001946154646F07FF90C4F04EB45050A366C
:10085000AC4202D10A4803B0F0BD394634F8022B4D
:100860006846FEF74BF86946304646F06CF9EFE70C
:100870005CE5002088E305087FE3050891E30508AF
:1008800066E50020F7B50C4E0C4F002306F83B3F01
:10089000044600EB4105AC4202D1094803B0F0BD6B
:1008A000394634F8022B6846FEF728F86946304688
:1008B00046F049F9EFE700BF5CE50020EBE50508ED
:1008C00097E50020F8B5084F4E1E054601F11F04BC
:1008D00016F8012F28463946FEF710F8A64205F112
:1008E0000205F5D1F8BD00BF96E305080246531C8A
:1008F000084605D1044B1A681B790A600B717047D2
:100900000249FDF7FBBF00BFD7E30508ECE505088A
:100910002DE9F341124D134F002305F8643F0446BF
:1009200000EB8106B44203D10F4802B0BDE8F0816C
:100930003946284646F007F92146684646F01FF931
:100940004FF000082021684646F00CF928B96946A6
:10095000284646F0F8F80434E4E780F80080F1E730
:100960005CE5002081E40508C0E50020024BD3F8D7
:10097000880034F043BF00BF5CE5002008B5254B7C
:100980001B68DB040AD5B5EE400AF1EE10FA12D16D
:100990009FED210A45F0D0FA80B208BDDFED1F7A45
:1009A000B4EEE70AF1EE10FA28DA9FED1D0A45F0E1
:1009B000C3FA80B208BDDFED197AB4EEE70AF1EEB2
:1009C00010FAE5D49FED177AB4EEC70AF1EE10FAEB
:1009D0008BBFDFED157A9FED157A9FED157A70EEDE
:1009E000677A8ABF70EE677A9FED120A9FED120A4E
:1009F000A7EE870A45F0A0FA80B208BD70EE677ACC
:100A00009FED0E7A9FED0E0AA7EE870A45F094FA45
:100A100080B208BD885C00200080BB4400004042DA
:100A200000007A4400E082440000834466BEFFBEBA
:100A300066BEFF3E0060BB4400A0BB4438DFFF3E03
:100A400000407A442DE9FF471E46C368BDF8307068
:100A5000DDF8348004468946924643B3CBB20C2B72
:100A60009ABF1A4AD5560025BAF1FF3F21D0236814
:100A7000174A3146CDE9005A3846C04752462079D8
:100A80005FFA89F1FAF744FB024600B10288D3B25B
:100A90000393C2F30323120BCDE9005202930D4AD4
:100AA000236831463846C04704B0BDE8F0874D1C86
:100AB000DAE77B06F8D42368074A0C9531463846B6
:100AC000C44604B0BDE8F047604700BF58E30508DE
:100AD0009BE30508A8E30508CDE305082DE9F041EF
:100AE000154686B06A1C8846BDF830600D9F1946D1
:100AF00026D0030900F00F044033CDE90045174A22
:100B000005933046B847C0B1EAB20D2AD8F80000C4
:100B100098F8051011D82A46FAF74CFB68B10288FC
:100B200001780391C2F30321120BCDE90042029137
:100B3000059B0B4A00213046B84706B0BDE8F0815E
:100B40007306FAD40309074A00F00F000C904033F3
:100B50003046BC4606B0BDE8F0416047DCE305081E
:100B6000EEE3050818E4050810B5013114460BF052
:100B700001FD28B9064B1A681B792260237110BD4C
:100B8000C27904492046BDE81040FDF7B7BE00BF5A
:100B9000D7E3050839E405082DE9F04188B01F4680
:100BA0000309DDF838801546403300F00F0429B3FF
:100BB00007930BF0DFFCC279079BCDE900420646A4
:100BC000134A29463846C047A8B13068114DFAF794
:100BD00043FBB2797179079B12F0020F0E4A08BFEE
:100BE0002A46F5790094CDE90101CDE903250021DC
:100BF0000A4A3846C04708B0BDE8F081084A0E945A
:100C000029463846C44608B0BDE8F041604700BFF9
:100C10002CE40508A5F305083EE605083EE40508B2
:100C200060E40508F8B5066904460F46002E5DD15C
:100C30000368C3F30A02CAB12368396803F1784232
:100C4000B2F5002F48D2324D2A6942F001022A61E2
:100C50004FF4801019603BF0C3FF2B696FF3000362
:100C60002B6103283FD06FF001063FE003F178428B
:100C7000B2F5002F16D2264D2A6942F002022A61EF
:100C80006B612B6943F040032B614FF000403BF058
:100C9000A7FF2B6966F341032B610328CCD04FF0EB
:100CA000FF3623E003F1774202F57802B2F5002F18
:100CB000C2D2174D2A6D42F002022A656B652B6D78
:100CC00043F040032B654FF000403BF0B5FF2B6D28
:100CD00066F341032B65E0E703F1774202F5780202
:100CE000B2F5002F04D32368043323603046F8BDE7
:100CF000074D2A6D42F001022A654FF480101960F9
:100D00003BF09AFF2B6D6FF300032B65A9E700BF43
:100D1000003C024090F88730DFED6A5A03EE903ACB
:100D200090F88B3006EE103A90F8893004EE103AC5
:100D300090F88A30F8EEE33A04EE903A90F88D306D
:100D400063EEA57AB8EEC66A03EE903A26EE256AFF
:100D5000B8EEC44AF8EEE44AF8EEE33A26EE276A23
:100D600024EE254A64EEA54A63EEA53AF0B5564D49
:100D700024EE064A64EEA74A63EEA73A002106264F
:100D8000F7EE002AA5F10C0C00F1660E06FB01F24D
:100D9000B7EE005AAC1890F886700244F0EE456A3F
:100DA00015E0012904F1060402F10602EED190F8E3
:100DB000883007EE903A90F8903006EE903AF8EED0
:100DC000E77AF8EEE66A27EEA55A66EEA56A23787A
:100DD00007EE103A66EE867AB8EEC77A27EE277AE3
:100DE000FDEEC77A17EE903AFA2BA8BFFA2323EA52
:100DF000E3731372637807EE103A66EE847AB8EE06
:100E0000C77A27EE277AFDEEC77A17EE903AFA2BCB
:100E1000A8BFFA2323EAE37353725CF8213007EE8C
:100E2000903A002BF8EEE77A49DDA37807EE103A06
:100E3000B8EE477A90F88C3037EE677A03EE103AC6
:100E400087EE272AB8EEC33AB0EE627A23EE253A4F
:100E5000A2EE037A64EEA77A66EEA36A67EE857A5D
:100E600027EE877AFDEEE77ABDEEC77A17EE103AE5
:100E7000FA2BA8BFFA2323EAE373937217EE903A92
:100E8000FA2BA8BFFA2323EAE3730EF80130A388F4
:100E900007EE903AF8EEE77A013167EEA67AFDEEBA
:100EA000E77A17EE903AB3F57A7FA8BF4FF47A73DA
:100EB00023EAE3738F429381BFF673AFF0BDB7EEC1
:100EC000007AC7E70AD7233C9487050890F88E304C
:100ED0006BB3B0F85A308BB190F88F2002EB8203DD
:100EE0006421C3EB0313B3FBF1F3A0F85A3096234C
:100EF00012FB03F3B3FBF1F3A0F85C3043884BB172
:100F000090F88F3003EB8303C3EB03136422B3FB2E
:100F1000F2F34380B0F846304BB190F88F30962210
:100F200013FB02F36422B3FBF2F3A0F846307047E0
:100F300090F821304BB3438B83B190F82230FA22E2
:100F400013FB02F203EB8303B3F57A7FA8BF4FF4E0
:100F50007A7364218383B2FBF1F24283838843B1C5
:100F600090F82230FA2213FB02F36422B3FBF2F36F
:100F70008380C3884BB190F8223003EB8303B3F531
:100F80007A7FA8BF4FF47A73C380704770B50A4C5C
:100F90000A4E002594F8863013B12046FFF7BAFEBA
:100FA0002046FFF793FF01353046FFF7C1FF042DC0
:100FB00004F1A404EED170BD50530020E055002090
:100FC000034BD3F88C0008B106F09ABB704700BF02
:100FD0005CE5002008B50B4605490246D1F88C00B7
:100FE00028B10449FDF778FBBDE80840E8E708BDF3
:100FF0005CE50020290601080FB407B504A951F8E3
:10100000040B0191FFF7E6FF03B05DF804EB04B0B9
:10101000704738B50A4B03EBC0050C4695F8902194
:10102000084803EB8203196AFFF7E6FF95F896314B
:101030002BB1611C0448BDE83840C9B2DCE738BDBB
:1010400088870508D8F20508EBE50508024B01463C
:10105000D3F88C00FFF7EABA5CE5002008B5044637
:101060000848FFF7F3FFFFF7ABFF074BD3F8880003
:101070000BF0B4FF09F0C4F8012C01D13FF004FDDE
:10108000FCF7A0FA72E405085CE500200048DDE703
:10109000A3F305080CB4C30607B500D561B90498DD
:1010A00005A90191FFF796FFFFF7F0FF012003B0BC
:1010B0005DF804EB02B070470020F8E708B5FFF7D1
:1010C000C5FFBDE80840E1E710B504460348FFF757
:1010D000BDFF2046BDE81040F0E700BF7EE40508F4
:1010E00008B5034610462AB1DB0600D511B1FFF75B
:1010F000EBFF002008BD2DE9F04F2DED028B0A46D5
:101100008BB000218246FFF7EBFF6F4D814605F162
:10111000800B00266D4B1C78AB7AB34200F39580B0
:101120001035AB45F5D140F21620FCF7BBFFD0E9F6
:1011300002530CB12C461D460DF1100B1522002157
:10114000584645F0F8FC00272E78002E44D06978E8
:10115000039130460BF00EFA95F9023002935A1CB7
:10116000534208EE100A5341002C00F0A980039965
:10117000002214F802C0B44504EB020040F09C8049
:1011800090F90280029A424540F0948042788A4267
:1011900008BF012301220BF8072003F001034A4690
:1011A00083F0010150460393FFF79AFF039B8146AA
:1011B0004CB1474A18EE101ACDE900A2304642461B
:1011C000FFF78CFC039B434A18EE101ACDE900A2EE
:1011D0003046029AFFF782FC0137152F05F103050F
:1011E000B2D16CB33A4FDFF8EC8004F13F061BF844
:1011F000013B02930BBB2078F8B194F90220013235
:101200001BD061780BF0B6F94A46054601215046DD
:10121000FFF766FF94F90220029B29468146207859
:10122000CDE900A7FFF75AFC2078029BCDE900A882
:101230004FF0FF322946FFF751FC0334B442D6D1B8
:101240000BB0BDEC028BBDE8F08FE888FCF72AFFFD
:10125000D0E902230CB114461A46297A6B7A06FBB0
:10126000013312F9038014B3E756B8450CBF0123CC
:1012700000234A4614BF0121002150460293FFF784
:101280002FFF029B814644B1114A3146CDE900A2AD
:1012900028463A46FFF7D6FB029B0E4A3146CDE977
:1012A00000A228464246FFF7CDFB013632E74FF059
:1012B000FF37DAE700236DE703323F2A7FF459AFA7
:1012C0004FF0FF386BE700BF6C0400205CE50020A6
:1012D000B11401089510010808B50948FFF7F4FE9C
:1012E000FFF76EFE074B002483F89040C3F890414F
:1012F00083F8944120F000FF2046FFF7AFFE00BFC7
:1013000083E405085CE500202DE9F04F8BB007462B
:1013100040F216200391FCF7C5FE039A0446002113
:101320003846FFF7DDFE404AD4E9025314780646FA
:101330000CB12C461D461522002104A845F0FBFBEC
:1013400005F13F03039395F80090B9F1000F31D0F8
:1013500095F801A0002C65D022460023117849455C
:1013600058D128336B4492F80180012203F8182CDD
:10137000D045324614BF0121002138460CBF4FF042
:10138000010B4FF0000BFFF7ABFE064654B1B8F16E
:10139000000F07D0254B00935A463B46414648462E
:1013A000FFF7FAFB224B00935A463B46514648460C
:1013B000FFF7F2FB039B03359D42C4D13CB3DFF83A
:1013C0006C90DFF86CA0651C0DF11008403418F823
:1013D000013BCBB915F8013CB3B116B13046FFF76C
:1013E00073FE297815F8010CCDF800903B460022D9
:1013F000FFF7D2FB002215F8010CCDF800A03B4608
:101400001146FFF7C9FB00260335A542DFD10BB01B
:10141000BDE8F08F0133152B02F103029ED14FF08E
:101420000008A5E7A046A3E75CE50020B114010889
:1014300095100108154B1B6870B52BB31448154E59
:10144000FFF73CFEFFF7BCFDFCF73EFC0025FCF778
:1014500071FC044640B113200BF03AFEFFF716FE74
:10146000BDE870400C4829E63046FFF7C5FD782DF1
:1014700006D80135FFF7A4FD64200AF00DFEE6E76B
:10148000FFF704FE2546F5E770BD00BFDC2A00200B
:10149000AAE4050876510608C4E40508034B014692
:1014A000D3F88C0008B106F017B970475CE500204E
:1014B0000CB407B510F020000BD079B92320FFF74A
:1014C000EDFF049805A90191FFF784FDFFF7DEFD0C
:1014D000012003B05DF804EB02B070470020F8E78C
:1014E0002DE9F04F914689B00C461A4600218046FE
:1014F000FFF7F6FDDFF8ECB006464D460027B9F1E0
:10150000000F6CD029460622204645F0EAFA002852
:10151000324614BF0121002140460CBF4FF0010AA2
:101520004FF0000AFFF7DCFD0646287814F0D2F8E9
:10153000079010B3687914F0CDF8079BEA785B79CF
:101540000793AB7895F801E04FF461714FF0190CF7
:101550001CFB03131CFB0212297900B14079CDF862
:1015600004E0CDE90232079B0093CDE904103B462D
:101570005A4651464046FFF79BFF207814F0AAF8E0
:10158000079010B3607914F0A5F8079BE2785B79B7
:101590000793A37894F801E04FF461714FF0190CB0
:1015A0001CFB03131CFB0212217900B14079CDF81A
:1015B00004E0CDE90232079B0093CDE904103B46DD
:1015C0005A4651464046FFF765FD0137142F04F196
:1015D000060405F1060592D109B0BDE8F08FCA46B0
:1015E000CBE700BFCAE405082DE9F04F174689B0E4
:1015F0001A460C4600218146FFF772FD3B4EDFF88C
:10160000F4B007F16C0380463D46079394F904104B
:10161000374A002392F90800884263D00133092B2E
:1016200002F10C02F6D1079B0C359D4204F10C042B
:10163000ECD109B0BDE8F08F29460C22204645F0D8
:1016400050FA0028424614BF0121002148460CBF31
:101650004FF0010A4FF0000AFFF742FDEA7995F9D1
:10166000043006EB82028046D2F8602204922A7A85
:1016700006EB82025146D2F860220392AA7906EB69
:1016800082024846D2F8602202926A7906EB820210
:10169000D2F8602201922A6800925A46FFF708FFAA
:1016A000E27994F9043006EB82025146D2F86022C6
:1016B0000492227A06EB82024846D2F86022039214
:1016C000A27906EB8202D2F860220292627906EBDE
:1016D0008202D2F860220192226800925A46FFF7F5
:1016E000D9FCA0E7002FA7D1BA46D9E7888705081B
:1016F000185C0020E3E405082DE9F04F8BB00C46A0
:10170000089200211A460746FFF7EAFCDFF8B4B05A
:10171000089D099000264FF019094FF46178089B45
:10172000002B4BD029460A22204645F0DAF9002842
:10173000099A14BF0121002138460CBF4FF0010A5D
:101740004FF0000AFFF7CCFC2A890692EA8805923E
:101750002A790492EA780392AA78099019FB028206
:1017600002926A7819FB028201922A78009233462B
:101770005A4651463846FFF79BFE22890692E28878
:10178000059222790492E2780392A27819FB0282F0
:101790000292627819FB0282019214F80A2B0092DD
:1017A00033465A46514638460136FFF773FC1E2E23
:1017B00005F10A05B3D10BB0BDE8F08FDDF820A02C
:1017C000DBE700BF00E505082DE9F04F2DED088BA4
:1017D000DFF82CA195B0804691461F460C46164670
:1017E0004FF0000B94ED008AB5EE408AF1EE10FA4E
:1017F0007FD0D4ED019A94ED029AD4ED038AB9F129
:10180000000F49D0D6ED00BA96ED01BAD6ED02AA86
:1018100096ED03AAB4EE6B8AF1EE10FA6ED1F4EEF7
:101820004B9AF1EE10FA69D1B4EE6A9AF1EE10FA21
:1018300064D1F4EE4A8AF1EE10FA0CBF01210021C6
:101840003A460D46404681F00101FFF749FCB0EEF3
:101850006B0A074611A8FDF723FEB0EE4B0A07906E
:101860000EA8FDF71DFEB0EE6A0A06900BA8FDF764
:1018700017FEB0EE4A0A059008A8FDF711FE05997B
:10188000069A079B039002910192009352465B4691
:1018900029464046FFF70CFEB0EE480A11A8FDF7B6
:1018A000FFFDB0EE690A05460EA8FDF7F9FDB0EEA2
:1018B000490A06900BA8FDF7F3FDB0EE680A059003
:1018C00008A8FDF7EDFD069B059A0390CDE90053AE
:1018D00002925B465246002140460BF1010BFFF796
:1018E000D9FBBBF1080F04F1100406F110067FF4D8
:1018F00079AF15B0BDEC088BBDE8F08F00219FE7F4
:1019000023E505082DE9F74F92460C461A460021BB
:101910008146FFF7E5FBDFF870B0804656460025AC
:10192000BAF1000F2ED031460422204645F0D9F8F6
:101930000028424614BF0121002148460CBF012760
:101940000027FFF7CDFB738801933AF82530009309
:1019500080462B465A4639464846FFF7A9FD63881C
:10196000019334F8043B00935A462B4639464846C7
:101970000135FFF78FFB042D06F10406D0D103B02B
:10198000BDE8F08F5746EAE737E505082DE9F04F47
:1019900089468FB0174600211A460646FFF7A0FB7E
:1019A000DFF878A0054600240DF1240B59F8243007
:1019B0000293594602A83CF0A7FF67B357F82430BA
:1019C000029A0393934218BF01212A4608BF0021BF
:1019D00030460CBF4FF001084FF00008FFF780FBC6
:1019E00004A9054603A83CF08FFF04A900912346F3
:1019F000524641463046FFF75BFD2346CDF800B026
:101A00005246414630460134FFF744FB202CCDD1ED
:101A10000FB0BDE8F08FB846EFE700BF48E5050816
:101A20002DE9F04F924685B00C461A4600218146BA
:101A3000FFF756FBDFF874B0804655460026BAF132
:101A4000000F31D029460422204645F04AF80028EC
:101A5000424614BF0121002148460CBF0127002740
:101A6000FFF73EFBEB780293AB7801932B88009352
:101A7000804633465A4639464846FFF719FDE37813
:101A80000293A378019334F8043B00935A463346FB
:101A9000394648460136FFF7FDFA102E05F10405D8
:101AA000CDD105B0BDE8F08F5746E8E752E505080F
:101AB0002DE9F04F87B0144603911A4600210546E0
:101AC000FFF70EFBDFF830B106464FF000080623A3
:101AD00003FB08F7C0374FF00009039BDB5D04935D
:101AE000002C00F08580E35D049A05939A4218BFAC
:101AF0000121324608BF002128460CBF4FF0010AE1
:101B00004FF0000AFFF7ECFA059B0646CDE900937B
:101B10005A46434651462846FFF7CAFC049B5A469C
:101B2000CDE9009351464346284609F10109FFF7E4
:101B3000B1FAB9F1060F07F10107CED108F101089A
:101B4000B8F1060FC3D1DFF8B0B0E427039BA7F1CB
:101B5000E40913F807A0002C4CD0E35D04939A45E8
:101B6000324614BF0121002128460CBF4FF0010866
:101B70004FF00008FFF7B4FA049B0646CDE9009346
:101B80005A46062341462846FFF792FCCDE9009AC3
:101B9000194A0623414628460137FFF77BFAEF2F03
:101BA000D4D1039B93F8EF70B4B194F8EF8047451C
:101BB000324614BF0121002128460CBF0124002415
:101BC000FFF78EFA002300930B4ACDF80480072319
:101BD00021462846FFF76CFC00230093064A019734
:101BE000072321462846FFF755FA07B0BDE8F08FD6
:101BF000A24693E7A046C9E764E505082DE9F04F42
:101C000089B00C46079200211A460746FFF768FA8A
:101C10000026079DDFF8A0B00690B2464FF01909E4
:101C20004FF46178079B43B329460622204644F0CF
:101C300058FF0028069A14BF0121002138460CBF26
:101C40004FF0010A4FF0000AFFF74AFA6A7906904E
:101C500019FB028205922A7919FB02820492EA7822
:101C60000392AA7802926A7801922A780092334607
:101C70005A4651463846FFF71BFC627919FB02822F
:101C80000592227919FB02820492E2780392A278EB
:101C900002926278019214F8062B009233465A465B
:101CA000514638460136FFF7F5F90A2E05F10605CB
:101CB000B8D109B0BDE8F08F78E505082DE9F04FFF
:101CC00089B00F4691460021139A98460646FFF7C1
:101CD00007FA87EA09096FEA0903DFF88490069397
:101CE0000446002528460AF05BFE129B184230D0BD
:101CF000069BDFF870B0034014BF4FF0010A4FF0AD
:101D0000000A049310EA070314BF4A465A462846BD
:101D1000059307920AF056FE079A039000904346F7
:101D200051463046FFF7C4FB049BB3FA83F12246C9
:101D300049093046FFF7D4F9059A039B00930446FE
:101D40004346002A14BF5A464A4651463046FFF7DA
:101D5000A1F90135182DC5D109B0BDE8F08F00BF3C
:101D600031E5050891E505082DE9F04F0A4687B0F1
:101D700000210646FFF7B4F93B4C05903B4A237817
:101D8000608802EB8303D3F820A0FCF78BF983680B
:101D90000493374BC1681A78002A4BD0DDF81080C5
:101DA0000491002721796279049B07FB012213F833
:101DB0000290B8F1000F3FD018F80250059A4D4537
:101DC00014BF0121002130460CBF4FF0010B4FF032
:101DD000000BFFF785F9013705907DB305F00F0281
:101DE0002D0940350292CDE90075224A53465946E5
:101DF0003046FFF75DFBB9F1000F2AD009F00F0262
:101E00004FEA1919029209F14002CDE900725346D6
:101E1000184A59463046FFF73DF9A279012A38BFE2
:101E20000122BA42BEDC144B0834A342A6D107B04B
:101E3000BDE8F08F9046B4E74546BFE7B8F1000F24
:101E4000D9D00E4A0097534659463046FFF730FB2B
:101E5000D1E77306E1D4094A009753465946304604
:101E6000FFF718F9D9E700BF188905088887050822
:101E70005CE5002098E50508E8890508AEE5050859
:101E80000FB407B504A951F8040B0191FFF7A2F8AC
:101E9000FFF7FCF803B05DF804EB04B070472DE9E0
:101EA000F041037903F0E002402A51D004D85AB13E
:101EB000202A29D0BDE8F081602A4CD0802AF9D1AF
:101EC00082794179264812E003F00703052B16D8E2
:101ED000DFE803F0101510150309D0F805102148AC
:101EE000BDE8F041CCE7D0F8052051421E48BDE8DE
:101EF000F041C5E7B0F80720B0F80510F6E7B0F9F3
:101F00000720B0F90510F1E74679184D184805EBA0
:101F1000C605FFF79BF895F8A47200240123A74299
:101F200003D8BDE8F041FFF7B1B8D5F8A06256F884
:101F300024204FEA84084AB113B90E48FFF786F807
:101F400056F808100C48FFF757F800230134E6E76D
:101F500041790A48C4E7BDE8F041094890E700BF6D
:101F600011E60508C2E50508D8E5050888870508D3
:101F7000EFE505088AE90508D8F2050800E6050836
:101F800028E605082DE9F04387B0FBF78DFE0269CE
:101F90008389018802928268019242880092426895
:101FA0001B4EDFF880801B4FDFF87C9004461A48F8
:101FB000FFF766FF002515B94046FFF77FF83B683D
:101FC0009D4213DA33781548052B96BF09EB83033E
:101FD0000022D3F84824B38800932946738801353A
:101FE000FFF74EFF062D06F10606E4D13EF036F966
:101FF00081884388CB1A616803FB01110591FBF7C7
:10200000DDFE05990246064807B0BDE8F04337E714
:10201000E44D0020544D002040E60508AAE60508DE
:10202000B9E605089EE605088887050802490348C1
:1020300001F5FD610EC923E700F0FF1FD6E6050894
:1020400010B57521044629F0BBFD01460948FFF78C
:1020500017FF1A21204629F0B3FD01460648FFF775
:102060000FFF1B21204629F0ABFDBDE810400146C3
:10207000024805E7EAE60508FDE6050810E7050859
:1020800038B50B4DE87810F0FD0405D10948FFF78D
:10209000F7FE2046FFF7D4FFEB78013B012B06D873
:1020A0000548FFF7EDFEBDE838400120C8E738BD20
:1020B000E055002023E705082EE705082DE9F04F3D
:1020C000634B644C1A686449644B6548B2FBF3F295
:1020D00093B0FEF791FFB4F89621624E624FDFF89D
:1020E000E481DFF8B4914FF47A73B2FBF3F103FBB0
:1020F00011220A20B4F9983192B2B2FBF0F25B4897
:10210000FFF7BEFE5A4A5B495B48FEF775FFFEF7D4
:10211000BDFF5A4B5A4A997B5A4B5B48D31A06EB80
:1021200081015A4AD1F860141288FFF7A9FE584875
:10213000FEF78CFF94F89A115648FEF75DFF56485B
:10214000FEF784FF94F89B115448FEF755FFFEF705
:102150009DFF5348FEF77AFF00210A46FB7F0B41A3
:1021600013F0010F01F1010508D012B14846FEF746
:102170006DFF29464046FEF73FFF0122072D294605
:10218000ECD1484D95F8CA1405F5C47305F13C022D
:10219000012918BF134693F88C30032B02D0424814
:1021A000FEF72AFF414B95F8CA14A3F5A672012940
:1021B00018BF134693F88C30012B02D13C48FEF730
:1021C0001BFF3A4B95F8CA14A3F5A672012918BF54
:1021D00013461B695B7B012B02D93648FEF70CFFC7
:1021E000354FDFF8E4A0DFF8E4B0FEF74FFFD4F896
:1021F0009C310393002507F1200957F8041B00299F
:1022000066D0012303FA05F8039B18EA030F1CD0DC
:1022100018F01F0F19D01AF8050059F8252052F8A8
:10222000202035B12548CDE90412FEF70FFFDDE986
:1022300004125846FEF7E0FEB8F1020F05D194F8FB
:10224000BD1111B11E48FEF7D7FE0135D5E700BF1D
:10225000000000205CE5002041E7050840420F0037
:102260004AE7050888870508E05500205DE705086E
:10227000F0FF0220000800007EE70508FC5A00205D
:102280000080000800400008A2E70508282B002075
:10229000D1E70508E3E70508EBE70508EDE70508E2
:1022A000F5E70508045600200EE805088C570020C5
:1022B00016E805081BE80508F08B05088AE90508FB
:1022C00029E8050805E80508EC04002023E80508CE
:1022D000FEF7DCFE7E4B7F481A687F4B1978137A35
:1022E000527A06EB8101D1F89C14FFF7C9FD7B49B6
:1022F0007B48FEF781FE7B497B48FEF77DFEFEF7BB
:10230000C5FE7A4B7A4819684FF47A73B1FBF3F142
:10231000FEF772FE07A8FDF771F838B107A90AA801
:1023200041F082FE73480AA9FEF766FEFEF7AEFE94
:10233000D4F88022002A00F0888007EE902ADFED92
:102340006E6AB8EEE77AC6EE877AFDEEE77A17EEA8
:10235000903AB4F8380958B107EE900ADFED666A92
:10236000F8EEE77A86EEA77AFDEEC77A17EE900AC6
:10237000D4F800525DB107EE905ADFED5F6AF8EED7
:10238000E77A86EEA77AFDEEC77A17EE905AB4F890
:102390003A196429A8BF6421CDE900055748FFF721
:1023A0006FFD94F83C3994F83D29B4F8401954482D
:1023B00006EB8303D3F8B034FFF762FDB4F850198D
:1023C000504889B2FFF75CFDFBF76EFC016921B153
:1023D00082684D48120DFFF753FD4C48FEF736FE5C
:1023E0004B4B1B681B065ED594F87039494F032B85
:1023F0008CBF49484948FEF729FE3B78022B26D17D
:102400004748FEF723FE94F87039042B43D845481B
:10241000FEF71CFE94F88039002B42D006EBC30374
:10242000D3F8C8144048FEF7E7FDFEF72FFE3F48FB
:102430003F4FFEF70BFE3F4B1C680125002C36D1A9
:10244000FEF724FE13B0BDE8F08F134681E70220AB
:102450000AF00EFD054608B93748D2E733F052FAC4
:1024600095F9041006EB80000131D0F86022334862
:10247000FEF7C2FDFB78012B04D13148FEF7E6FDE3
:102480003048BEE7AB79304806EB8303D3F86012DF
:10249000FEF7B2FDF4E7BB780BB92C48B8E72C483F
:1024A000B6E72C49BEE72C48FEF7D0FDBDE794FA0D
:1024B000A4F3B3FA83F305FA03F206EB8303384679
:1024C000D3F8FC1424EA0204FEF796FDB6E700BF39
:1024D000886900202DE80508876900203FE8050885
:1024E00060E805086EE8050874E80508782A002009
:1024F0007AE8050894E8050800247449A7E8050867
:10250000EDE8050814E9050823E905083EE9050892
:10251000885C0020C85B002044E9050850E90508F4
:1025200060E90508CE610608A8E90508C4E90508C0
:10253000B4E90508786A002066E9050870E905082D
:1025400084E9050889E90508FCE405088DE9050822
:102550009DE9050839E70508B8E905082DE9F04FB8
:10256000DFF8788198F8033099B0002B00F098805C
:102570005148524EDFF868B1DFF86891DFF868A182
:10258000FEF79CFD00252F460BA9E8B214F00CFACB
:102590009DF83430002B53D0139C54B107EE904A71
:1025A0009FED470AF8EE677A80EE270A43F0C4FCF5
:1025B00004460B9A29465846FEF71EFD109A002A3B
:1025C00070D002FB04F04FF47A73B0FBF3F309937D
:1025D000DDF848C0BCF1000F66D00CFB04F142F2FC
:1025E0001073B1FBF3F198F80330082D18BF7F1872
:1025F000002B5BD0179807901598069016980590B9
:102600000A2311984FF47A7EB0FBFEFE0998CDF8AC
:1026100010E0B1FBF3FE03FB1E11CDE902E10999C5
:10262000B1FBF3F103FB1100CDE90010BCFBF3F3A8
:1026300021465046FFF724FC0023C6E90D33B36260
:1026400001351D2D06F140069ED198F8033023B3C5
:102650001C4C1D48D4F88829D4F88419D2084FF4AA
:102660007A73B1FBF3F3D4F88C19FFF709FC0A2253
:102670001648B7FBF2F102FB1172FFF701FC144B95
:102680001B78432B06D1D4F89029D4F8941911481B
:10269000FFF7F6FB0023C4F88C3919B0BDE8F08FC2
:1026A0000D4866E7099293E761469CE72146484654
:1026B000FFF7E6FBC0E700BFDAE9050854E70020B2
:1026C0008096184B5CE5002081EA0508A1EA050820
:1026D000732B0020C5EA050838EA0508FC5A0020DB
:1026E00042EA050883ED050851EA050810B586B0F1
:1026F000104B0493104B0393104B0293104B019318
:10270000104B1149114A00930446114B1148FEF732
:1027100073FCFEF7BBFC10491048FFF7B1FB3CB15E
:102720000F4A1049104806B0BDE81040FFF7A8BB9B
:1027300006B010BD2FEB050834EB05083EEB05088D
:1027400047EB05086EE80508F9EA0508EFEA050811
:10275000035B002004EB050853EB05085BEB050861
:102760006CEB05087CEB050881EB05080120BDE753
:1027700013B52C48FEF76AFC2B4B93F82130002B45
:102780004DD02A4C2A48FEF799FC94F82C3A2BB1EC
:1027900094F82E3A13B194F82D3A7BB9254B26487C
:1027A00093ED280A8DED010AFEF750FCB4F8383994
:1027B0009DED010A33BB2148FEF780FCB4F8301AC6
:1027C0001F48FEF719FC94F82C3A13B31D48FEF786
:1027D00075FCB4F8341A1C48FEF70EFC94F82E3A37
:1027E000CBB11848FEF76AFCB4F8321A1748FEF766
:1027F00003FC94F82D3A83B1124802B0BDE81040B2
:10280000FEF75CBC43F098FB81B21148FFF738FB40
:10281000D4E71048DBE70F48E4E70E48EDE70E4841
:10282000EBE700BFAEEB05081C5B00205CE5002079
:10283000C4EB0508F4EE0020CBEB0508E5EB05083A
:10284000F4EB050814EC050824EC05083EEC05083B
:10285000EFEB05081DEC0508FA6A06082DE9F04FB4
:102860006F4B1B7889B0002B00F0D4806D4D6E4803
:10287000A9686E4CDFF8F0A1FFF702FB69686C48AD
:10288000FFF7FEFA6B4B6C48D4F84C2AD3E90031C1
:10289000C91AB1FBF2F2FFF7F3FAFEF7F7FB67484C
:1028A000FEF70CFC6648FEF709FC04F525634FF0C3
:1028B00000080793634B1B785FFA88F4A34222D881
:1028C000614C624FFEF7E2FB2646002556F8041BDA
:1028D00038460135FEF790FB162DF7D1FEF7D6FBF3
:1028E0005A4E0125234661681B683046C91A0135D6
:1028F000FEF782FB162D04F10404F3D109B0BDE804
:10290000F04FFEF7C3BB079B142603EB840306FBC3
:10291000045693ED000AB6F80E9043F00DFB96F8BE
:102920001EE01EF0010F14BF52222D221EF0020FD6
:1029300014BF54232D231EF0040F07EE903A14BF4A
:1029400056232D231EF0080F14BF4FF0430C4FF0F9
:102950002D0C81B21EF0800F4FF03C0BB1FBFBF150
:1029600005914FF0640114BF4FF0530E4FF02D0E40
:1029700080B201FB09F1671CCDE902E100930490EC
:1029800017EE903ACDF804C039465046FEF734FBB6
:10299000B37FDB073AD55C232D4A6343D118D05867
:1029A00091ED010A70B1DFED2B7AB8EE400A20EE0E
:1029B000270A07EE900AF8EE677A80EE270A43F0BE
:1029C000BBFA00B2642290FBF2F102FB1102224832
:1029D000FEF712FB142101FB075701FB0454F98891
:1029E000628A0491218B0391E18A0291A18B01916A
:1029F000A18A009102F0030319214B431748218A51
:102A00009208FFF73DFA08F1010853E71448FEF772
:102A10001DFBDFE7134809B0BDE8F04FFEF74EBBE2
:102A2000581D0020642E00205EEC05085CE50020A7
:102A30006EEC0508E02F002085EC0508B2EC0508D7
:102A40000EED0508805D0020102F0020BEED05086A
:102A5000842B002000401C4687ED05089CED0508EE
:102A600093ED0508C2ED05086AED05080EB403B53F
:102A700003AA52F8041B0192FDF7EAFD064BD3F8B6
:102A80008C201AB905495868FDF7D0FD02B05DF8F1
:102A900004EB03B0704700BF5CE50020A3F305081A
:102AA0002DE9F04798460B7903F0E004402C81466D
:102AB0000F46164631D1684DDFF8A081DFF8C0918E
:102AC000002422E03B7903F00703013B042B04D8E8
:102AD000DFE803F006080B0E2000315D28460AE00F
:102AE0003157FBE736F81410F8E736F91410F5E71C
:102AF00056F824104046FEF77FFA7B79013BA3424B
:102B000002DD4846FEF7A2FA01347B79A342D9DC04
:102B1000BDE8F08756F82410E0E703F00703052B23
:102B200058D8DFE803F0030C141619313578602CFF
:102B30005ED045D8002C66D0202C7CD0E8E796F9F2
:102B40000050602C54D03BD8002CF5D148E035889B
:102B5000EDE7B6F90050F4E7D6F800A0202C554672
:102B600069D02BD8002CD3D151463C48FEF744FA0B
:102B7000D7F805108A4518D8B8F1000FC8D03848E2
:102B8000BDE8F047FEF738BA202C356853D015D889
:102B9000002CBDD129463048FEF72EFAD7F8051093
:102BA000A94202DB4B42AB42E6DDFEF76FFA3A6820
:102BB0002C492B464846BDE8F04757E7602C17D014
:102BC000802CA5D13178284B2848002914BF3146E4
:102BD0001946D5E7202C2DD007D8002C98D12546B2
:102BE000B7F90540B7F9076011E0602CE8D100257E
:102BF0007B7945FA03F3DB07BDE8F0474CBF1C487F
:102C00001C48FEF7F9B9B7F80540B7F80760124855
:102C10002946FEF7F1F9AC42C7DCAE42C5DBB8F19C
:102C2000000F3FF475AF324621461348BDE8F04728
:102C3000FEF7E2B900257A79104B03EBC20393F853
:102C4000A4229542B1DAD3F8A03253F82500BDE8AA
:102C5000F047FEF7FBB900BFECE50508D5E5050830
:102C6000DEED0508E4ED05084A620608D8F205081D
:102C70003DE60508FA6A0608A1E305088887050805
:102C8000EBE705082DE9F04F85B0164601911A468D
:102C9000824600213046FEF723FA324C06F010033C
:102CA00005464FF000090293FEF78AF92379019A4D
:102CB00003F01803934203D0002A48D1182B46D1C1
:102CC000284B4FF00D0B0BFB0933B3F80900FBF752
:102CD000E9F980462046FDF7F9FBD8E902210746CD
:102CE000024401442046FDF789FB80F001012A4699
:102CF0000390C9B23046FEF7F3F9DDE90223054639
:102D000002B123BB174A0BFB09FB52F80BB0B2060A
:102D10000FD573B9144803935946FEF76DF9D8F8E7
:102D20000820039B3A4421465046FFF7B9FEFEF7C0
:102D3000ADF90E485946FEF75FF9D8F80C2000238C
:102D40003A4421465046FFF7ABFEFEF79FF909F1E2
:102D5000010940F23A23994504F10D04A4D105B0CC
:102D6000BDE8F08F38980508FEED0508FFED050871
:102D700013B50446084601920091FDF795FCDDE984
:102D800000130246204602B0BDE8104088E60EB4AB
:102D900003B503AA52F8041B0192FDF759FC054B39
:102DA00005495868FDF742FC02B05DF804EB03B03A
:102DB000704700BF5CE50020A3F305080049E6E783
:102DC00009EE050801490246E1E700BF18EE0508D3
:102DD0002DE9F04380468BB00846FDF7ADFB40B1CE
:102DE00000234D491A4601200BB0BDE8F043FEF721
:102DF000FBBBCDE90700099008464D1CFCF758FACB
:102E000044B2204609F0B8FF0646002842D08DF8AB
:102E1000204001242846FDF79FFC054638B10023D9
:102E20000A221946FBF7F6FE01340790E4B2DFF8F8
:102E3000F09000272846FDF78FFC054618B3FCF7F5
:102E400037FA3649002251F804CB6045D3B203D09B
:102E50000132102AF7D1002309EB8302D2F8602255
:102E6000904210D1022F1CD0032F1FD05A1E012FC9
:102E7000D2B211D00B2A03D88DF821300134E4B23C
:102E80000137042FD6D1052C16D840460BB0BDE82B
:102E9000F04397E70446BDE7042AF1D88DF82230C5
:102EA000ECE7052BECD88DF82430E7E79A1E0D2AC5
:102EB000E6D88DF82330E1E707AB03CB9DF823205C
:102EC00030601868164B716003EB8202B060D2F874
:102ED000602204929DF8242003EB82020021D2F8A4
:102EE000602203929DF8222003EB82020846D2F86A
:102EF000602202929DF8212003EB8203094AD3F855
:102F000060320193079B00939DF92030FEF7C2F8D1
:102F10000BB0BDE8F08300BF545B0020E8890508D2
:102F200088870508E3E40508F0B5054687B008463C
:102F3000FDF702FB0B46044640B100231C491A462C
:102F4000012007B0BDE8F040FEF7B2BD1949194FA6
:102F500002AA184643F0C2FD03AEB8B1032C04D157
:102F60002846FFF72FFF07B0F0BDFCF7A1F902AA32
:102F700046F8040B39460020013443F0AFFDECE77E
:102F80000D4832462146FEF77BFFECE7032CE7D1E4
:102F9000DDE90346059B01931A463146E0B232F063
:102FA00001FE019B0028EBD12846FFF707FFDAE777
:102FB000CCEF002081E4050864E50508F8B5064675
:102FC00008460C46FCF774F920210546204643F0DC
:102FD000C9FD044618B93046BDE8F840F2E6114F85
:102FE000114E3B7832789A4201D0FAF79FFF0F4B8F
:102FF00020461D6041F058FB012201462046FAF7A9
:103000003DFF3B7832789A4201D0FAF78FFF204695
:1030100041F04AFB2A460146BDE8F8400448FEF765
:103020002FBF00BFD82A00205C4D0020D42A0020EA
:103030002FEE05082DE9F041064688B008460D46FA
:10304000FCF736F920210446284643F08BFD20B9D1
:10305000304608B0BDE8F041B4E6FCF729F9224655
:10306000054601460F48FEF70BFF85B1202D2A4685
:10307000694628BF20222046FAF774FFE846064634
:103080000027B74208DBAD1B3444002EEDD1FDF71D
:10309000FDFF08B0BDE8F08118F8010BFEF7FEF95E
:1030A0000137EEE745EE050807B5009313460A46DB
:1030B0000249FFF76CFE03B05DF804FB5DEE050806
:1030C0002DE9F041064686B00846FDF735FA0F4671
:1030D000054640B1002354491A46012006B0BDE818
:1030E000F041FEF7FDB90846FCF7E2F81328044664
:1030F00000F3928006264643781C8DF81750FDF7A2
:103100002BFB494D074660B1FCF7D2F8C0B212F074
:10311000F5FA30B10379AB559DF8173001338DF8CE
:1031200017303846FDF718FB074660B1FCF7C0F8CA
:103130000D2808D8062303FB045358709DF8173058
:1031400001338DF81730B11C0DF1170229443846B0
:10315000FDF70FFBFDF700FB074660B1FCF7A8F891
:10316000012808D8062303FB045318719DF8173073
:1031700001338DF817303846FDF7EEFA78B1FCF7D9
:1031800097F8C0B212F0BAFA48B1062303FB045311
:1031900002795A719DF8173001338DF817309DF878
:1031A0001720042A4FF0060328D103FB0453002202
:1031B0009A801DF065FC06236343EE18E85C12F06C
:1031C00089FAF278B778192380464FF461757079DF
:1031D00013FB075713FB025512F07CFA437998F85A
:1031E0000520039333790097CDE901530F48737895
:1031F0002146FEF745FE06B0BDE8F081052A04D160
:1032000003FB045300225A71D3E7062A1FBFAA19F1
:103210000023AB519380CCE7054913232A4630465F
:1032200006B0BDE8F0413FE7E05C0020CAE40508D5
:1032300076EE05082DE9F04380468BB00846FDF791
:103240007BF90F46044640B1002365491A46012028
:103250000BB0BDE8F043FEF74FBA0846FCF728F87C
:103260001D28054600F3B3800A264643781C8DF8D6
:103270002740FDF771FA044630B1FCF719F89DF8C4
:10328000273001338DF827302046FDF765FA554C7D
:10329000074668B1FCF70CF80D2809D80A2303FB90
:1032A000054383F8600B9DF8273001338DF82730F4
:1032B000DFF82C91711C0DF1270249443846FDF7C7
:1032C00058FAFDF749FA074668B1FBF7F1FF2228E3
:1032D00009D80A2303FB054383F8630B9DF82730C5
:1032E00001338DF827303846FDF736FA074668B1C6
:1032F000FBF7DEFF0D2809D80A2303FB054383F8FB
:10330000640B9DF8273001338DF827309DF8273066
:10331000062B0CD009EB0602002349F80630404684
:1033200053601381FFF74EFD0BB0BDE8F0830A2612
:1033300006FB054600233846A6F8663BA6F8683B20
:10334000FDF70AFA074640B1FBF7B2FF9DF82730B8
:10335000A6F8660B01338DF827303846FDF7FCF9E7
:1033600058B1FBF7A5FF0A2303FB0543A3F8680B3D
:103370009DF8273001338DF827301B4B4FF0FF327B
:103380001A600A2202FB05424FF46170B2F8683BF2
:103390000693B2F8663B059392F8643B049392F867
:1033A000633B039392F8621B192313FB0101029103
:1033B00092F8611B13FB0103019392F8603B0093A9
:1033C00000210A4A2B460846FDF764FEACE708498F
:1033D0001D23224640460BB0BDE8F04364E600BF23
:1033E000BCF000205CE500204804002000E5050852
:1033F00076EE0508F0B5074689B00846FDF79CF85B
:103400000E46054640B1002319491A46012009B06D
:10341000BDE8F040FEF7BABA0846FBF749FF1F289F
:1034200004461CD83046FDF797F90146204632F095
:10343000F7FB78B10E4803AE314600EB84003BF059
:1034400063FA0C4A0096234629462846FDF722FED9
:1034500009B0F0BD384609B0BDE8F040AEE4064919
:103460001F232A46384609B0BDE8F0401CE600BFDD
:10347000CCEF002048E5050876EE0508F0B50746D4
:1034800085B00846FDF758F80E46054640B10023C2
:103490001C491A46012005B0BDE8F040FEF7C0BA4D
:1034A0000846FBF705FF0F28044622DC3046FDF7EF
:1034B00053F90146204632F031FBA8B1124B04F11A
:1034C000200203EB8203294693F8732A029293F8B1
:1034D000722A0192B3F8703A00930C4A23462846A8
:1034E000FDF7D8FD05B0F0BD384605B0BDE8F040A9
:1034F00064E407490F232A46384605B0BDE8F0408A
:10350000D2E500BF4CF000205CE5002052E5050844
:1035100076EE05082DE9F04F074689B00846FDF71D
:103520000BF88B46054640B100234C491A46012052
:1035300009B0BDE8F04FFEF761BB494B084693F870
:1035400000A093F8019093F8EA80FBF7B1FE0928F8
:1035500004467BDC062646430BF101008DF81F5024
:10356000FDF7FAF83D4D834648B1FBF7A1FE0D2863
:103570009FBF9DF81F30A85501338DF81F30584666
:10358000FDF7EAF8834660B1FBF792FE824508D367
:10359000062303FB045358709DF81F3001338DF848
:1035A0001F305846FDF7D8F8824660B1FBF780FE21
:1035B000484508D8062303FB045398709DF81F3034
:1035C00001338DF81F305046FDF7C6F8814660B1D3
:1035D000FBF76EFE804508D3062303FB0453D87027
:1035E0009DF81F3001338DF81F30311D0DF11F0282
:1035F00029444846FDF7BDF89DF81F30062B09D039
:10360000AA190023AB5138469380FFF7DBFB09B0C2
:10361000BDE8F08F6343EA184FF4617650791921C1
:1036200011FB00600590107911FB00610491D178C5
:1036300003919178029152780192EB5C0093002102
:10364000084A23460846FDF725FDE0E70649092319
:103650002A46384609B0BDE8F04F25E598660020B7
:103660005C5F002078E5050876EE05082DE9F74354
:1036700080460846FCF760FF0B46054628B14046E9
:10368000FFF7A0FB03B0BDE8F0832D49DFF8B09051
:1036900001AA184643F022FA2F4604462E467CB96A
:1036A000022DECD1A7F57A73B3F57A7F20D925499D
:1036B0004FF4FA634FF47A724046FFF7F5FCE1E706
:1036C0004DB1012D0FD001AA4946002043F006FA62
:1036D00001350446E3E7214640463BF0C5F8431C6C
:1036E0000646F0D1CEE72046FBF7E2FD0746EAE7C3
:1036F000154B1B68B8B25B689847FF2EBCEEC00A3A
:10370000124B0BD1124AF8EE407A1278A24212DC28
:1037100010EE101A0F48FEF7B3FBB3E7F8EE407A4D
:1037200003EB860310EE102A0B48C3ED007A3146F6
:10373000FEF7A6FBA6E7E3EC017A0134E6E700BF5B
:1037400081E405085DF605082C6A0020E8F10020F8
:10375000805D002089EE05087CEE05082DE9F34127
:1037600006460846FCF7E8FE0D46074670B1002401
:1037700001A920463BF066F9013401463046FFF7C7
:10378000EDFF122CF4D102B0BDE8F0810846FBF742
:103790008FFDC4B2112C72D8681CFCF7DDFF3C4DC4
:1037A0008046E8B93B4B03EB440393F8AC1C8A1EFC
:1037B00051425141374B03EB440393F8AC2CAA5CC4
:1037C000002955D093F8AD3C192040F2EE2100FBC2
:1037D00003133148214602B0BDE8F041FEF750BB6B
:1037E0000178284643F0BEF970B1032C94BF002243
:1037F00001222A4902EB4202431B0A4452FA83F394
:1038000093F86475032F05D1304602B0BDE8F0414E
:10381000FFF7D4BA4046FCF79FFF08B3022FF3D15D
:10382000FBF746FD40F6CA0280B29042194BA8BF92
:10383000104640F2EE22904203EB4403B8BF10461C
:10384000A0F2EE201922B0FBF2F083F8AD0CBB1E03
:10385000594259410F4B03EB440383F8AC7CA9E771
:10386000022FF4D1304602B0BDE8F041FFF7AABA0A
:103870000B48214602B0BDE8F041FEF701BB094903
:1038800011233A46304602B0BDE8F0410CE400BFD7
:103890000C1C06085CE5002098EE050888870508E2
:1038A000A8EE0508B5EE050810B504460848FDF772
:1038B00005FCFBF739F820B1BDE810400548FDF7DD
:1038C000FDBB20460449BDE81040FFF760BA00BFC9
:1038D000BDEE0508C7EE0508CFEE05082DE9F0415D
:1038E000144B1B6888B00446F3B11A6804A9D56A62
:1038F00018466A46A847064688B1DFF8448004ACFB
:103900006D46002735F8022B34F8021B404601377C
:10391000FEF7B6FABE42F5DC08B0BDE8F081064914
:103920002046FFF734FAF7E7044908B0BDE8F04154
:10393000FFF72DBA80660020F0EE050808EF0508B5
:10394000D6EE050813B504460846019140F0ACFEDA
:10395000024678B10F2804D101990A4843F028F9AA
:1039600040B1084B084A0949204602B0BDE8104062
:10397000FFF70DBA0349064802B0BDE81040FEF754
:103980007FBA00BF6CEB05080FEF05081AEF0508BA
:1039900044EF050813B504460846019140F084FE43
:1039A0000199024670B1042803D10A4843F000F996
:1039B00040B1084B084A0949204602B0BDE8104012
:1039C000FFF7E5B90349064802B0BDE81040FEF72D
:1039D00057BA00BF7CEB050852EF05081AEF05083F
:1039E00062EF05082DE9F04306469BB008460C46F9
:1039F00040F05AFE002705461C22394602A80197CE
:103A000043F099F82DB3402D08D03A4940232A4677
:103A100030461BB0BDE8F043FFF7B9B90DF104081B
:103A200004F1400902222146684643F0D5F80023FC
:103A3000102209A968468DF80270FBF7EBF8099B84
:103A40000DF10202934221D10234A14508F8010B85
:103A5000E8D100213D220AA8099109AC43F06BF896
:103A6000002D39D0244B1D78C5B12449202201A84E
:103A700043F037F890B120462049FCF723FF204A55
:103A8000204923463046FFF782F904E01A781E49A0
:103A90003046FFF77CF91BB0BDE8F0831B4E33784E
:103AA000D3B9CDB9154A01AD2B4603CBA342106063
:103AB00051601D4602F10802F6D1012320460F494C
:103AC00086F8D03CFCF7FEFE1148FDF7FDFA1148E0
:103AD0002146FEF7D5F9DEE70C4B93F8D03C1BB935
:103AE000054B1B78002BF2D004492046FCF7EAFE78
:103AF000EDE700BF75EF0508863A0020883A002000
:103B0000B3EF05081AEF050897EF05085CE50020FC
:103B1000BDEF0508CCEF050808B50A4B93F8D42C87
:103B2000032A0AD193F8D53C092B06D127F06AFD68
:103B3000BDE808400448FEF7A3B9BDE808400349C2
:103B4000FFF725B95CE50020D9EF0508E4EF05088B
:103B50002DE9F04F074691B08248834D0E46FEF79F
:103B60008FF98249C5F8F4DC002385F8F83C062279
:103B7000012309783046402485F8F94C06F008FB0B
:103B80000A2008F089FA95F8F83C0C2BDAB240F2DA
:103B9000E4809DF80C50FE2D36D0FF2D0BBF152470
:103BA0000F2401260026944240F0D780611EC9B23E
:103BB000684636F0C7FF04F140030DEB030414F828
:103BC000413C834240F0C48006F1FF389DF80D303F
:103BD00067485FFA88F8B8F1010F8DBF03F01F073F
:103BE0009DF80E709DF80F4061378CBF5C091D4633
:103BF000FDF72CFA022E64D0013C042C5FD8DFE8DC
:103C000004F005585A5E5C000226CCE75948DFF8FC
:103C1000C091DFF8C0B1FDF751FA5748FDF716FA29
:103C20006C464FF0000A14F8011B48460AF1010ADD
:103C3000FDF7E2F9BAF10C0F49D1FDF727FA022E90
:103C40004FD06422B5FBF2F102FB11524B483B46C8
:103C5000D2B2C9B2FEF714F9B8F1010F71D8484ACF
:103C6000484B9DF810104848484D002914BF114694
:103C70001946FEF705F99DF81110454B45480029F6
:103C800014BF19462946FEF7FBF8022E59D19DF8BC
:103C900012404148FDF7DAF94CB3FF2C37D00A2225
:103CA000B4FBF2F102FB11423C48D2B2FEF7E8F855
:103CB00020E03B48ABE73B48A9E73B48A7E73B4848
:103CC000A5E700238DF83F300DF11F009FE7384B2B
:103CD00003FB0AF2B2F1553FA5D85846FDF7B6F9F5
:103CE000A1E734483A462946FEF7CAF8B7E728461E
:103CF000FDF7E4F99DF813402F48FDF7A7F944B10B
:103D0000FF2C21D02D482146FEF7BAF804E02C48BC
:103D1000EEE71E48FDF7D2F91C4E294FDFF8708000
:103D20000DF11305002415F8013F7BB1FF2B0CBFEB
:103D30003A464246214623480134FEF7A1F8042CB6
:103D4000F1D111B0BDE8F08F1D48E3E73246F1E74D
:103D50001D493846FFF71BF8F3E71C48FDF7AEF99D
:103D6000EFE700BF13F005085CE50020805D002050
:103D700024F005082FF0050855F0050867F0050840
:103D8000F3EF0508FCEF05089EF0050803F00508B1
:103D90004CFC0508B5F00508BCF00508D0F0050896
:103DA00036F005083EF0050846F0050839E7050835
:103DB000ABAAAAAA83F00508D8F00508ECE5050827
:103DC00007F00508E8F00508F3F0050803F1050819
:103DD00096E305084A6206082DE9F74F05460846AE
:103DE000FCF7AAFB0B46044618B9324A92F8FA7C53
:103DF0002FB9284603B0BDE8F04FFEF7DFBF2E49CC
:103E0000DFF8C080DFF8C090DFF8C0A001AA184634
:103E100042F064FE264610B904F002FB07E04EB9FA
:103E2000014628463AF020FD421C04461AD103B050
:103E3000BDE8F08FFBF73CFA2F28834634D80FB14A
:103E400004F0E0FABBF1060F13D01C4901230978F6
:103E50005FFA8BF2E0B206F09BF959464846FEF74E
:103E60000FF80027144901AA0020013642F036FE5F
:103E7000D1E7DAF800301B0112D5FF2C0ED0E1B2E9
:103E80002846FFF765FEE8E72846FFF761FE0137A1
:103E90000A4B1A78F9B28A42F6D8DEE70027F7E72C
:103EA0000748FDF70BF9D8E72F2241462846FEF7D1
:103EB0006EFFD7E75CE5002081E40508805D002007
:103EC000E4EF05081DF105080CF10508885C0020E9
:103ED000F8B507460846FCF72FFBD0B1204BD3F8C6
:103EE0008C600136304608F06DFD34460546F0B969
:103EF0000134192CA8BF0024204608F063FD0546B4
:103F0000A8B9B442F4D138461649BDE8F840FEF7E6
:103F10003EBF0846FBF7CCF9044608F053FD0546C2
:103F200028B921461048BDE8F840FDF7A9BF0C4B61
:103F3000C3F88C4009F09AF80C4821462A46FDF750
:103F40009FFF182C9DBF0A480C2101FB0400002094
:103F5000BDE8F84098BF90F86C0509F0B9B800BF0B
:103F6000680400203DF1050851F1050867F10508D6
:103F70008887050838B5124D04460846FCF7DCFA78
:103F800060B1104B104893F900104B1C0ABF0F4B47
:103F9000C9B21978BDE83840FDF772BF0846FBF793
:103FA00087F9032804D8C0B2FCF7DCF92946E4E716
:103FB00020460749BDE838400322FEF7E8BE00BFAF
:103FC000A5F305086804002080F10508FC5A0020CC
:103FD00090F10508F0B5032985B005460C46164654
:103FE00014D80B4F3970FDF751F80A492846FFF7EE
:103FF000C1FF0949224601A8FAF780FC01AB32460D
:1040000008212846FEF73EFEFF233B7005B0F0BDB9
:1040100068040020A5F3050880F1050838B5124DA5
:1040200004460846FCF788FA60B1104B104893F933
:1040300001104B1C0ABF0F4BC9B25978BDE838407C
:10404000FDF71EBF0846FBF733F9032804D8C0B2BA
:1040500013F004FE2946E4E720460749BDE838404E
:104060000322FEF794BE00BFA5F3050868040020F4
:104070007CF10508FC5A00208BF10508F0B50329F6
:1040800085B005460C46164614D80B4F7970FCF7E0
:10409000FDFF0A492846FFF7C1FF09492246684645
:1040A000FAF72CFC6B46324610212846FEF7EAFD53
:1040B000FF237B7005B0F0BD68040020A5F3050860
:1040C0007CF10508F8B5174C237A054663B1637A8D
:1040D00053B11549FEF75BFE28461449FEF757FE1B
:1040E000002020726072F8BD94F8D05CBDB1104B16
:1040F00018780028F7D10F4B0F4A03F12007164616
:1041000018685968144603C40833BB422246F7D1E5
:10411000012386F83B3008F0BDFB2846E3E7012089
:10412000E1E700BF5CE50020ABF10508E2F105081E
:10413000863A0020883A00205471002008B5FFF725
:10414000C1FF50B1054B01229A73FCF7BDF804483A
:10415000FCF7BAFF0020FCF781FF08BDFC5A0020E5
:1041600000F205082DE9F74F064601AA08462E4938
:10417000DFF8C480DFF8C490DFF8ACA042F0AEFCFA
:104180004FF0000B04465D4601270CBBBBF1000F4E
:1041900026D1264C002D42D025482946FDF770FE39
:1041A00023780BB9FCF7D0F9F9F7B4FF0023637259
:1041B000FCF7ECFE15B12846FCF767F99FB13046D5
:1041C000FFF780FF78B1FCF77FF80020FCF746FF8F
:1041D000BBF1000F0AD02046FBF76AF885B2C5B9DB
:1041E0003046FEF7EBFD03B0BDE8F08F41462046B8
:1041F000FAF7F8FC80B949462046FAF7F3FC0028A4
:10420000EED05F4601AA5146002042F067FC04460A
:10421000BBE74FF0000BF5E74FF0010BF2E7054865
:10422000FCF752FFC0E700BF81E405085CE5002011
:1042300010F2050833F2050807F20508E1FB05084E
:104240002DE9F74F444BDFF82CA11A785B788AF8F8
:104250000130424B8AF800201B78054688460BB98E
:10426000FCF772F9F9F756FF00263D4CB1460D23D5
:104270003B4A7343414652F803B05846FAF7B2FC42
:10428000002841D0B9F1000F01D0FCF7FFFE3548FE
:104290005946FCF7B1FE002221462846FEF768FD8C
:1042A000FCF7F4FE237903F01803082B46D0102BFB
:1042B00049D02046FDF7F3FD294A0D2303FB0623D1
:1042C000B3F80900F9F7EEFE0746D8B12046FCF72F
:1042D000FDF8D7E902210090024401442046FCF792
:1042E0008DF878B9019059461F48FCF785FE019A70
:1042F000B9681346009A28460A442146FEF7D0FBC7
:10430000FCF7C4FE09F10109013640F23A239E424E
:1043100004F10D04ABD10020FCF7B7F8FF238AF8B5
:1043200000308AF80130B9F1000F11D10F4942462F
:10433000284603B0BDE8F04FFEF729BD0C492846DA
:10434000FFF718FEB5E70A492846FFF767FEB0E712
:1043500003B0BDE8F08F00BFFC5A00205CE50020F0
:104360003898050803EE050849F2050859F20508D2
:10437000A5F305086804002038B51A4B5B79012BBA
:1043800005462AD1184B1B683BB30846FCF7D4F806
:1043900070B90846FAF78CFF00F54373B3F5C36FA5
:1043A000044608D928461149BDE83840FEF7EFBC5D
:1043B0000F4BB3F9FC4C0F48FCF786FE0E48FCF798
:1043C00045FEFCF7FDFD0A4BD3F8880008F006FE19
:1043D00005F016FF2046F9F73BFCBDE838400748DA
:1043E000FCF772BE6C3A0020DC2A00206AF2050855
:1043F0005CE5002082F2050872E40508A2F20508D7
:104400002DE9F84F1F4DDFF88490DFF884A00646B1
:104410000C4637274FF000082046FCF78DF8D5F8FA
:1044200000B048B921465846FAF7DCFB20B9686865
:104430002146FAF7D7FB80B15846FCF707FE6968BA
:1044400011B15046FCF7D8FDA96811B14846FCF7F8
:10445000D3FDFCF71BFE4FF00108013F05F11005ED
:10446000DAD12046FCF768F848B9B8F1000F06D158
:10447000224630460449BDE8F84FFEF788BCBDE847
:10448000F88F00BF208E0508DBF20508D5F205087D
:10449000CFF205082DE9F04F024691B00846FCF72F
:1044A0004BF80B46044628B1104611B0BDE8F04F5A
:1044B000FEF788BC4FF0FF32CDE90820A74ADFF8AD
:1044C000E482D2F88820DFF8E09292F83810DFF822
:1044D000DCA2CDE90C10CDE90E02CDE90A00A0491D
:1044E00007AA184642F0FAFA2746054604942646DB
:1044F0004DB9089A0C9FBA4262D19A48FDF7C0FCA8
:1045000011B0BDE8F08F062F12D8DFE807F0041EC7
:104510002328454C510051462846FAF763FB78B1F1
:104520004FF4806008F0A4FC90F904300893012453
:104530008B4907AA002042F0D1FA01370546D7E798
:104540002846FAF7B5FE0890F2E72846FAF7B0FEDB
:104550000990EDE72846FCF752F90A90E8E728466B
:1045600040F0A2F84146024605902846FAF716FBAD
:1045700018B3059A49462846FAF710FB0646002864
:10458000D6D02846FAF794FE04280646D0D901462C
:104590007548FDF775FCB3E72846FAF789FE002356
:1045A0000C900F93C4E72846FAF782FE0D90BFE700
:1045B0002846FCF724F90E90BAE701230493B7E7E5
:1045C000DFF8EC8151B2434613F9010B884208D061
:1045D0000135092DF8D1002164480131FDF750FC67
:1045E0008EE763480121FDF74BFC7AB2002318F9EE
:1045F000011B8A4200F00D810133092BF7D13A46A5
:104600000121E9E7A7F1140253425341059308AD94
:10461000002303F10108EB68A3BB95F900B05846ED
:1046200008F0EEFBD5F804A020B1D0F80090B9F165
:10463000000F5ED1BAF1000F19D14FF461436B60E6
:104640004FF0010AAB680BB90323AB600023D5F828
:10465000049002932A7A1946CDE9009258461A46E8
:1046600008F063FCE86028B94248414691E74FF002
:10467000000AE7E74A464146BAF1000F37D03E4804
:10468000FCF7BAFCB8F1020F05F110054FF0010379
:10469000BFD1059BDDF83C800B9D53B13748FCF73B
:1046A0000DFDD8F800301B6A1BB135492A4640463B
:1046B0009847049B002B4ED03249334B142F18BF20
:1046C00019463248FDF7DCFB142F09D1049B03B9CE
:1046D00036B12B68DB691BB12D4932462846984715
:1046E000002C67D10022414628463AF05FF929485C
:1046F000C6E7C5F80C90BAF1000F25D02648414610
:104700005246FCF779FC5146484602F007FAD5F8C4
:1047100008A0BAF1000F0FD099F8042092450BD0F1
:104720001E4853464146FCF767FCD9F800305FFA53
:104730008AF19B6948469847D9F82C30002BA1D0C4
:104740000023C9F82C309DE7D9F8082014484146C9
:10475000FCF752FCDBE70C49B3E700BF5CE5002047
:1047600081E4050825F305080DF3050869F405083B
:104770003EF305084AF3050866F305081DF405082D
:104780001D6B0108EFF20508A5F3050846F40508BE
:10479000E30701088AF30508A6F30508F8F30508FE
:1047A000D3F3050807F30508C0F40508FCF2050873
:1047B0000880050803F026FE052007F06DFC1A4F5F
:1047C000DFF86C9000264FF0030A99F80030B342EE
:1047D00088D917F801BBBBF1000F15D0584607F078
:1047E000F3FE044680B1584603F05EFD08B1A0F820
:1047F00006A009210490F6F795FDA379049813F01B
:10480000010F03D0F6F7A8FB0136DEE7F6F79EFBB3
:10481000FAE706483A460221FDF732FB099B002BD6
:104820003FF4F0AE0023F1E6843C00203EF305089F
:10483000805D00202DE9F74FDFF89C91DFF89C8127
:1048400005460F463846FBF777FE064640B1002383
:104850005A491A46012003B0BDE8F04FFCF7B4BF37
:10486000052249463846FAF799F960B9534B0022B8
:104870001A601A611A621A631A641A651A661A674C
:1048800003B0BDE8F08F4E4904223846FAF786F9A6
:1048900004463846002C44D1FBF75EFF83460028CF
:1048A000EED03FF001FF474BC2B253F804ABBAF170
:1048B000000F07D144493A46284603B0BDE8F04FFF
:1048C000FEF765BA51465846CDE90023FAF766F976
:1048D0000134DDE9002306460028E6D1374A0346C5
:1048E000174600210133082B42F8101BFAD108EBC0
:1048F000C403D3F804C0BCF1000F03D018F834E0AF
:10490000764505DB3148324F5146FDF7B9FA99E754
:104910000CEB06130FCB07EB061484E80F000136EF
:10492000EEE7FAF7C5FC072804463DD83846FBF702
:1049300013FF064658B3FAF723FE204B03EB04138C
:1049400083ED000A01273046FBF706FF064638B123
:10495000FAF716FE194B03EB041383ED010A013736
:104960003046FBF7F9FE064638B1FAF709FE134B5D
:1049700003EB041383ED020A01373046FBF7ECFE2C
:1049800038B9284603B0BDE8F04FFEF71BBA07461A
:10499000D9E7FAF7F5FD0948032F00EB041484ED7D
:1049A000030A3FF454AFECE70A490723324628468E
:1049B00003B0BDE8F04FFEF777BB00BF40650020B5
:1049C0007BF405089091050859F2050880F4050864
:1049D000A5F3050876EE050807F30508187D050818
:1049E0002DE9F74F834608460D463FF05DFE364FF2
:1049F0000446D7F80090B8B93448354D354FFCF728
:104A000025FB012655F8041B49B106FA04F313EA05
:104A1000090F02D03846FCF7EFFA0134F2E703B091
:104A2000BDE8F04FFCF732BB02462B492846FAF7A7
:104A3000B5F878B92948264C294DFCF707FB54F8FE
:104A4000041B0029EBD00B78002BF8D02846FCF78C
:104A5000D3FAF4E72B782D2B1D4B03BF013504F15E
:104A6000FF344FF0010A4FF0000A002653F8048B80
:104A7000B8F1000F07D11B492A46584603B0BDE8DC
:104A8000F04FFEF784B92246414628460193FAF7D3
:104A900085F8019BB0B90123B340BAF1000F0CD0E7
:104AA00029EA030310483B60FCF7D0FA0C48414662
:104AB00003B0BDE8F04FFDF7E3B949EA03030B4843
:104AC0003B60F1E70136D1E7845C00208AF40508F9
:104AD000FC91050894F405083DEA050898F40508DA
:104AE000B4E9050859F20508A3F40508ACF4050873
:104AF0002DE9F74F814608460E46174698463FF087
:104B0000D3FD0446E8B94048404DFCF775FA20460D
:104B100007F046FF3B68184206D0204607F052FFD8
:104B200001462846FCF768FA0134182CEFD13B689F
:104B300013B93748FCF78AFA03B0BDE8F04FFCF729
:104B4000A5BA024633493046FAF728F80546A8B90F
:104B50003148FCF77BFA2C46304D204607F020FF09
:104B600010EA080F06D0204607F02CFF0146284621
:104B7000FCF742FA0134192CEFD1DDE733782D2B05
:104B800048F0807303BF013604F1FF34012500258E
:104B90004FF0000A0193504607F014FF2246834667
:104BA00001463046F9F7FAFF00BB504607F0F8FE21
:104BB000019B03421AD08DB1BAF1180F1CBF3B689C
:104BC00040EA03081648C7F80080FCF73FFA13488C
:104BD000594603B0BDE8F04FFDF752B9BAF1180FCE
:104BE0001CBF3D6885433D600E48EEE70AF1010AAF
:104BF000BAF1190FCFD10C493246484603B0BDE88F
:104C0000F04FFEF7C4B800BFB4F40508B3E90508D7
:104C1000BEF405083DEA050898F40508B4E905085E
:104C2000A3F40508ACF4050859F20508014A40F25E
:104C300002235DE77C5D0020014A6FF07F4357E768
:104C4000745D002010B5044608460B46FBF774FC63
:104C500028B9094903221846F9F7A0FF28B90748DF
:104C6000FCF732FA0120FCF7F9F920460449BDE8C7
:104C70001040FEF78CB800BFC5F40508C9F405085C
:104C8000EBF405082DE9F84FDFF8A880DFF88890ED
:104C9000DFF8A4A007460C4620463FF005FD064677
:104CA00058B91D4B1D481A781D4B03EB8203D3F8EE
:104CB000041ABDE8F84FFDF7E3B802464146204626
:104CC000F9F76CFF60B1DFF864B000255BF8041BF6
:104CD000B1B9224638461349BDE8F84FFEF757B838
:104CE0001148124C124DFCF7B1F954F8041B19B1DC
:104CF0002846FCF781F9F8E7BDE8F84FFCF7C6B99C
:104D000032462046F9F74AFF01350028DED189F8FE
:104D100000505446C0E700BF145B0020FAF40508B9
:104D20008887050859F2050898F405089091050848
:104D3000B4E905083DEA0508A5F3050838B50D46B0
:104D40000446174905222846F9F728FF50B9154BA4
:104D50001A7A12B9012119725A72BDE83840124804
:104D6000FCF7ACB9114903222846F9F717FF80B9BF
:104D70000C4D2B7A4BB16B7A3BB10D492046FEF7B7
:104D800006F800232B726B7238BD0A48FCF796F9BF
:104D9000F7E720460849BDE83840FDF7F8BF00BFF7
:104DA000AAFB05085CE5002004F50508F5FC0508EC
:104DB000ABF105081AF50508EBF405082DE9F341F8
:104DC00005460846FBF7B8FB0C46074640B10023F2
:104DD00034491A46012002B0BDE8F041FCF792BD0B
:104DE00031492046F9F7B6FE034670B92D4A4FF413
:104DF0007A704FF4FA610133042B1080518002F174
:104E00000402F8D102B0BDE8F0812046FAF750FA6A
:104E10000328064641D82046FBF79EFC074670B1A2
:104E2000FAF746FA4FF0010804463846FBF794FCBF
:104E300048B9284602B0BDE8F041FDF7C3BF40F2D3
:104E4000EE248046F1E7FAF733FAB8F1000FF0D01C
:104E5000A4F2EE2240F2DC539A4203D8A0F2EE22F2
:104E60009A420AD9114940F6CA0340F2EE22284676
:104E700002B0BDE8F041FEF717B90D4B0D4A03EB48
:104E800086030021A3F8004DA3F8020DCDE90040F0
:104E900033460846FCF7FEF8B4E7074903233A46D1
:104EA000E5E700BF5CF2002007F305082EF50508D2
:104EB0005CE5002037E50508B5EE05082DE9F04F63
:104EC0000F4689B0144600211A460646FCF708F939
:104ED0000546002C00F0DB8022783B789A4218BF10
:104EE0000121024608BF002130460CBF4FF00108E7
:104EF0004FF00008FCF7F4F823789B4A054641463A
:104F00003046FCF7D5FA3B78974A41463046FCF7E5
:104F1000C1F8002C00F0BD8062787B789A4218BFFF
:104F200001212A4608BF002130460CBF4FF001087E
:104F30004FF00008FCF7D4F863788C4A05464146E8
:104F40003046FCF7B5FA7B78884A41463046FCF794
:104F5000A1F807F1CA030493822304F1CA0B059355
:104F60004FF002094FF0000A3B78534500F393805D
:104F7000002C00F0F38097F8EA3094F8EA209A4287
:104F800018BF01212A4608BF002130460CBF4FF050
:104F900001084FF00008FCF7A3F894F8EA30744ACF
:104FA000054641463046FCF783FA97F8EA30704AE6
:104FB00041463046FCF76EF807F1EC09002C00F092
:104FC000CF8004F1EC034A4604F1FC014FF00108E4
:104FD0009A4633F802CB32F8020B844518BF4FF0E3
:104FE00000088B42F5D188F001012A46C9B230464B
:104FF000FCF776F8082105465046FBF743FC5D4A6E
:10500000034641463046FCF753FA97F8EA10484603
:10501000FBF738FC574A034641463046FCF73AF85E
:10502000002C00F09F804FF0FC094FF0010807EBC7
:10503000090104EB0900F9F78DFD09F104090028C5
:1050400018BF4FF00008B9F58E7FF0D188F001014C
:105050002A46C9B23046FCF743F8082104F1FC00A7
:10506000FBF756FC444A034641463046FCF720FA1B
:1050700097F8EA1007F1FC00FBF74AFC3E4A0346AA
:105080004146304609B0BDE8F04FFCF703B8A046F2
:1050900039E7A04657E7059B3B440693002C5BD0BD
:1050A000059B0698234419460793F9F753FD049B83
:1050B0001A789BF800309A4206BFB0FA80F84FEA9F
:1050C00058184FF000084B4609F11002F85AE15AFF
:1050D0000233884218BF4FF000089342F6D188F09F
:1050E00001012A46C9B23046FBF7FAFF627804EBA9
:1050F000090105469BF81800FBF796FB02909BF808
:1051000000300193079B00931C4A0AF101034146BA
:105110003046FCF7CDF9049B7A78187E079307EBAD
:105120000901FBF781FB079B049A02901B7801930E
:105130000132069B04920AF1010A00930F4A53467A
:1051400041463046FBF7A6FF059B09330BF1010BE7
:1051500009F11009059307E7A046DCE7A04624E71C
:10516000A04652E7A04683E73CF505084EF5050842
:105170007CF5050894F50508ABF5050863F5050809
:1051800038B50C46054616492046F9F7E3FC30B918
:10519000FBF7FCFE1348BDE83840FBF78FBF124910
:1051A0002046F9F7D7FCA8B9104A82F8860082F8A1
:1051B0008E0082F82A0182F8320182F8CE0182F84C
:1051C000D60182F8720282F87A02094A82F8210036
:1051D0000848E0E72846BDE83840FDF7EFBD00BFCE
:1051E000C2F50508C8F50508E3F505085053002089
:1051F000E0550020EBF505082DE9F74F0746084676
:105200000E463FF051FA044620B1012826D13278EB
:105210002A2A23D1B448B54EDFF8EC92FBF74EFFB3
:105220000025B2464FF00D0B40F23A280BFB05F378
:1052300048465AF80310FBF7DFFE221E18BF012272
:10524000314638460135FDF793FDFBF71FFF454515
:1052500006F10D06EAD103B0BDE8F08F3D213046DE
:1052600041F080FC002800F0378101460A4611F821
:10527000014D202CFAD0921B0130814610F8011B01
:105280002029FAD0DFF864B25FFA82FA4FF0000802
:105290000D2303FB08F10BEB010452465BF80110F0
:1052A00000913046F9F77AFC0546002857D100995D
:1052B00008463FF0F9F9824551D1267906F0E00120
:1052C000402900F0CC800ED8002956D0202900F0CB
:1052D0009E8038468649FDF75AFD204603B0BDE85A
:1052E000F04FFCF7DCBD602900F092808029F0D1FE
:1052F00048463FF0D9F9E379A679DB0705460CD596
:105300002046FBF7D1F90378014633B12A464846D7
:1053100041F04EFC002840F0D980002D00F0D680EE
:10532000AE42C0F0D3800D2303FB08B3204693F8B0
:1053300005A0FBF7B9F93246002141F0FCFBAA4574
:105340002CD86C492A46484641F032FC30B32046FE
:10535000FBF7AAF92A46494641F08AFB1EE008F10C
:10536000010840F23A23984592D1634932463846C3
:1053700003B0BDE8F04FFDF70ABD06F00703042BAC
:105380001CD10B460A224846F9F744FCD4F80530F4
:10539000834201469DD32046FBF79AF90D2303FB78
:1053A00008F856485BF80810FBF726FE0022214655
:1053B000384603B0BDE8F04FFDF7DABC052B0FD13E
:1053C00001230A224846F9F725FCD4F80530834228
:1053D0000146FFF67EAF5B4283423FF77AAFDAE7E2
:1053E0004846F9F765FFB4F80550B4F8071016F011
:1053F000050FAAB218BF2AB28BB218BF0BB29042E7
:10540000FFF667AF98423FF764AF0146C3E765799F
:105410003B4A02EBC505002695F8A4220092B2464D
:105420003346009AB24202D9BAF1000F03D0002BE2
:105430003FF44FAFB2E7D5F8A01251F8260060B1A3
:1054400049460193F9F786FB019B30B93146204666
:105450004FF0010AFBF73CF953460136E1E7637967
:10546000009306F00706013E009BAB4296DD4846DE
:10547000814610F8013B202BFAD02046FBF714F9A7
:105480008246042E04D8DFE806F0031010161F0031
:105490004846F9F70DFF0AF8050048462C2141F06F
:1054A00061FB013500F10109DEE74846F9F700FF2D
:1054B0002AF81500F1E700230A2200214846F9F7EF
:1054C000A9FB4AF82500E8E70123F5E70D49324634
:1054D0003846FDF75CFCFCE63146384603B0BDE8D3
:1054E000F04FFEF7ADBE00BF07F605083898050877
:1054F00055F605084A62060859F205084AF60508F5
:10550000888705081AF6050803EE050873B50E46E8
:1055100011490546F9F71EFB18B93070012002B099
:1055200070BD2C78602C8CBF613C413C072C10D89E
:10553000013501230A2201A92846F9F76BFB019BDB
:105540009D4206D00F2804D8013440EA0414347078
:10555000E4E70020E3E700BFD7E305082DE9F04FBB
:1055600080468BB008460D463FF09EF8024690B349
:10557000A5492846F9F712FB044660BBFBF786FDF8
:10558000A248A34DA34FA44EDFF8D482FBF796FDAB
:10559000142039F0A5F90721B4FBF1F1C1EBC102E8
:1055A000A21A013201313846FBF726FD2B7E6A7EB6
:1055B00006EB8303196A52B19848FCF761FC013489
:1055C0000E2C05F12405E6D10BB0BDE8F08F404666
:1055D000FCF756FCF3E72846914905AA41F07EFA0C
:1055E000054620B901464120FBF785FDECE78D49D2
:1055F000F9F7B0FA20B98C494046FDF7C8FBE3E75C
:105600008A4E0827002431682846F9F7A3FA0028B3
:1056100008BF3446013F06F11006F4D154B984495D
:105620002846F9F797FA28B182492A464046FDF7FD
:10563000AEFBC9E700207A498DF8130005AA41F0B6
:105640004DFA0546002C3AD080B1F9F731FE461EDE
:1056500009D4A37A9E4206DAE2684AB1012303FA2A
:1056600000F0104204D174492A46DFE7734DFAE78F
:10567000E088F8F717FD7249D0E90232097800296D
:1056800008BF1A46217A637A06FB0133002712F914
:1056900003A0039702EB030B614905AA002041F028
:1056A0001DFA8146A0BB6749012344B39BF9002042
:1056B0002046CDE900313146FBF7C4F984E768B1F3
:1056C0000DF11301FFF722FF28B19DF8136030465A
:1056D00002F0EAFD20B95C492A46A7E7574DFAE7F0
:1056E0003046F5F74BFD8246304606F02FFF03901B
:1056F000304606F069FFA34607462646CCE7CDE9CB
:1057000000319DF8130052463946FBF7E7F95BE795
:105710004449F9F71FFA054670BBACB14B4FF6B2DE
:1057200020796AB23146F5F7F3FC00283FF44CAF1C
:105730000288037800932946C2F303233846120BEC
:10574000FCF79EFB0135EBE7404C386879790E2D6C
:105750006AB23FF439AFF5F72DFD00283FF434AFBE
:105760000288037800932946C2F303232046120BD4
:10577000FCF786FB0135E8E735494846F9F7EAF9D1
:1057800000283ED04846F9F793FD054642B26CB179
:105790002079F1B2F5F7BCFCD8B9CDF800902268B9
:1057A0002C49731C4046FDF7F2FA0DE7EBB20D2BC6
:1057B0003868797909D99DF813302749CDF80090D8
:1057C0001A09403203F00F03ECE7F5F7F3FC002869
:1057D000F1D006AF39462846FBF788F808A95046AD
:1057E000FBF784F8554549D06DB2002C3AD08BF8C0
:1057F000005000972168194808AB721CFCF740FB69
:10580000E2E64FF0FF35E4E763F6050868F60508C1
:105810001C0100207EF6050888870508F3F70508B7
:1058200081E405083DEA050890F605086C040020AF
:10583000A4F60508A8F60508B7F60508A5F30508B7
:105840005CE5002095100108C7F60508D9F60508A3
:10585000C0F40508FBF605081EF7050846F705081D
:10586000B4E905089DF81320039B0D489D701109AC
:10587000009708AB02F00F024031BFE734B1216856
:10588000084808AB721CFCF7FBFA9DE69DF8132054
:105890000548110908AB02F00F024031F3E700BFE1
:1058A00069F7050891F70508ACF705082DE9F04FF1
:1058B00080468BB008460D463EF0F6FE024630B9F3
:1058C000014601200BB0BDE8F04FFBF71DBD029073
:1058D000AC492846F9F762F9029A30B9AA4940461C
:1058E0000BB0BDE8F04FFDF752BAA8492846F9F7CA
:1058F00055F90446002855D1FBF7C8FBA448A54F2D
:10590000DFF8D0B2DFF8D082FBF7D8FB172038F0F1
:10591000E7FF17F9016B002E37D031465846DFF804
:105920009092DFF880A2FBF767FB01250023A9B264
:105930003046039306F080FE029006F00BFF0278DB
:10594000039BC2B11BB90390FBF7A0FB0398029B1A
:1059500041789A79037802F0020208EB8303B9B127
:1059600000911B6A8C48002A14BF4A4652462946B9
:10597000FCF786FA01230135052DD8D113B98748E4
:10598000FBF79CFB01340D2CC3D10BB0BDE8F08FAD
:105990001B6A8348002A14BF4A4652462946FCF730
:1059A0006FFAE7E700247F498DF8134005AA2846DF
:1059B00041F094F818B94046FDF700FAE5E70DF11B
:1059C0001301FFF7A3FD05460028F4D09DF81360EE
:1059D000304602F069FC20B973494046FDF7D7F91B
:1059E000D3E7DFF8F89123464FF0FF3403EB43028F
:1059F00012F8092096420BD0611C02D1002A08BF80
:105A00001C460133152BF1D1631C15D16749E4E71E
:105A10001C46644905AA002041F060F806460028AB
:105A200000F09C805749F9F795F818BB604E614F1C
:105A3000DFF8AC81044613E00025EAE7E97928683D
:105A40000291F5F709FC0246A8796B79029910F0EA
:105A5000020F14BF3046384600904046FCF710FA5B
:105A600001349DF81300214606F084FD0546002808
:105A7000E4D18AE7504902223046F9F78FF8074609
:105A8000002849D1B01CF9F713FC9DF813B0034668
:105A9000BA46013739465846029306F06BFD029B21
:105AA00038B94FEA1B12454900960BF00F034032FC
:105AB0003FE0C2799A42EBD1002D40D14FF0FF3642
:105AC000BAF1FF3F9DF8135008BF002504EB4404D2
:105AD00009EB04030AF101025A7009F80450FF228D
:105AE00008AC9A709DF8130022465146FBF73CF82B
:105AF00006AA31469DF81300FBF736F89DF81320EF
:105B0000B2454FEA121120D12D4806AB02F00F0228
:105B10004031FCF7B5F938E72A493046F9F71AF869
:105B200050B39DF81330284900961A09403203F00B
:105B30000F034046FDF72BF927E74FF0FF3A04EB40
:105B400044034B445E78013EBAE72048009406AB1C
:105B500002F00F024031FCF793F916E704EB44041E
:105B60001B4B0093A144024699F801109DF81300C5
:105B70000123FBF711F808E7002DDED14FF0FF36C7
:105B8000B246A3E73DEA050890F6050863F6050866
:105B9000C8F7050858E30508E8F7050809F80508F7
:105BA000FAF7050881E405080FF8050826F8050846
:105BB0003EE60508A5F305084FF80508BCF80508FA
:105BC00078F80508C0F4050852F8050896F80508A5
:105BD00095100108E1F7050888870508FC3B0020BF
:105BE0003AF805082DE9F04F2DED028B85B00646F9
:105BF00003AA0846914940F071FF074640B90146A3
:105C00004120FCF7B1F805B0BDEC028BBDE8F08F88
:105C10008B49DFF86082F8F79DFF044600283BD1EE
:105C20008848894D894FDFF85092FBF747FA1420D6
:105C300038F056FE2968AB79AA8801F13F4108EB9C
:105C4000830301F57E01B2FA82F2890A41311B6AAF
:105C5000C2F11F023846FBF7CFF9E97911B1484686
:105C6000FBF7CAF90134FBF711FA502C05F10805CE
:105C7000E0D1724903AA002040F030FF7449F8F7E0
:105C800069FF0028BFD130466D49FFF70FFE6C4910
:105C90003046FFF763FCB6E7002508F5C87919F828
:105CA000353008EB8303196A019108463EF0FCFC8D
:105CB000019902463846F8F771FF40B101351A2DB7
:105CC000EDD164493A463046FDF761F89BE75B4900
:105CD00003AA40F003FF08EBC5080746F9F7E8FA06
:105CE00098F8963104464FEAC50A2BBB002825DCFC
:105CF0003B78002B00F09E80D144B9F80200F8F701
:105D0000D1F9E3B2019399F8058099F80430019A2A
:105D1000846802FB038804EB08013846FFF7F6FBB2
:105D2000002800F0878014F808A0BAF1000F1CD1F9
:105D30004948FBF7C3F966E7002805DD012B1A4641
:105D400038BF0122A24208DA012B444938BF01239F
:105D500001223046FDF7A8F955E7384903AA00208B
:105D600040F0BCFE013C0746C2E7504602F09CFAF8
:105D7000814600285ED04FEA1A13403308EE103AED
:105D80000AF00F03DFF8F48008EE903A00270026AF
:105D9000B8F80200F8F786F998F8042098F805306A
:105DA00006FB02338268D15C514523D1BD4204D148
:105DB00001998E421ED00021D15418EE902A18EE7F
:105DC000101A27485FFA86FBFCB2FBF715F9594613
:105DD0002046FBF71EF9BD4209D12248FBF70CF91A
:105DE00020465946FBF715F91F48FBF705F91F48F0
:105DF000FBF764F998F80630012B06F1010638BF6D
:105E000001239E42C4DB01371A2F08F10808BED1D6
:105E1000D9F80010B9F80420154801F13F4101F507
:105E20007E01B2FA82F2890AC2F11F024131FCF707
:105E300027F8E8E63046FCF7C1FFE4E681E4050810
:105E400063F60508E8F80508EC37002026F9050890
:105E500031F9050835F9050851F9050876EE050808
:105E600063F90508C1E4050887F9050876510608B5
:105E700091F9050888870508EBE5050818890508E4
:105E80002DE9F04F8FB0044602AA0846B14940F010
:105E900025FE064640B903460246AF494120FFF7BA
:105EA0000DF80FB0BDE8F08FAC49F8F753FE074688
:105EB000F8B9A84902AA40F011FEF9F7F9F9082843
:105EC000054606D9A64908233A462046FDF7ECF8D0
:105ED000E7E7A14C2378834201DC2570E1E7064621
:105EE000314620462CF070FE23780136B342F7DCB1
:105EF000F3E79C493046F8F72DFE0546D0B99549A1
:105F000002AA40F0EBFDF9F7D3F90828064603D9B9
:105F1000954908232A46D8E78F4C6378834201DCF1
:105F20006670BEE728463146013538F0C5FC082DBD
:105F3000F8D1F5E78D493046F8F70CFE0746F0B981
:105F4000844902AA40F0CAFD0028AAD0F9F7B0F9A6
:105F50000828054603D9864908233A46B5E77E4C0A
:105F600094F8EA30834207DD014620462CF076FEA5
:105F7000294620462CF080FE84F8EA5091E77D49BE
:105F80003046F8F7E7FD054618BB734BDFF8C491C0
:105F900093F8EA7006AE01461022304640F0CBFD81
:105FA000B046BD4202AA80F20E814946002040F070
:105FB00095FD10B970493A460EE1F9F779F90135C6
:105FC00028F8020BEDE796E80F006C4C84E80F0010
:105FD00067E76B493046F8F7BDFD054600283BD121
:105FE0005D4B0DF1180893F8EA90464607464F4579
:105FF000584902AA4FF0000080F2F28040F06EFD96
:10600000014610B95F494A46E6E00322304640F0B7
:10601000E3FDB2464FF0000B30463EF045FB5845DD
:1060200002D801370436E2E79AF80000F8F78CFD51
:106030000BF1010B0AF8010BEEE753494A46CBE09E
:106040004146204603222CF0A7FD0135043408F117
:106050000408AF42F4D124E74C493046F8F77AFD02
:106060000546002840F0AC803B4F3A4997F8008045
:1060700002AA40F033FD00283FF413AFF9F718F9F6
:10608000461E01D4B04503DC4149434601221CE7CA
:10609000304902AA002040F021FD014600283FF4CB
:1060A00000AF4FF00008082203A8CDE903888DF85F
:1060B000148040F091FD0DF10C0903A83EF0F4FAB4
:1060C00040451CD8234902AA002040F007FD0028C3
:1060D0003FF4E7AE90F800A097F80190DFF8C4B065
:1060E0004FF000084D451B4902AA4FF000007EDA30
:1060F00040F0F4FC024658B926494A466CE099F84B
:106100000000F8F721FD08F1010809F8010BD4E7B8
:10611000B5B91378303B092B12D91F490192F8F712
:1061200019FD019A40B110465946F8F713FD019A3E
:10613000002839D019494FE04FF001084FF0FF35E2
:1061400010460192F9F7B4F80028019A2EDA1449A2
:1061500042E000BF81E405085C5F0020ADF905085E
:10616000B3F90508BEF90508C7F90508D5F905080A
:10617000E1F90508F3F90508E2FA0508486000208E
:106180001DFA050802FB050829FA050847FA050863
:106190004CFA050822FB050880E305085FFA0508AC
:1061A00094FA050858FA0508A846C7E70EAB03EBB2
:1061B0004503013523F8200C94E71B494A460BE0C0
:1061C0001A49324608E01A49002040F087FC0028AE
:1061D0003FF4F9AE17493A462046FCF7D8FD60E691
:1061E00040F07CFC00287FF428AF134C31E740F0EE
:1061F00075FC0028E1D106EBC6008230082203A915
:1062000038442CF0C9FC5046F8F79EFCBC196A00D3
:1062100084F8CA0007EB061006A9023040F028FCFB
:1062200084F8E2803DE600BFA9FA0508CCFA05082B
:1062300081E40508FFF90508586000202DE9F047C2
:10624000064686B008460C463EF02EFA082843D192
:10625000671E03AD0734AA46B946A84619F8010FD0
:10626000F8F772FCA1450AF8010BF7D10023DFF81B
:106270007C908DF8143017F8010FF8F765FCC1B267
:1062800005F8010B4846019140F06CFC20B10199E2
:10629000284640F067FC28B13046FCF78FFD06B079
:1062A000BDE8F087A742E6D10F49404625F022F924
:1062B0000D480E49082310F8012B11F8014B183234
:1062C0006A44013B02F80C4CF5D109488DF81430B2
:1062D00003A9FBF7D5FDE2E70028E9D0304606B078
:1062E000BDE8F047FCF76EBD1C5B0020101A0608E5
:1062F00047FB050873B50446084601913EF0D4F902
:106300000199054602462046F8F748FC70B9665DDB
:106310003046F8F709FC00B936B901352C4420465F
:1063200001340378202BFAD002B070BD0020FBE7C7
:106330002DE9F04F0C4695B03449054620461746E6
:10634000FFF7D8FF064600284FD131492046FFF716
:10635000D1FF064600284AD12E492046FFF7CAFF42
:106360000646002845D12C492046FFF7C3FF0646C4
:10637000002840D120462949FFF7BCFF00280646E7
:1063800012BF0824264601240FB144F0100424490A
:106390003046FFF7AFFF80B344F02004214E33783E
:1063A0000BB9FAF7D1F8F7F7B5FE14F0090F00F0C2
:1063B0001A831D48FAF788FE0020FCF797F914F4B9
:1063C000807307933CD11948FAF77EFE1848FAF714
:1063D00075FE04F01803182B05D11648FAF774FE61
:1063E0001548FAF76BFE01232BE00124CCE70224C9
:1063F000CAE70424C8E78124C6E710493046FFF7FE
:1064000079FF0028CAD044F48074C7E761FB05080F
:1064100068FB050870FB050876FB050831F90508DF
:106420002AF205085CE5002084FB05088CFB0508C2
:10643000A4FB0508B0FB0508D8FB05087FFB050891
:1064400000230693FAF722FE04F01003BC49BD486E
:106450000593FBF715FDBC49BC48FBF711FD04F49F
:106460008473082B07D1BA492846FBF7DFFDB849EA
:106470002846FDF7B7FA14F0800309930DD196F87A
:10648000103DB44A002B08BF0121B34B1CBF0021B3
:1064900013462046B14AFAF7FDFDB1492046FBF705
:1064A00063FCB0492046FAF72FFFAF492046FAF7C0
:1064B00022FEAE4BD3F800B0AD4B1B680493059B96
:1064C000002B40F0D281AB48FAF7FEFD059EAA4BA7
:1064D00008939946049BDFF840A36BEA03034FF04F
:1064E00000080A9359F8047B002F40F0C081049BF8
:1064F000DFF8289363EA0B0A089B53F8042B0392F6
:106500000893002A40F0DD819C4B9D4A9D4920461E
:10651000FBF76AF8099B002B40F07782DFF80093C5
:10652000DFF800A399F800209AF80030964E9A42BE
:1065300014BF01210021954A20460CBF4FF00108ED
:106540004FF00008FAF7CCFD9AF80030904A06EBBD
:1065500083030746D3F8043A41462046FAF7A8FFDA
:1065600099F800308A4A06EB83064146D6F8043A89
:10657000884E2046FAF78EFDD6ED007A864AF5EE73
:10658000407AF1EE10FA0CBF012100212046FAF703
:1065900081FD3B4632468149814F824E2046FBF7C2
:1065A00013F9814B01936FF07F4200923A68316892
:1065B0002046FBF783FB7D4B019340F202220092C1
:1065C000BA68B1682046FBF779FB059B002B40F0C9
:1065D000A7817748FAF778FD059A76487649DFF87B
:1065E00048C20826012710F8013B11F8018B03F17E
:1065F000500EEE440EF8208C1CF801EB0EF1500901
:10660000E94409F8108C2FB1A3EB0E0EDEF1000760
:1066100047EB0E07013EE6D187F0010120468DF8D9
:106620003860FAF75DFD654A8DF8486010AB394671
:106630002046FAF73DFF614A0CAB39462046FAF78F
:1066400029FD5F4A5F4B02F531712046FBF79EF949
:106650005D4A5E4B02F531712046FBF7E1F9584A7D
:106660005B4B02F531712046FBF722FA594B5A4A2F
:106670005A492046FAF734FF594A5A4B02F531710C
:106680002046FBF739F8584A584B02F5147120465A
:10669000FBF738F9564B574A57492046FEF70EFC90
:1066A000564B574A57492046FBF7A8FA059B002B43
:1066B00040F038815448FAF707FD544F4FF0000B73
:1066C000A7F52D7841460222384640F00AFA002804
:1066D00014BF01210021039A97F800A020460CBFA7
:1066E0004FF001094FF00009FAF7FAFCBAF1020F76
:1066F000039040F01A8198F801204FF0190A40F2F7
:10670000EE231AFB0232019298F80020404B9A5C6B
:1067100000925B463F4A49462046FAF7C9FE7A781E
:106720003B4B40F2EE211AFB021201923A789A5C3E
:1067300000925B46374A49462046FAF7ABFC75E0C3
:106740006CEB050844EF05087CEB050862EF0508D3
:10675000A5F305086CF200204A620608E8FB05086C
:10676000F5FB0508FFFB050817E805086C7300201A
:10677000845C00204EFB0508FC9105081CFC050804
:10678000545B0020BC6E00208887050823FC0508A8
:1067900029FC05084065002032FC050894710020A2
:1067A000745D0020F473002041FC050848FC0508D6
:1067B00056FB050884700020101A060847FB0508E0
:1067C000CCEF0020B0F405084CF0002054FC050884
:1067D0004FFC05085AFC0508E05C0020146B002003
:1067E000BCF000205EFC05085CF2002067FC050898
:1067F0006FFC05085C5F0020306F002078FC050806
:1068000098660020847200205AFB0508BCF4002022
:106810000C1C060898EE050805FC050811FC050887
:1068200088740020145B00201C5B00200BF1010B1E
:10683000BBF1120F07F1020708F102087FF442AF23
:10684000754B224600212846FCF71CFA230700F16D
:106850008280724E224631782846FDF7BBFB717864
:1068600022462846FDF70AFCB3E06D4E2FE63B7842
:1068700023B30A9A012303FA08F31A400CBF01213B
:1068800000210392204632460B93FAF729FC049B21
:1068900063EA0B020B9B1A4214BF012100213B4605
:1068A000524606462046FAF703FE039900393B4656
:1068B000524618BF01212046FAF7ECFB08F1010807
:1068C00010E6039B1B784BB3049B4FF0010808FABA
:1068D00007F813EA080F0BD06BEA030313EA080F5B
:1068E0004A46039B14BF012100212046FAF7E0FD30
:1068F0001BEA080F12D01AEA080832460CBF012121
:1069000000212046FAF7ECFBB8F100010646039B94
:106910004A4618BF01212046FAF7BCFB0137EBE5D8
:10692000404A5AE6404B0393C7E698F800203F4B95
:106930009A5C00925B4649463D4A2046FAF7B8FD0C
:106940003A783A4B9A5C00925B46394A494620466F
:10695000FAF7A0FB6AE70027F9B22246284601377A
:10696000FDF738FB042FF7D1DFF8B080314F98F8EE
:1069700000303B70079B33B92F48FAF7A5FB2F492E
:106980002846FDF7F7FAFF233B70F1B2224628466E
:106990000136FDF773FB042EF7D198F801307B70B8
:1069A000079BA3B92648FAF78FFB24492846FDF731
:1069B00035FB2448FAF788FB2348FAF747FBFF2307
:1069C0007B70002015B0BDE8F04FF9F75EBDFF23E6
:1069D0007B70069B002BF4D01C48FAF775FB1C4813
:1069E000FAF76CFBEDE7A10706D50C4B22461978A8
:1069F0002846FDF7EFFAE4E76207E2D5074B2246A7
:106A000059782846FDF73AFBDBE7034B224618216D
:106A10002846FCF737F9DCE761FB0508C474002061
:106A20004EFB050856FB05085AFB05080C1C06081A
:106A3000A8EE0508680400207CFC0508A5F30508FD
:106A40009FFC0508C6FC0508E3FB0508D9FC050802
:106A5000EFFC050800226BE4012269E410B58446CE
:106A60004FEA810E102312F4004F14BF0E240724A6
:106A70005200013BCCF8004092B2F444F3D100EB59
:106A800081128C01035142F82130122010BD00BF49
:106A900010B584464FEA810E0424130B03EB430325
:106AA00018331201013CCCF8003092B2F444F4D116
:106AB00000EB01130A01845043F82140062010BD69
:106AC000704700BF704700BF034B00EB400003EB73
:106AD000C000407C704700BF981D00200023182292
:106AE000027043708370C370704700BF704700BF6F
:106AF000704700BF0020704701207047704700BFFB
:106B0000704700BF704700BF704700BF9FED010A8C
:106B1000704700BF000000000020704703681B6939
:106B2000184730B5084B002293F900405D780119F1
:106B30000132CD729D780555082ADC788C7503F1F9
:106B40000403F1D130BD00BF2CB50508C36B33B1D0
:106B50005B68C26D9BB29A4205D3D01A7047D0E9E8
:106B600007239A42F9D2C0681044C01A704700BF88
:106B7000D0E909120369914238BFC9188A1A016C19
:106B800039B14968013B12FA81F2934204D9981A4B
:106B90007047013B981A704700207047036C13B18F
:106BA00090F86C007047D0E90903181AB0FA80F029
:106BB00040097047C26B10B4034662B1C26DC16830
:106BC0005C69881A013A205C5DF8044B08BF0A46EC
:106BD000C0B2DA657047006A5C69411C205CDC6801
:106BE000A14238BF0A46C0B25DF8044B1A62704732
:106BF000036F70B504460D460BB19847B8B1636A90
:106C0000A269D554636A2169226C01338B4228BF83
:106C10000023636232B3EFF31183502282F31288B0
:106C2000266C3268D20703D5DBB283F3118870BDBE
:106C3000726892B272B9D4E909518D421ED0A0692E
:106C40000844F06014D9691A89B27160A562002203
:106C500084F86C20326842F00102DBB2326083F3C8
:106C6000118870BDA26ED36843F08003D36070BDFD
:106C70002069411A89B27160A262E8E7012284F8B2
:106C80006C20D1E7036F03B118477047F8B590F84F
:106C90008530012B1CD0002A164619DD0269436A93
:106CA00005460F46D41AB442A869A8BF34463946EF
:106CB000184422463FF0DCFE6B6A2A692344361BE7
:106CC000B3FBF2F0002E02FB10336B622744E9DCC9
:106CD000F8BD00BF90F88530012B2BD0036C53B367
:106CE00070B4EFF31183502282F31288066C32687D
:106CF000D20704D5DBB283F3118870BC7047726889
:106D000092B272B9D0E909518D4220D084690C4405
:106D1000F46016D9691A89B271608562002280F820
:106D20006C20326842F00102DBB2326083F31188DA
:106D300070BC70477047826ED36843F08003D360A5
:106D400070470469611A89B271608262E6E70122C4
:106D500080F86C20CEE700BF70B5094C236873B192
:106D60000546002606E099681A681E732160904760
:106D7000236823B15A68AA1A002A1846F3DA70BDAC
:106D800028F5002070B5204C2378012B00D070BD71
:106D90001E4B1B68002BFAD01D4D2B6828465B68E4
:106DA00098470028F3D01B4B1B4E1A6833889288F3
:106DB0009A4219D31949096800224968EA622A6887
:106DC00003FB01F12846D3689847154A3388526877
:106DD00001333380002ADAD0116893884A6913425C
:106DE00018BF1B048B6170BD0D4B5B6800222270C5
:106DF000002BCCD00B499A8809781B68890748BFBB
:106E000012049A6170BD00BF604D0020DC2A002092
:106E1000E02A0020584D00205E4D0020504D0020FB
:106E2000802A00208C2A0020914B1B68D90600D4B0
:106E30007047F0B58F4C2DED028B636987B00BB1B5
:106E4000201D9847A369002B70D08B4894ED168ABB
:106E50009847C21C054675D0002877DA431C00F01D
:106E6000F9806FF001022262844E3368EB1A03FB53
:106E700003F34FF609218B42DCBF8149A1FB0313C9
:106E800094F8751004EB4100D4BF43F3CF034FF4E3
:106E9000C853A0F878304B1CDBB2052B84F8753052
:106EA00000F0888094F882303560002B00F08E80EE
:106EB000B4F87A00B4F87830B4F87C1094F82C6008
:106EC0000344B4F87E000B44B4F8801003440B4430
:106ED0001BB2B3F5FA4F1946A8BF4FF4FA4121EAA5
:106EE000E171A1863EB9002A05DDB3F5167F78DB96
:106EF000012684F82C60634B18781B2844D01C288A
:106F000037D1676A604D236B2A80002F6E80AB807B
:106F10002DDD002A2BDDB1F5167F28DA002E00F0DA
:106F2000A1809342D4BF0023012321E055494FF0B3
:106F3000FF33087823621A461B28636202D1524D40
:106F40006A80AB8007B0BDEC028BF0BDE36D4F49AA
:106F500004EB830201330968A162052B1066E36527
:106F60004DD094F87430002B4ED102467BE70023BD
:106F7000EB80D4ED077AB4EEE78AF1EE10FA0CD587
:106F80004FF0FF336362DDE7D4ED077A3E4DB4EE98
:106F9000E78AF1EE10FAE98014D4002A64DB07EEE8
:106FA000902AF8EEE77A67EE887AFDEEE77A17EE38
:106FB000903AC1E7002384F87530012384F88230C9
:106FC000356075E74FF0FF336362B9E794F82C60E2
:106FD0004FF6FF73A3864FF0FF31002E8BD1002AAE
:106FE00089DD236B93423BDA294802EB8203C3EB32
:106FF0000313A0FB03035B09236300267BE7002246
:107000000123E26584F87430224F0FCF01AE0FC622
:10701000029A3B683360904202DC134602461846EF
:10702000DDE90413994202DC1E460B4631468142DB
:10703000A8BF01469A42B8BF1A46039B8B4202DBA7
:107040000846194603468A42A8BF0A469A42B8BF74
:107050001A4608E70D4B20621B68A362024603E74D
:10706000002648E7012383E74FF0FF3364E700BFC2
:10707000F8E6002028F500202CF50020F804002078
:10708000CDCCCCCC732B0020742B0020782A002090
:107090001F85EB5188F50020704700BFF6F7FCBC58
:1070A00010B504463EF048FF81B22046BDE81040CE
:1070B000F6F7F2BCF8B5C64B1D6815F004072DEDC8
:1070C000048B40F00081DFEDC38AC34C15F020052E
:1070D00005D094F8005115F0020540F0908094F826
:1070E00038319FEDBE8A13F0010340F0AC8094F874
:1070F0003921002A7ED1D4ED4F7A9FEDB97ADFEDA8
:10710000B96A67EE877A94ED517AE8EEA67A38EE9E
:10711000C77AC4ED4F7A84ED507A65B194F84C216A
:10712000D4F80431C4F8483101218A4284F83A1174
:1071300018BFC4F84031AC4B1E780E2E00F007810A
:10714000DFEDA47A002794ED577A94ED586A77EE34
:10715000C76AD4ED567AA6EE267A77EE676A84ED92
:10716000577AE6EE267AC4ED567AC4ED557A0FB119
:10717000C4ED507AD4ED596A94ED5B7A9FED9B5A39
:1071800094ED5C6AC4ED597A77EEE66AF0EE475A00
:10719000D6EE855AF0EE477AE6EE257A94ED5A0A55
:1071A000C4ED5B7A37EEC07AA6EE070A84ED5A0A80
:1071B0003EF0C2FE02B282EAE273A3EBE2739BB23C
:1071C000092B7ED9002AACBF0A380A3005B20E2E30
:1071D000A4F8745160D0242E09D1DFED857A94EDA6
:1071E000500A20EE270A3EF0A7FE824B5880BDECE5
:1071F000048BF8BD84F83A3184F839317BE7D4ED5B
:10720000447AB4F81431F8EEE77AC4ED417A002BF1
:1072100000F08A8007EE903ADFED746A9FED767A8F
:10722000F8EEE77A86EEA78AB4EEC78AF1EE10FA96
:1072300088BFB0EE478A94F8383113F001034FF05D
:1072400001053FF454AF94F83931002B56D094ED3A
:10725000519A78EEC99A002D3AD094F83A31002B21
:1072600054D0D4ED417A94ED520A5F4B1E7877EEFC
:10727000C07A0E2EC4ED557A5FD094F84C31002BB5
:1072800075D0022B02D00FB1012B31D0D4ED557A3D
:10729000F0EE698A012756E7DFED547A554C9FEDF1
:1072A000540A28EE278A28EE800ABDEEC88A18EE16
:1072B000103A23803EF040FEBDEC048B6080E580F8
:1072C000F8BD002583E7444C0127D4ED3D8AFDE657
:1072D000454B1E780E2E2AD094F83A519FED3D8AE8
:1072E000002DCAD1002FD1D094F84C31002BCBD136
:1072F000F0EE697A0127F0EE698A24E794ED4F9A5F
:10730000012384ED519A84F83931A2E7002F56D039
:10731000D4ED417A37EEE80A012330EE090A84F809
:107320003A3184ED520AA0E79FED2C8A83E7D4ED31
:10733000557A94F83A519FED278A9FED2D0A27EE52
:10734000800A3EF0F9FD2B4B0E269880C8E7DFED52
:107350002B7A94ED417A274B27EE277A0027BDEE52
:10736000C77ADFED1C7A17EE102A9A80EBE6002F21
:107370008CD094ED556A94F84D31DFED216A07EE1B
:10738000903A76EE688AB8EEE77A78EE897AF0EE8F
:10739000698AF0EEE77A67EE877AF4EEE67AF1EE44
:1073A00010FAC4BF68EE266A86EEA78AF7EE007A66
:1073B00077EEC87A67EEA97AE6EE087AC3E60A4B5A
:1073C0001E780E2E7FF462AFD4ED557A3D46B4E7B9
:1073D000F8E600200000000028F500209A99993E68
:1073E000CDCC4C3FCDCC4C3E732B00200000C8428E
:1073F000CDCCCC3D742B00206666663F0AD7233C7B
:1074000000401C46F8B54569002D67D02C68236AFA
:107410001B7B002B40F09080D4E9041763684E6812
:10742000002F3ED030687A686FF30000306010683B
:107430006FF300001060087C0E68022202FA00F16F
:1074400041F00C017160397C8A40396842F00C02CD
:107450004A605A686FF341025A605A686FF300023B
:107460005A60236A1B697BB1236A686C1B69984761
:10747000012800F09D80022801D005E02362236AE4
:10748000DA691433002AF9D1236ADA693ABB5869F8
:1074900018B399692162C3E90522BDE8F840F3F702
:1074A000D1BA9A681006FCD49A68D20713D430680F
:1074B0006FF300003060087C09680222824042F0CD
:1074C0000C024A605A686FF341025A60236A1B69D2
:1074D000002BC9D1D8E7DA68E6E72062F8BD226A56
:1074E00094F82410127B1433D2B22362002932D1D3
:1074F000002A51D12846F3F7BDF929680A6AD369F1
:10750000002BEBD0D06953698C69002B4BD001263E
:1075100066732D68636083B2686963810028DDD07B
:1075200092693C48C969002A0ABF0246012000202E
:1075300048734A604B81F8BDAB68002B3FF46CAFD9
:10754000D4E904171A689B8893614E686368002F1A
:107550007FF468AFA5E72E68376AB069B9683B6801
:10756000002B48D04FF0010C80F80DC043608BB267
:1075700029684381496951B1F06979684381254B94
:1075800000290ABF194601230023416043730023E9
:1075900084F82430002AADD0AB68002BAAD01A683A
:1075A0009B889362A6E71E461B4BFF271F70AFE721
:1075B000236A2968143B23620A6AD369002B3FF4CB
:1075C00063AFD66953698F69E3B1844687F80DC00C
:1075D0007B60B3B22E687B817669002E3FF454AF96
:1075E000C96992694B810B4B002A04BF00201A46DF
:1075F00048734A6048E79C46074B4FF0FF0E83F8FC
:1076000000E0B1E79C46044B4FF0FF0E83F800E02A
:10761000DCE700BFF83B00201A0100208160F5F78D
:107620004DBC00BF0171F5F749BC00BF244B82B0CF
:107630009A79019092B393F82630DFED226A224ABC
:1076400007EE903AF8EEE77A204B127886EEA77AAA
:1076500083ED717A02B3B3F88211DFED1D6ADDEDBF
:10766000017A07EE101AB8EE477AF8EE677A27EE3D
:10767000267AF7EE006A27EE277A03F5C27377EED3
:10768000266A0021C7EE267A03EBC202196008338E
:1076900043ED017A9A42F9D102B070470D4A12685F
:1076A0001201F9D593F82630DFED066A07EE903A1D
:1076B000F8EEE77A054B86EEA77A83ED717AEBE771
:1076C0007C3C002055555540805D002028F5002069
:1076D00027D4D236885C002010B5437B82680446EC
:1076E000581C6073D154627B237B934206D82AB125
:1076F0002368D4E9010198470023637310BD00BFDC
:10770000427B42B110B503680446D0E901019847B5
:107710000023637310BD7047F0B506683578012DFE
:1077200093B0044607D0022D02D1356A002D3BD01C
:10773000002013B0F0BD96F90460771CF8D0032E3A
:10774000F6DC5C4F4FF0540C0CFB067CDCF81800A8
:107750000028EED09BB22479CCF830508CF834500D
:10776000ACF82C3000238CF83630CCF824208CF880
:10777000363040F67103826915044FD4542303FB5D
:10778000067393F83630DBB2002B5DD0542303FB35
:107790000673012283F8362093F83600C0B2002821
:1077A0005BD1012013B0F0BDCDE908230DF1070333
:1077B00002930123CDE9035361F07F018DF8283056
:1077C0008DF83C3000220023CDE90655CDE90C238D
:1077D0008DF807108DF814500B950E951095EFF35A
:1077E0001185102383F3128803681B6A002B59D07C
:1077F000049B02A802461BB1D3691432002BFBD1B3
:10780000336ACBB1996839B9934215D0196889B1F7
:107810005B6899680029F7D01433F3E7013BAAD1DC
:10782000542303FB0673122283F8362093F8363074
:10783000DBB2A9E7C3E90040EDB285F31188226805
:10784000136A002BFCD1ACE7542000FB06700A46FB
:10785000183061003AF09CF9A1E7542303FB06734A
:107860000022996983F8362040F671038A699206EE
:107870000DD5542303FB067696F836300E4A2023A6
:10788000CB61138801339BB20020138051E7013B89
:10789000ECD1542303FB0676122386F8363096F893
:1078A0003630EBE702AB3362EDB285F31188F3F7C4
:1078B000C9F8C4E7A83A0020ACEE002030B593B078
:1078C0000DF1070508920022CDE90252CDE906220A
:1078D0008DF807108DF81420012109930B920E9258
:1078E00010920023002204918DF828108DF83C108E
:1078F000CDE90C2301680446EFF3118C102383F3C8
:10790000128803681B6A0BB3049B02A802461BB1D2
:10791000D3691432002BFBD10B6A6BB1996839B96A
:10792000934209D0196829B15B6899680029F7D09A
:107930001433F3E7C3E900405FFA8CFC8CF3118841
:107940002268136A002BFCD113B030BD02AB0B626E
:107950005FFA8CFC8CF31188F3F774F8F0E700BF42
:1079600030B40568EFF3118C102383F31288036899
:107970001B6AEBB18B6804460A461BB1D36914320B
:10798000002BFBD12B6A6BB1986838B9934209D0B0
:10799000186828B15B6898680028F7D01433F3E7BB
:1079A000C3E900415FFA8CFC8CF3118830BC70474E
:1079B00029625FFA8CFC8CF3118830BCF3F742B873
:1079C00030B58BB04FF0010C00910021CDE90123BF
:1079D000CDE90411CDE9061105688DF80CC0044607
:1079E0008DF820C00991EFF3118C102383F31288D6
:1079F00003681B6A0BB3029B684602461BB1D3693E
:107A00001432002BFBD12B6A6BB1996839B99342C0
:107A100009D0196829B15B6899680029F7D0143337
:107A2000F3E7C3E900405FFA8CFC8CF3118822680D
:107A3000136A002BFCD10BB030BDC5F820D05FFA23
:107A40008CFC8CF31188F2F7FDFFF0E730B593B0B2
:107A500000238DF807108DF806200DF10601012294
:107A6000CDE90332CDE90631CDE908320DF1070544
:107A70008DF814308DF828208DF83C200B930E9350
:107A8000109300220023CDE90C23016802950446DF
:107A9000EFF3118C102383F3128803681B6A0BB376
:107AA000049B02A802461BB1D3691432002BFBD100
:107AB0000B6A6BB1996839B9934209D0196829B139
:107AC0005B6899680029F7D01433F3E7C3E90040F5
:107AD0005FFA8CFC8CF311882268136A002BFCD1AE
:107AE00013B030BD02AB0B625FFA8CFC8CF31188D3
:107AF000F2F7A8FFF0E700BF30B595B000230122F0
:107B0000CDE90532CDE908338DF81C300D93109383
:107B100012930DF10F030DF107050B928DF8302034
:107B20008DF844200A93002200238DF80710CDE938
:107B30000E23016804950446EFF3118C102383F3A0
:107B4000128803681B6A1BB3069B04A802461BB17C
:107B5000D3691432002BFBD10B6A6BB1996839B928
:107B6000934209D0196829B15B6899680029F7D058
:107B70001433F3E7C3E900405FFA8CFC8CF31188FF
:107B80002268136A002BFCD19DF80F0015B030BDA0
:107B900004AB0B625FFA8CFC8CF31188F2F752FF96
:107BA000EEE700BF154A164B90421B6828BF1046EF
:107BB000B0EB930F14D2B0EBD30F13D2B0EB131F73
:107BC00012D2B0EB531F11D2B0EB931F10D2B0EB17
:107BD000D31F0FD2B0EB132F0ED24FF4807070472B
:107BE000022070470420704708207047102070471B
:107BF00020207047402070478020704700512502A8
:107C000000000020013903292CD81B4B4FF0280C11
:107C10000CFB01FC10B403F5E4746344644493F872
:107C2000C82104604FF0010C022A80F838C003F527
:107C3000E47419D0C9B2114A09015258C3F8CC21D1
:107C400072B1022283F8C82100F110014FF4807252
:107C50002430A281C3E9781060465DF8044B704778
:107C60000020FAE70020704793F8D521624460466F
:107C700083F8D521F1E700BF28F500203C3C002027
:107C80002DE9F04FDFF88482DFF884B29C4C85B098
:107C90004FF0010A4FF0000998F80030022B0DD088
:107CA00009F10109B9F1040F0AF1010A08F12808E4
:107CB0000BF1050BF0D105B0BDE8F08F9BF9035037
:107CC0006A1C00F0E480EDB228465FFA89F30D2DBE
:107CD00062D88C4A002104E00131202902F103021C
:107CE0005AD01778002FF7D156789E42F4D1854AA2
:107CF000854E01EB4101114405EB4502897806F8F8
:107D0000221006EB82026E009160526861688A421E
:107D100000F0CF80A16A8A4200F06281E16C8A4261
:107D200000F06281216F8A4200F06781D4F89410DC
:107D30008A4200F06C81D4F8B8108A4200F0758154
:107D4000D4F8DC108A4200F06C81D4F800118A4229
:107D500000F07281D4F824118A4200F07681D4F8C0
:107D600048118A4200F06C81D4F86C118A4200F00C
:107D70007E81D4F890118A4200F07481D4F8B41155
:107D80008A4200F08181D4F8D8118A4200F08181C2
:107D900014F80C2C002A7DD00135EDB2854296D91D
:107DA000002301939BF904506B1C79D0EDB22E4651
:107DB0005FFA89F20D2D62D8524B002104E00131A7
:107DC000202903F103035AD018780128F7D15F78EE
:107DD0009742F4D14B4B4C4F01EB4101194405EB59
:107DE0004503897807F8231007EB83034FEA450E14
:107DF00099605B6861688B4200F08C80A16A8B425D
:107E000000F0F680E16C8B4200F0F480216F8B4231
:107E100000F0F780D4F894108B4200F0F580D4F88D
:107E2000B8108B4200F0FA80D4F8DC108B4200F0DE
:107E3000F280D4F800118B4200F0FB80D4F82411BA
:107E40008B4200F00B81D4F848118B4200F0028184
:107E5000D4F86C118B4200F01381D4F890118B424E
:107E600000F00A81D4F8B4118B4200F01B81D4F8E1
:107E7000D8118B4200F0128114F80C3C9BB10135F3
:107E8000EDB2AE4296D20023C8E9043308E70D20D4
:107E900000251AE7142204F80BAC04F80C2C7BE73D
:107EA0000D26002584E7132304F80BAC04F80C3CE2
:107EB000E5E73A46BC460CEBCC0104EB81070CF13C
:107EC000010197F818C0019107F11801BCF1000FEA
:107ED0007FF462AF142322440B70019887F819A035
:107EE000C8F81020F3F7CAF807493A6A731901EB8A
:107EF00083039968136861F30603136052E700BFB8
:107F00001C0100205079050814030020F0F6002021
:107F1000D06500200021084600EBC00304EB83037A
:107F200001301F7E03F1180C002FA8D11322214429
:107F3000764683F819A08CF80020C8F81410039333
:107F40000290F3F79BF833462B441D46039B1A6AB5
:107F5000564B03EB85039968136861F306031360BE
:107F6000DDE90130002B8ED0D8F8142053681D684D
:107F700067F300051D60137CD8F810501268D5F81F
:107F800004C0022101FA03F343F00C035360DCF850
:107F900000E067F3000ECCF800E095F810C02D6803
:107FA00001FA0CF141F00C016960D8F81850102664
:107FB000C5E902672F82D8F804106F600C31296080
:107FC000D8F81C503B46C5E90017C5E90277384987
:107FD0002F823A46F3F770F8012388F80C305FE6F9
:107FE00024224FF0010C66E748224FF0020C62E7B2
:107FF000242191E7482102208EE76C224FF0030CE8
:1080000059E76C21032087E79021042084E7902220
:108010004FF0040C4FE7D82106207DE7B42105205E
:108020007AE7D8224FF0060C45E7B4224FF0050C52
:1080300041E7FC2107206FE7FC224FF0070C3AE7ED
:108040004FF4A2724FF0090C35E74FF490724FF0E5
:10805000080C30E74FF4A27109205DE74FF49071EE
:10806000082059E74FF4C6724FF00B0C23E74FF48A
:10807000B4724FF00A0C1EE74FF4C6710B204BE7A9
:108080004FF4B4710A2047E74FF4D8724FF00C0C4C
:1080900011E74FF4EA724FF00D0C0CE74FF4EA7160
:1080A0000D2039E74FF4D8710C2035E71403002078
:1080B0000574010810B5036804469B689847FF23C0
:1080C0000122A373627310BD036810B504461B68D8
:1080D0009847236801219B6820469847E37B01333A
:1080E000E37310BDF0B583B00446089F0193384692
:1080F00016460D463CF0D8FA2268E6722844A07273
:108100009769019B324629462046BC4603B0BDE82C
:10811000F040604703689B6A184700BF03685B6DC7
:1081200003B11847704700BF0368DB6C03B1184701
:10813000704700BF002310B5C37342748A6C01609E
:10814000044603730AB119469047236801219B68CE
:1081500020469847FF222368A273DB6C01226273DA
:108160001BB12046BDE81040184710BD4A484B4996
:108170004B4BDFF830C12DE9F04F4FF0010A4FF0C3
:1081800002094FF0040808271026202540244FF04C
:10819000800E30F8022F12F0010F03D01960A3F8FF
:1081A00004A0083312F0020F03D01960A3F8049062
:1081B000083312F0040F03D01960A3F804800833C9
:1081C00012F0080F02D019609F80083312F0100FD0
:1081D00002D019609E80083312F0200F02D019607F
:1081E0009D80083312F0400F02D019609C80083344
:1081F00012F0800F03D01960A3F804E0083312F4E2
:10820000807F05D04FF4807B1960A3F804B0083359
:1082100012F4007F05D04FF4007B1960A3F804B07E
:10822000083312F4806F05D04FF4806B1960A3F807
:1082300004B0083312F4006F05D04FF4006B1960DE
:10824000A3F804B0083312F4805F05D04FF4805BCC
:108250001960A3F804B0083312F4005F05D04FF49E
:10826000005B1960A3F804B0083312F4804F05D006
:108270004FF4804B1960A3F804B00833D20B04D03C
:108280004FF4004219609A80083301F5806161451E
:108290007FF47FAFBDE8F08F7E7B050800000240D1
:1082A000EC3700200020024010B50409013C072CE7
:1082B00016D80D4A32F8141000F00F0341FA03F2F9
:1082C00012F001020ED001209840013808403CF025
:1082D00017FF064B064A1B5D184402EBC00010BD99
:1082E000002010BD104610BD807B0508907B05085E
:1082F000EC370020F8B50C4F97F834308BB10B4CAD
:108300000025A66830790135FFF7CEFF18B1217D31
:10831000F279F3F78DF897F83430AB4204F14C045E
:10832000EFDC0120F8BD00BF88440020941A002033
:1083300038B5054600780C46FFF7B6FF611CC9B298
:10834000044610B141238371C17120466978F2F768
:10835000E9FFAB7820461BB1BDE83840F2F7F6BD27
:10836000BDE83840F2F7F8BD2DE9F041FFF79CFF7A
:108370000C4B0D4E1F6805460024BC4201DBBDE8D6
:10838000F08104EB440303EB0608F05CFFF78CFF7D
:10839000854204D121464046BDE8F041C8E701349A
:1083A000EBE700BF20660020F0650020054B53F886
:1083B000203033B11A689B8851690B4218BF1B04E7
:1083C00093617047802A00200C4B0D4A93F800C03F
:1083D00052F820200123834003EA0C0341B1003B03
:1083E00018BF01231AB1918833B11368996170479E
:1083F000B3FA83F35B09F5E70904F6E78C2A00205A
:10840000802A002010B5054C23681B699847236813
:10841000002283F836209A6310BD00BF2C6A00202A
:1084200010B5084C236893F8352012B1DB689847E3
:1084300000B910BD044A236812689A63012183F8C9
:10844000361010BD2C6A0020782A00200D4A02EB5D
:10845000C00310B593F86CE293F86D428EEA010CFC
:10846000644500D110BDD3F86832C0002BB19C88A0
:108470001B688E4508BF24049C61104480F86DC2BF
:1084800010BD00BF28F500202DE9F0411D4D1E4F05
:1084900082B000246E46A5F5227815F8013BFF2B2B
:1084A00017D097E8030003F108020DEB020C86E8F1
:1084B000030001229BB1072B15D81CF8083C9A40F9
:1084C000B8F88C321A4214BF012100212046FFF770
:1084D000BDFF0134042CE0D102B0BDE8F08198F872
:1084E00038111140F2E75A0908EB820203F01F032A
:1084F000D2F89012012202FA03F30B4214BF114684
:108500000021E3E7B0F700204CB505082DE9F04164
:10851000104E114D01244FF05208532716F8010B4D
:10852000FFF7C2FE282120B1C47180F80680F2F75F
:10853000CBFE15F8010BFFF7B7FE482118B1C47147
:108540008771F2F7C1FE0134E4B2052CE6D1BDE833
:10855000F08100BFF4700020E870002038B50C46B0
:1085600014F8011B41B105462B6828461B68984743
:1085700014F8011B0029F7D138BD00BF03681B6840
:10858000184700BF03682DE9F0415F6A1FB13B4601
:10859000BDE8F041184704460D46164600E0236842
:1085A0009B6820469847B042F9D3002E08DD2E4440
:1085B000236815F8011B1B6820469847B542F7D180
:1085C000BDE8F08103685B68184700BF03689B68DB
:1085D000184700BF0368DB68184700BF03685B6982
:1085E000184700BF03689B6A03B11847704700BF74
:1085F0000368DB6A03B11847704700BF03682DE9C1
:10860000F04116469A6A04460D460AB1904723681F
:108610005F6A5FB1324629462046B8472368DB6A65
:10862000C3B12046BDE8F041184723689B68204647
:108630009847B042F9D3002EF0DD2E44236815F898
:10864000011B1B6820469847B542F7D12368DB6AB7
:10865000002BE6D1BDE8F08170B504460E46154604
:10866000236820469B689847A842F9D32A4631469A
:108670002046BDE87040C1E72DE9F04F8E4B1E78D3
:108680008FB016B10FB0BDE8F08F8C4F3B68590525
:10869000F8D58B4D9FED8B7AD5F8C434C31A07EE0D
:1086A000903AF8EEE77A0446F4EEC77AF1EE10FA63
:1086B00059DA95F8C834002BE4D095F8CC349A07F1
:1086C000E0D195F8D424002A52D0D5F8D80410B1BE
:1086D0007D49FFF793FF002385F8D43495F81C35C6
:1086E000002B49D195F8F036002B40F0FD8095F82D
:1086F0007B24002A40F07C81744B196895F8F13690
:108700002BB17348D5F8F436834200F0AF8195F869
:108710002027704BB3FBF2F3D5F8EC2613449C42B0
:10872000B0D395F82937C5F8EC462B4493F8244785
:10873000E30700F18183A60700F12983600700F1B8
:10874000FA82230700F19D82E70600F1838295F803
:10875000293795F820270133B3FBF2F102FB1133DF
:1087600085F829378EE723F0E5F8C5F8C444A0E77B
:1087700095F81C35002BB5D095F81D35002B40F031
:10878000FF81D5F88035002B00F02D81DFF8508176
:10879000DFF850B108F168094B460027A146A8F55B
:1087A000227A1C4662E0012900F03681052E4ED95E
:1087B000537885F8E43690885388A5F8E036911D03
:1087C0009319C02800F2358200220AEB000EA5F8AA
:1087D000E2264148C5F8D8A60122C5F8DCE685F8AE
:1087E000E826AEEB00025B1A934285F8E9C6C0F2B8
:1087F0001582002A40F0CA81384AC5F8DC060023F9
:1088000085F8E836C5F8D0360693DBF80400C5F8DD
:10881000D8A606AB02F11001C5F8C846C5F8CC26AB
:1088200008F0CCFD013000F02482069B0BB1002043
:108830009847D5F8C836C5F8CC36C5F8C84695F877
:10884000D434002B00F0FA80012385F81D35013661
:108850003744EFF31183502282F31288D5F8802534
:10886000974280F2B780DBB283F31188EB1993F85B
:108870002065012EEBD97A1CAB1893F82035C3F391
:108880004111032985F8841503F00F0C00F0DB80FB
:1088900013F01003424486D195F8E8160029D6D08B
:1088A00095F8E916013101F00F01614500F0D7801C
:1088B00085F8E836CBE700BFF0E60020885C0020B2
:1088C00028F50020001B374A04FA0020782A0020EF
:1088D00020FC0020A0860100C0F70020F0FB002053
:1088E00048FA0020F8040020BF4BC0490091A3F1D2
:1088F0003F02C827BE4904920593BE4ABE4B85F885
:10890000847406A8F5F7FAFFDDF81080002608F158
:108910000103049388F80060049B2922591C0491E8
:108920001A70049BEA22591C04911A70049B5A1C69
:10893000049206A81F703BF0B7FE471C06A93A46F2
:1089400004983EF095F804990122CB19134404933E
:10895000CE55049B991804911E70049B991804919C
:108960001E70049B991804911E70049B9918049121
:108970001E70049B991804911E70049B9918049111
:108980001E70049B991804911E70049B9918049101
:108990001E70049B991804911E70049B99180491F1
:1089A0001E70049B991804911E70049B99180491E1
:1089B0001E70049B991804911A70049BA3EB080382
:1089C00004A888F8003031F043FF85F8F066C5F858
:1089D000EC4657E600224C4695F81D65C5F8802503
:1089E000DBB283F3118885F81C65C5F8EC4649E6CF
:1089F000824A85F87B3402F13A03CDE906238049A7
:108A0000C5F884144FF4327306A8A5F8883431F001
:108A10001FFFC5F8EC4635E6022E3FF418AF50783C
:108A20009378A5F8E036FF2840F0DB80042E7FF62F
:108A30000EAFB2F80300511D9319C2E635F02AFEBD
:108A400085F81D0503E76F4BC5F8CC366E4BC5F8AE
:108A5000D0360023C5F8C84685F88835EFE6D5F846
:108A6000D806D5F8DCE6511C9319BAE6D5F80C0700
:108A70008842BFF44CAE95F87814002940F08E80FF
:108A8000D5F81067002E3FF442AED6E900218A42A5
:108A90003FF43DAED5F81837D5F81C27E31A9342BA
:108AA0007FF735AE95F8143795F8152785F88A3491
:108AB000564B0392114603F13802CDE90632544A6F
:108AC000C5F884244FF4E47285F88B14A5F8882443
:108AD000D6E90019494500F01584984603F1320B98
:108AE0000F78ABEB080A09F1FF3E0B46C1F1010C10
:108AF00003E013F8012FBA4203D173450CEB0300D6
:108B0000F7D183B2012B5FFA8AFA00F267839A45A4
:108B100080F09683494500F0F583D845E0D3039B68
:108B20007BB995F88A3463F07F0385F88A34D6E9F7
:108B30000019494505D195F88A3443F0400385F87A
:108B40008A34069B334E06A89B1B85F8853431F08A
:108B50007FFE95F8D4244AB1D5F8D80418B106F1AF
:108B60005701FFF74BFD002385F8D43495F81537EE
:108B7000C5F81847013385F81537C5F8EC4681E587
:108B800035F088FD85F81D0506462CE703923DF07B
:108B90006FFFD5F8D806039A10442DE695F8141700
:108BA00085F8782485F815271B4A013182FB0102DC
:108BB0000A445211C2EB82128A1A95F8790495F888
:108BC0007A1485F81427A3F5687200FB0121A3F538
:108BD0001F73C5F87C24C5F88014C5F810371E46ED
:108BE00055E7D11C9319ECE5ECF90020035B00205C
:108BF000384906082C49060824490608B2F900201D
:108C0000C8057DEAB1FA00200000F6FFB4F90020A3
:108C1000C8007DEAADF90020832008821A4603933C
:108C20003DF026FFD5F8D826039B1344C5F8D83667
:108C30000DE6774BC5F8CC36B5F8E036A5F8D0365A
:108C4000032385F888354FF6F673C5F8C846A5F8AE
:108C5000D236F4E56F4B7048C5F8840403F13B014C
:108C6000C82206A80693079185F8882431F0F0FD04
:108C70006DE5D5F8C8360222591CC5F8C8161A7019
:108C8000D3E5D5E94201B5F82A31B5F82C2185F8AC
:108C90008A04242707FB03F3070E85F88774070C63
:108CA00085F8887402EB820264273233B3FBF7F352
:108CB00085F89034C3F3072385F88F34000A5300F6
:108CC00085F8890485F89234080E41F2C81385F8B6
:108CD0008E1485F88B04C2F3C712080CA5F88434EF
:108CE000090A02234D4E95ED500A079685F8912406
:108CF00085F8863485F88C0485F88D143DF01CF9D0
:108D0000474A03469342A8BF134623EAE373B3FBE3
:108D1000F7F303F57A73C3F307222E3E85F8932405
:108D200006A895F82E21069685F8952485F89434A2
:108D300031F08EFD08E5394B95F838910793C8223C
:108D4000A3F13D08A5F8842419F001094FF0210290
:108D5000CDF8188085F8862400F09A82B5F88C2228
:108D6000500540F189822F4A393B1068C5F88704C5
:108D70000693069B0022591C06911A70069B2A4AEC
:108D800006A89B1A85F8853431F062FDD9E4234AA0
:108D9000079295F83F3740F6C822A5F884240822A8
:108DA00085F88624002B00F05A82204B1B781BB1DB
:108DB0001F4A1288B2FBF3F30A220533B3FBF2F326
:108DC000C3F3072285F8872485F88834D5F8583707
:108DD000184E06960A2293FBF2F3C3F3072285F896
:108DE0008A3485F889240EF0E5FEB5F860870346DD
:108DF00098FA98F8043685F88E3406A8B5F86237E4
:108E0000A5F88C84069685F88B3431F021FD95E425
:108E1000B1FA0020B1F90020C8040B00ECF90020E1
:108E200020A107004C490608ADF9002099EE00206A
:108E30009CEE0020B3F900209F4AB5F92E37079227
:108E400040F6C802A5F88424B3F5E16F4FF01E0286
:108E500085F8862440F37C819AB2A2F561631BB247
:108E6000B3F5E16F31DDA2F5E1531BB2B3F5E16F6C
:108E70002BDDA2F52853303B1BB2B3F5E16F24DDA7
:108E8000A2F561531BB2B3F5E16F1EDDA2F58C4371
:108E9000503B1BB2B3F5E16F17DDA2F5A843603B71
:108EA0001BB2B3F5E16F10DDA2F5C443703B1BB2FA
:108EB000B3F5E16F09DDA2F5E1431BB2B3F5E16F54
:108EC00003DDA2F5FD43103B1BB207EE903A9FED88
:108ED0007B7AF8EEE77A67EE877AFDEEE77A17EEAF
:108EE000902AC2F3072385F88734B5F92C3785F823
:108EF0008824B3F5E16F40F3E5809AB2A2F561638F
:108F00001BB2B3F5E16F31DDA2F5E1531BB2B3F54E
:108F1000E16F2BDDA2F52853303B1BB2B3F5E16FB7
:108F200024DDA2F561531BB2B3F5E16F1EDDA2F59E
:108F30008C43503B1BB2B3F5E16F17DDA2F5A8439C
:108F4000603B1BB2B3F5E16F10DDA2F5C443703B8B
:108F50001BB2B3F5E16F09DDA2F5E1431BB2B3F536
:108F6000E16F03DDA2F5FD43103B1BB207EE903A23
:108F70009FED527AF8EEE77A67EE877AFDEEE77AB0
:108F800017EE902AC2F3072385F88934B5F93037F4
:108F900085F88A24B3F5E16F51DD9AB2A2F56163D9
:108FA0001BB2B3F5E16F31DDA2F5E1531BB2B3F5AE
:108FB000E16F2BDDA2F52853303B1BB2B3F5E16F17
:108FC00024DDA2F561531BB2B3F5E16F1EDDA2F5FE
:108FD0008C43503B1BB2B3F5E16F17DDA2F5A843FC
:108FE000603B1BB2B3F5E16F10DDA2F5C443703BEB
:108FF0001BB2B3F5E16F09DDA2F5E1431BB2B3F596
:10900000E16F03DDA2F5FD43103B1BB207EE903A82
:109010009FED2A7AF8EEE77A06A867EE877AFDEEEA
:10902000E77A17EE903AC3F3072285F88B24244A97
:10903000069285F88C3431F00BFCFFF77CBB13F5FE
:10904000E16FE3DA9AB202F561631BB213F5E16FE7
:10905000DCDA02F5E1531BB213F5E16FD6DA02F563
:10906000285330331BB213F5E16FCFDA02F56153A9
:109070001BB213F5E16FC9DA02F58C4350331BB212
:1090800013F5E16FC2DA02F5A84360331BB213F5A2
:10909000E16FBBDA02F5C44370331BB213F5E16F25
:1090A000B4DA02F5E1431BB213F5E16FAEDA02F573
:1090B000FD4310331BB2A9E7ECF9002058A08B4107
:1090C000B5F9002013F5E16FBFF650AF9AB202F583
:1090D00061631BB213F5E16FBFF648AF02F5E153D0
:1090E0001BB213F5E16FBFF641AF02F528533033E1
:1090F0001BB213F5E16FBFF639AF02F561531BB236
:1091000013F5E16FBFF632AF02F58C4350331BB25B
:1091100013F5E16FBFF62AAF02F5A84360331BB227
:1091200013F5E16FBFF622AF02F5C44370331BB2F3
:1091300013F5E16FBFF61AAF02F5E1431BB213F569
:10914000E16FBFF613AF02F5FD4310331BB20DE71D
:1091500013F5E16FBFF6B9AE9AB202F561631BB2C7
:1091600013F5E16FBFF6B1AE02F5E1531BB213F593
:10917000E16FBFF6AAAE02F5285330331BB213F5E8
:10918000E16FBFF6A2AE02F561531BB213F5E16FBA
:10919000BFF69BAE02F58C4350331BB213F5E16F63
:1091A000BFF693AE02F5A84360331BB213F5E16F2F
:1091B000BFF68BAE02F5C44370331BB213F5E16FFB
:1091C000BFF683AE02F5E1431BB213F5E16FBFF6C4
:1091D0007CAE02F5FD4310331BB276E610F0FF0CB7
:1091E00014BF0122002202EB13235FFA83FEBAEBC5
:1091F0004E0F47F080077246C0F2918001239AB16A
:10920000069901F1010ECDF818E00F7006999A4207
:1092100001F1010E03F10103CDF818E00BD881F83C
:1092200000C0EDD1D6F80490316811FA80F13160B8
:10923000DDF818806EE44FF0000E81F800E0DFE703
:1092400008F10103069388F800703368D6F804909B
:1092500013FA80F03060DDF8188001465AE4454B7F
:109260001B880A220533B3FBF2F3C3F3072285F808
:10927000872485F88834A9E5110526D53E4A3A3B6E
:1092800006931388A5F88734937888F8023070E540
:109290003A6811060FD595F8002102F00302032A5F
:1092A00009D0364A1068C5F88704393B591C2A2270
:1092B00006911A705DE5B5F88C2256050ED5304A38
:1092C000304B1068C5F88704F0E7D60511D52E4A53
:1092D000393B1068C5F8870406934AE5130516D58F
:1092E000254B1A88A5F887249A7888F80220274BFE
:1092F000DCE7D10719D5264A393B1068C5F8870441
:10930000069336E5039B002B7FF415AC09E4D705E3
:1093100020D51D4A1B4B1068C5F88704C6E7039B80
:10932000002B7FF406ACFFF7FCBB92071AD5194956
:10933000039108463BF0B8F90399064602464046B9
:109340003DF096FB08EB06030693B9F1000F7FF49E
:1093500010ADABE7D007E8D50D4A0A4B1068C5F849
:109360008704A3E795F864270B490C4B002A18BF24
:109370001946DDE79CEE00203C0306084449060838
:109380004C490608B3F9002054490608B2F90020F8
:109390005C490608144906081849060820490608C9
:1093A0002DE9F843456FC04F95F800C017F91CE050
:1093B0005FFA8EF30D2B044640F29B80006C002870
:1093C00049D0BA4E7368834200F00881B36A98426C
:1093D00000F06081F36C984200F06281336F984234
:1093E00000F06E81D6F89430984200F06B81D6F888
:1093F000B830984200F06A81D6F8DC30984200F02C
:109400006981D6F80031984200F06881D6F824319D
:10941000984200F06981D6F84831984200F068819E
:10942000D6F86C31984200F06581D6F890319842B8
:1094300000F06481D6F8B431984200F06581D6F826
:10944000D831984208BF0D2700F0C98016F80C3CAF
:10945000002B00F00E81E36B002B48D0934E726816
:10946000934200F08E80B26A934200F01581F26C54
:10947000934200F01381326F934200F01381D6F8CB
:109480009420934200F02081D6F8B820934200F057
:109490001F81D6F8DC20934200F01E81D6F800210F
:1094A000934200F01D81D6F824219A4200F01A81DF
:1094B000D6F84821934200F01981D6F86C219342E6
:1094C00000F01A81D6F89021934200F01981D6F865
:1094D000B421934200F01681D6F8D821934208BFF8
:1094E0000D234FD016F80C3C002B00F0CA80BDE8CD
:1094F000F8836F4B00211E461A4604E001312029F3
:1095000002F103023BD010780428F7D1507860456F
:10951000F4D101EB410131440EEB4E00654A8978EC
:1095200002F8201002EB80025068916021652064EF
:1095300007EB4C0797F9012001323FF440AF0022BE
:1095400005E00132202A03F103033FF438AF197814
:109550000529F6D159786145F3D102EB4202324434
:10956000544B92780EEB4E0E03F82E2003EB8E0E2A
:10957000DEF80430CEF80820E363E2641FE7206CD5
:10958000D6E7002303EBC30306EB83082A789F008A
:1095900098F818300132D2B2002BA8D1F059464BBE
:1095A00088F8192098420CBF362038200C2388F800
:1095B000183038F061FCF259D2F8003143F0010361
:1095C000C2F80031D8F82030E16C1A6861F3060265
:1095D0001A606B6804336366BDE8F883002707EB05
:1095E000C70706EB87080CF1010C98F818305FFAF2
:1095F0008CFCBF00002B7FF42EAFDFF8BC90F0593D
:1096000088F819C00B2348450CBF3620382088F84D
:10961000183038F031FCF359D3F8002142F0010240
:10962000C3F800214B450CBF36203820D8F8203035
:10963000226D196862F30601196095F82F9038F0D1
:109640001BFCF2591D49D2F8003143F00103C2F866
:10965000003198F91100C8F80C10C9F301124FEA53
:109660009911C8F8144033F05FFB6B68043323662C
:10967000F1E60B230CF1010C06F80C3C06F80BCCC0
:10968000E9E62B780C22013306F80C2C06F80B3C8B
:10969000BDE8F8830127A2E7012373E7022371E7FE
:1096A00002279CE703236DE7687000201C0100205F
:1096B00050790508140300200064024071B30008CB
:1096C00003278CE704278AE704235BE7052786E75F
:1096D000052357E7062782E7062353E707277EE798
:1096E00007234FE708234DE7082778E7092349E7D1
:1096F000092774E70A2772E70A2343E70B276EE777
:109700000B233FE70C233DE70C2768E7324B70B58E
:109710001D68EB6BAC6E002B3ED02368580605D558
:109720006FF04003236095F8856086B12B6C03B31E
:1097300023681A0744BF236863682368DB0605D5DE
:109740006B6B0BB19847AC6E2368636870BD95F87E
:109750007A00FEF7A9FDE36866F3C303E360012323
:1097600085F885300028E1D02821F1F7ADFDAC6EF9
:10977000DCE723681906DBD5D5E90923934216D027
:10978000AA692969D25C0133D2B26260B3FBF1F2FB
:1097900001FB1233AB62CBE723689E06BDD5EB6AB3
:1097A00053B16068296B80B29847AC6EB5E7E36847
:1097B00023F08003E360BBE76368EA696969DBB2B1
:1097C0008B54EB69EA68AC6E0133B3FBF2F102FB38
:1097D0001133EB61A1E700BFC4440020324B70B5E8
:1097E0005D68EB6BAC6E002B3ED02368580605D548
:1097F0006FF04003236095F8856086B12B6C03B34E
:1098000023681A0744BF236863682368DB0605D50D
:109810006B6B0BB19847AC6E2368636870BD95F8AD
:109820007A00FEF741FDE36866F3C303E3600123BA
:1098300085F885300028E1D02821F1F745FDAC6E90
:10984000DCE723681906DBD5D5E90923934216D056
:10985000AA692969D25C0133D2B26260B3FBF1F22A
:1098600001FB1233AB62CBE723689E06BDD5EB6AE2
:1098700053B16068296B80B29847AC6EB5E7E36876
:1098800023F08003E360BBE76368EA696969DBB2E0
:109890008B54EB69EA68AC6E0133B3FBF2F102FB67
:1098A0001133EB61A1E700BFC4440020324B70B517
:1098B0009D68EB6BAC6E002B3ED02368580605D537
:1098C0006FF04003236095F8856086B12B6C03B37D
:1098D00023681A0744BF236863682368DB0605D53D
:1098E0006B6B0BB19847AC6E2368636870BD95F8DD
:1098F0007A00FEF7D9FCE36866F3C303E360012353
:1099000085F885300028E1D02821F1F7DDFCAC6E28
:10991000DCE723681906DBD5D5E90923934216D085
:10992000AA692969D25C0133D2B26260B3FBF1F259
:1099300001FB1233AB62CBE723689E06BDD5EB6A11
:1099400053B16068296B80B29847AC6EB5E7E368A5
:1099500023F08003E360BBE76368EA696969DBB20F
:109960008B54EB69EA68AC6E0133B3FBF2F102FB96
:109970001133EB61A1E700BFC4440020324B70B546
:10998000DD68EB6BAC6E002B3ED02368580605D526
:109990006FF04003236095F8856086B12B6C03B3AC
:1099A00023681A0744BF236863682368DB0605D56C
:1099B0006B6B0BB19847AC6E2368636870BD95F80C
:1099C0007A00FEF771FCE36866F3C303E3600123EA
:1099D00085F885300028E1D02821F1F775FCAC6EC0
:1099E000DCE723681906DBD5D5E90923934216D0B5
